:020000040800F2
:100000000000011079CA07086D2B0008718E0208E4
:1000100019CB070819CB070819CB07080000000007
:100020000000000000000000000000007D48000803
:100030008148000800000000854800087107010899
:1000400019CB070819CB070819CB070819CB0708E4
:1000500019CB070819CB070839C900083DC90008A2
:1000600019CB070841C9000845C9000871320008CA
:100070008532000899320008AD320008C13200080C
:10008000D5320008E932000819CB070819CB070858
:1000900019CB070819CB070819CB070849C900086D
:1000A0001D310008453100086D3100080931000894
:1000B00095310008A9310008BD31000819CB0708A7
:1000C00019CB070819CB070819CB070819CB070864
:1000D00019CB0708F12C0008FD2C000819CB0708E4
:1000E0004DC9000819CB070889480008F9310008F4
:1000F0002132000849320008E5310008FD320008CD
:1001000019CB070811370008D131000819CB0708AF
:10011000092D000819CB070819CB070819CB0708C8
:100120001133000825330008393300084D33000827
:100130006133000819CB070819CB070819CB07084A
:1001400019CB070819CB070819CB0708D5480008B1
:1001500075330008893300089D330008152D000809
:1001600019CB070819CB070819CB070819CB0708C3
:1001700019CB070819CB070819CB070819CB0708B3
:0801800019CB070819CB070891
:10019000D0E907239A423CBFC1685218D01A704771
:1001A000D0E9092300699A4238BF1218D31A0138DE
:1001B000C01A7047D0E90902101AB0FA80F040095D
:1001C000704700BF0246036A4069D168C05C0133D2
:1001D0008B4228BF00231362704700BF436A8269C5
:1001E000D154436A0169426B01338B4228BF00231B
:1001F0004362D36843F08003D3607047436B188831
:1002000010F0100002D01A889B880120704700BFB0
:10021000436B99891A88890610B504460AD592B2AB
:10022000900607D5E26A002A2AD09888216B80B20E
:100230009047636B99891A88090692B210D5100607
:100240000ED5D4E909128A4215D0A1692069895CCA
:100250000132C9B29980B2FBF0F100FB1122A26217
:10026000998A1A88C90592B204D5D20744BF4FF6BD
:10027000F7721A8010BDDA6822F08002DA60EFE7C8
:100280009B88E2696169DBB28B54E269E168636B68
:100290000132B2FBF1F001FB1022E261CAE700BFBC
:1002A000036942681F2B10B40AD95468A3F1200CCB
:1002B000202101FA0CF1214207D15DF8044B70476F
:1002C0001468202199402142F7D081690024C86830
:1002D0000C7480684C68016821F00101016020689D
:1002E00094F805C00C4C818934F81C4089B221EA8D
:1002F00004011F2B818107D9A3F1200120238B400A
:100300005DF8044BD3607047202101FA03F35DF8D8
:10031000044B9360704700BF503C08084A1C10B45F
:1003200018BF4FF0450C494C08BF4FF0800C4FF4FC
:10033000003300E00BB3626B12EA0C0F03F1FF33E2
:10034000F8D0002924DD626B54071DD403291FD087
:100350003E4B5A6BD2071FD402291BD01A69D2B266
:1003600082421DD101295B691CD0062912D113F4E8
:10037000604F43D1364A13600CE0002904DD636B03
:100380005B0701D40329E3D103205DF8044B7047D8
:10039000002BF9D00020F8E701205DF8044B7047EE
:1003A0001020F2E72B4A1A40002AF3D0002B31DB51
:1003B0005C002DD4980031D4D9002DD41A0131D449
:1003C0005C012DD4D80137D419021DD45A02E7D4C8
:1003D0009C022DD4D80229D4190317D45A0323D44C
:1003E0009C0331D4D8032DD4190429D45A0425D41C
:1003F0009C041FD41807CDD51A20C6E7990405D44C
:100400005A04CDD41B04C5D50F20BEE71320BCE78A
:100410000920BAE71C20B8E70B20B6E70A20B4E7AA
:100420000D20B2E70C20B0E71420AEE71220ACE7B5
:100430001120AAE71920A8E70E20A6E71820A4E7B4
:100440001720A2E71620A0E715209EE7002C014008
:100450001020002008E0FFFDF8B5154DEB6A93B1C0
:10046000696B0129044614D0124BDA6A22F00802A3
:10047000DA6240F2FF5100229963EA62236823F0B6
:1004800001032360F8BD0B4AD36B43F48073D3633D
:10049000F8BD084E40F2FF570023B763B36040F247
:1004A0004C43F3600C20FFF739FFB763DCE700BF74
:1004B00010200020002C0140B14BD3E9011270B58F
:1004C0008C0F83F83840C1F3836483F83940C1F35B
:1004D000016483F83A40100EC1F3074483F83B40AF
:1004E0000001C1F30724C9B283F83C4083F83D10F2
:1004F000D887D98F93F89050C2F3035089B2014343
:10050000C2F30344D987C2F3C03083F84040C2F33A
:100510004031C2F3803483F84100012D83F842401A
:100520004FF0000083F84310C2F3003183F8441009
:10053000C2F3072CD96883F8450040F2D680022D1B
:1005400000F0B0802A204FEA4C0C0CF07E0C83F8AF
:10055000514083F852C093F85240C1F3C012144383
:100560001A6983F8524001F07F01D40F83F85310C9
:1005700083F85440910DC2F3417483F8554001F063
:100580000C01C2F3826483F8564083F8571093F845
:100590005710C2F381542143C2F3405583F85710DA
:1005A00083F85850002583F85950C2F3004583F86A
:1005B0005A50C2F3C03583F85B50C2F3803583F8DC
:1005C0005C50C2F3403583F85D505C69C2F300357E
:1005D00083F85E50C2F3812583F85F50C4F307416E
:1005E000C2F30125C2F3460283F860504FF0010CBC
:1005F00083F861200902220E83F862C083F8642028
:10060000A3F86610B3F86610C4F3072289B2114349
:100610002406A3F8661099699C669A6E0C0E42EA4D
:1006200004429A669C6E0A0A02F47F4222439A664A
:100630009D6EDA69C1F307242C43C9B29C6683F826
:100640006C10110E83F86D10110C090619671C6FE0
:10065000110201F47F0121431967196F120292B24E
:100660000A431A67196F1A6A41EA1261196793F807
:100670007410C2F30354214383F87410110A01F477
:100680007061A3F87610B3F87610C2F3072489B22C
:100690002143C2F34602A3F8761083F8782083F84A
:1006A00079C070BD120402F47C129A649A6C0C0E2C
:1006B00042EA04229A649C6CC1F3074222439A6482
:1006C0009A6C013240F10004A40244EA925492026E
:1006D000C3F880204FF40072C3F88440C1F3072CA4
:1006E000C3F88820C1F380342DE74FEA8C2C0CF43A
:1006F00040649C649C6C920002F47F7222439A6472
:100700009D6CC1F3C26445EA91759D6483F84C40C9
:10071000C1F3026483F84D40CA0BC1F3425483F81D
:100720004E4002F00602C1F3824483F84F4083F842
:10073000502093F85020C1F3C034224383F8502056
:100740009D6C93F8504093F840600234012202FA05
:1007500006F6A2404FEAE27EA2FB062406FB0E4408
:1007600005F1010EA2FB0E2E05FB04447444C3E9FF
:100770002024C1F3072CC3F88860C1F38034E2E67B
:100780001020002038B50D4B0D4C1A6840F2FF5573
:1007900040F24D43A5630121A2600D20E360FFF705
:1007A000BDFDA56340B96069C0F34320A0F104001A
:1007B000B0FA80F0400938BD002038BD102000207C
:1007C000002C01402F4B1A68910102D59A6D5207F7
:1007D0004BD42C4B1A68500202D5DA6E11063CD469
:1007E000284B1A68D20102D59A6D90072DD4254B5B
:1007F0001A68510102D59A6D120717D4214B1A6855
:10080000120112D59A6DD0060FD59A6D510334D4CA
:100810009A6DD20503D49A6D22F010029A65194B95
:1008200019484FF000629A6016E670479A6D5003BF
:1008300007D49A6DD10503D49A6D22F008029A6507
:10084000104B4FF080629A60D8E79A6D4FF080713C
:1008500022F002029A659960C9E7DA6E4FF48001CE
:1008600022F08002DA669960BAE79A6D4FF0007163
:1008700022F004029A659960ABE74FF000629A603B
:10088000704700BF0064024058640240384B5A6809
:10089000110303D5D3F8A02052075BD4344B5A6818
:1008A000D00303D5D3F8B420110649D4304B5A688D
:1008B000520303D5D3F8A020900737D42C4B5A68A5
:1008C000D10203D5D3F8A02012071CD4284B5A68B4
:1008D000920217D5D3F8A020D00613D5D3F8A020C4
:1008E000510341D4D3F8A020D20505D4D3F8A020D9
:1008F00022F01002C3F8A0201D4B1E484FF4001236
:10090000DA60A9E57047D3F8A02050030AD4D3F8E1
:10091000A020D10505D4D3F8A02022F00802C3F806
:10092000A020134B4FF48012DA60CFE7D3F8A02059
:100930004FF4802122F00202C3F8A020D960BDE765
:10094000D3F8B4204FF4803122F08002C3F8B420F1
:10095000D960ABE7D3F8A0204FF4002122F00402C5
:10096000C3F8A020D96099E74FF40012DA6070470D
:1009700000640240A064024082B00922274B8DF837
:100980000720DA68D00319D4DA68D10640D4DA68CF
:10099000D20541D4DA6812F0E00F3BD1DB6813F0E6
:1009A000020F0CBF092308238DF807309DF807308C
:1009B000012B0AD09DF8070002B0704701238DF883
:1009C00007309DF80730012BF4D1144A12E0D368A8
:1009D000DB0519D4D36813F0E00F17D1D36813F0F7
:1009E000020F0CBF092308238DF807309DF807304C
:1009F000012BDFD1D168C8034FF00103F4D4D368D1
:100A0000D906E4D50623EFE70223EDE70723EBE75A
:100A10000623D4E70723D2E70223D0E7003C0240B5
:100A2000704700BF704700BF704700BF012070478C
:100A3000034BD3E92503C01AC0F30A00704700BF77
:100A400010200020064AD2E925139942FDD0D11882
:100A50000133C3F30A0391F89C00C2F89830704741
:100A600010200020064BD3F89C0800B97047D3F83B
:100A70009C08A0F10500B0FA80F04009704700BF63
:100A800010200020012380F849307047044BD3E93F
:100A90002503C01AC0F30A00C0F50060704700BF0C
:100AA0001020002010B5D0F8E83504461B6998479F
:100AB000032384F81231002010BD00BF08B50422C2
:100AC00090F81211D0F8E83580F8131180F812214F
:100AD000DB689847002008BD08B5D0F8E435DB692D
:100AE00003B19847002008BD08B5D0F8E4351B6A6B
:100AF0009847002008BD00BF08B5D0F8E4355B6A10
:100B00009847002008BD00BF70B5037805460E4623
:100B10001446DBB101307BF02BF9431CDBB201330F
:100B20005B00DAB223800323327073702C7864B1D7
:100B30002846022300215A1CD2B2F454B15410F8B2
:100B4000014F0233DBB2002CF5D170BD02221346F7
:100B5000E8E700BF10B5074C2068FF2808D0064919
:100B6000D1F8A02801F6A40100F082F8FF23236049
:100B7000002010BD00000020102000204323014869
:100B80000B80704704000020122301480B8070473F
:100B900048000020042301480B8070475C000020BF
:100BA00010B5044C04480A462146FFF7ADFF204625
:100BB00010BD00BFBC280020FCE2080810B5044CA2
:100BC00004480A462146FFF79FFF204610BD00BF9C
:100BD000BC28002010E3080810B5044C04480A465D
:100BE0002146FFF791FF204610BD00BFBC28002022
:100BF00018E3080810B5044C04480A462146FFF7DC
:100C000083FF204610BD00BFBC28002024E3080855
:100C100010B5044C04480A462146FFF775FF2046EC
:100C200010BD00BFBC28002030E30808704700BF9B
:100C3000704700BF704700BF704700BF704700BFDC
:100C4000704700BF704700BF044B00200522C3F867
:100C50009C28C3F8AC09C3F8B009704710200020E5
:100C6000024B0020C3F89C08704700BF10200020F2
:100C7000212838B50C4625D0222816D0202812D19C
:100C800089B1072A0FD1174DD5F8B03913B10968CA
:100C9000002098472168A288A379C5F8B419A5F85F
:100CA000B82985F8BA39002038BD0029FBD0022ABE
:100CB000F9D10C4BD3F8AC39002BF4D009880020C3
:100CC0009847F0E70029EED0072AECD1054BD3F87E
:100CD000B419B3F8B82993F8BA392160A280A37186
:100CE000E1E700BF1020002010B4114CD4E92532F8
:100CF0009A1AC2F30A020A44B2F5006F14D879B105
:100D000001444A1E013810F801CFE118904203F166
:100D1000010381F89CC0C3F30A03F4D1C4F89430F2
:100D200000205DF8044B704702205DF8044B7047CB
:100D300010200020034B93F8E009003818BF012071
:100D4000704700BF1020002070B5124D124C29686A
:100D500040F2FF5640F24D430022A6630D20A160F1
:100D6000C5F8DC290121E360FFF7D8FAA66320B9B2
:100D70006369C3F34323042B08D0D5F8143AC5F8AC
:100D8000D039092385F8E039002070BD85F8E039B5
:100D9000022070BD10200020002C014070B50E4DC7
:100DA00095F8E039042B04460E460BD0082B07D1EA
:100DB000D5F8D83983420CD0FFF7C6FF022801D0FE
:100DC000012070BD082385F8E039C5F8DC69C5F855
:100DD000D849022070BD00BF10200020034B93F8BB
:100DE000E009032894BF0020012070471020002054
:100DF00000487047F429002030B4184B00209C7B39
:100E000014B11D688D4206D00130082803F110038B
:100E1000F5D130BC7047D2B1114B03EB40218A426F
:100E200011D0104B93F8B42112B9012283F8B421E8
:100E30000D4B01225A7000F5817003EB0013012263
:100E40009A7130BC7047022CEBD1183BF3E7064B8C
:100E500000F5817003EB00139A71DAE7F45C00206F
:100E6000F44C0020DC5C0020DC4C002030B41D4C35
:100E7000002384F8A03004F1180004E00133082BAB
:100E800000F110001ED005688D42F7D190F80EC019
:100E9000BCF1030FF2D1BAB1134901EB43208242F6
:100EA00009D094F8B42112B9012284F8B4210F4971
:100EB00001224A7000E0183903F5817301EB031138
:100EC00001238B7130BC70470849D4F89C2003F58E
:100ED000817301EB0313013204219971C4F89C2042
:100EE000F0E700BFDC5C0020F44C0020DC4C00206C
:100EF000A8B183681BB10E4B07229A7070470C4A49
:100F00001178D36003294FF0040014BF4FF48071AF
:100F10008021C2E901111361137590707047044A72
:100F200002F580510123537081F8B431704700BF3E
:100F3000DC4C002010B58121044679F061FD20468B
:100F4000012179F05DFD2046822179F059FDFFF7FE
:100F500087FE002010BD00BF034610B4D9691A698E
:100F6000002040F20114A3F844410860D1699C6D4F
:100F700021F002014FF0010CD161A3F89CC3206065
:100F8000D369044923F4003381F8180A5DF8044B4F
:100F9000D361704710200020202301480B80704748
:100FA00060000020122301480B8070478000002061
:100FB000042301480B807047940000200A4608B5BE
:100FC000054920B90548FFF79FFD034808BD0448BF
:100FD000FFF79AFD004808BD2C2A002040E30808CE
:100FE00058E3080810B5044C04480A462146FFF7A8
:100FF0008BFD204610BD00BF2C2A002070E308089E
:101000001C48D0F8E837D0F8EC2710B59B184FF003
:101010001A040C8001D1184810BD174AD0F8EA070D
:1010200002F1100411464FF0000E4FEA137CB3F1A9
:10103000204F34BF0CF1300C0CF1370C81F802C09A
:1010400081F803E002318C424FEA0313EDD102F143
:1010500008040021030FB0F1204F34BF3033373381
:101060009374D174023294424FEA0010F2D10248D4
:1010700010BD00BF00F0FF1F9800002010B5044C09
:1010800004480A462146FFF73FFD204610BD00BF39
:101090002C2A002084E3080810B5044C04480A46B2
:1010A0002146FFF731FD204610BD00BF2C2A00204D
:1010B00090E3080810B50E4C0E4BD4F8F41BB4F8AE
:1010C000F80B088303F1B402C4F8682DD3F8B430E8
:1010D0009847D4F8683D002BFBD01B69984700283F
:1010E000F7D0D4F8F43BB4F8F82B5A83002010BDA5
:1010F000102000200000002038B5084BD3F8683DD0
:1011000053B1DB6914460D4698474FF400730268EB
:101110002A600020236038BD1B68FFDE10200020FD
:1011200008B5064BD3F8683D23B11B6998470138D1
:1011300040B208BD4FF0FF3008BD00BF10200020B6
:10114000002070472DE9F041184CD4F8B80B154633
:10115000B4F8BC2B428323B30E4603EB050804E02E
:10116000D4F8683D0BB31B699847D4F8681DE1B10A
:1011700000234F681A4631462846B8470028EFD06A
:10118000D4F8683D002BFBD01B6998470028F7D0A6
:101190000135A84506F50076E7D1D4F8B80BB4F8C8
:1011A000BC2B02830020BDE8F081FEE71020002068
:1011B0002DE9F041184CD4F8B80B1546B4F8BC2B07
:1011C000428323B30E4603EB050801E01B699847F1
:1011D000D4F8681D51B10023CF681A46314628461D
:1011E000B847D4F8683D10B1002BEFD1002313B1FC
:1011F0001B69984710B9D4F8683DF8E701354545B3
:1012000006F50076E4D1D4F8B80BB4F8BC2B028311
:101210000020BDE8F08100BF10200020A14A5368E3
:1012200023F4FD4323F07F032DE9F04143F07603DF
:1012300053605368032123F48073536082B01160BC
:101240000FF0E2FA04460D460FF0DEFA001B61EBE8
:101250000501B0F57A7F71F10001F5D30FF0D4FAF2
:1012600004460D460FF0D0FA001B61EB0501B0F506
:101270007A7F71F10001F5D38A4C6368002040F257
:10128000FF5543F480734FF4806263604FF0FF3189
:10129000A563A060E260FFF741F8A563074618B1B7
:1012A000012002B0BDE8F0814FF4D5724FF489639C
:1012B000A5630721A2600820E360FFF72FF8A5636C
:1012C00028B9794B012283F890204FF08047754C64
:1012D00040F2FF55002240F27743A5630121A2604E
:1012E0003720E360FFF71AF8A5630028D8D147F04C
:1012F00000470646804647F4801701E09642CFD06B
:1013000040F27743A5630121C4F808803720E360E9
:10131000FFF704F8034640F2694203212920A56340
:10132000002BBDD1A563A760E260FEF7F7FF013691
:101330004FF6FF72A5630028B2D16369002BDDDA96
:101340004FF6FF729642ABD05D0000F1B380236888
:101350009807A5D0544D95F89060042E40F0B280C7
:10136000FFF7AAF800289BD14E4C2B6840F2FF579C
:10137000A763A36040F24743E36001210720FEF723
:10138000CDFFA763636823F4FD4323F07F0363600D
:10139000002885D1022E83D8636913F000737FF48F
:1013A0007FAF009308264FF48A63A7630121A660EC
:1013B0001020E360FEF7B2FFA76300287FF470AF50
:1013C0002B68A763A36040F27743E36001213720D5
:1013D000FEF7A4FFA76300287FF462AF334A62627E
:1013E000A662E26A42F03302E26240F27342A7630D
:1013F0000121A060E2603320FEF790FFA763002880
:101400007FF44EAF6B4640F22A4206E0616B8902E0
:1014100044BFD4F8801043F8041B616B1142F5D02F
:10142000636B1B073FF53CAF636B9F073FF538AF1E
:10143000636B9E063FF534AF636B98023FF530AFA8
:10144000009B1BBA59037FF52BAF2A6840F2774304
:1014500040F2FF55A5630121A2603720E360FEF74B
:101460005DFFA56300287FF41BAF022240F24643D4
:10147000A5630121A2600620E360FEF74FFFA5638C
:1014800000287FF40DAF63681A0509D4054A08499E
:1014900053680B4043F40063536053681B05F7D552
:1014A0000020FEE6002C01401020002000E1F505A0
:1014B0000081FFFF274D022685F8906023689C0776
:1014C0003FF4EEAE244C40F2FF570023A763022105
:1014D000A36040F2C243E3600846FEF71FFFA76324
:1014E00000287FF4DDAE63696B61A369AB61E369DA
:1014F000EB61236A2B62022E1BD9062E19D0164CE3
:101500002B6840F2FF57A763A36040F2C943E36032
:1015100002210920FEF702FFA76300287FF4C0AE76
:1015200063696B60A369AB60E369EB60236A2B615D
:1015300016E7094C40F2FF570023A763A36040F26F
:101540004343E36006210320FEF7E8FEA76300287B
:10155000D5D0A5E610200020002C014010B5104C7D
:10156000D4F80C3A43B119689A880B691A4203D12E
:10157000002384F8E03910BDFFF750FE0028F7D1B2
:1015800094F8D4390133DBB2072B84F8D439EFD87F
:10159000D4F8143AC4F8D039012384F8E03910BDE6
:1015A0001020002070B5A14CD4F8100A002800F0DB
:1015B000138194F8E0596B1E082B0ED8DFE803F076
:1015C000C6057F0D61CA340D1500FFF7DBF8002852
:1015D00040F0058194F8E0596B1EDBB2022B40F21B
:1015E000D380042D47D1012070BD914D226840F277
:1015F000FF5640F24D43AE630121AA600D20EB601F
:10160000FEF78CFEAE6328B96B69C3F34323042B4A
:1016100000F0C780D4F8D039D4F8142AFA339342B2
:10162000D8D2FFF79BFFC4E7814D226840F2FF56F6
:1016300040F24D43AE630121AA600D20EB60FEF73E
:101640006DFEAE630028E5D16B69C3F34323042B21
:10165000E0D1D4F8DC3984F8D409012B40F2DF80E2
:10166000D4F8D8290825013B0132C4F8DC39C4F884
:10167000D82984F8E059A5F10800B0FA80F04009B3
:1016800070BDE66A002E40F09080FFF77BF80028DE
:1016900000F09380D4F8C85984F8D469042384F8FE
:1016A000E039002D9FD0D4F8CC39D4F8BC29D4F837
:1016B000C0193046A84794F8E0596B1E8DE7FEF735
:1016C000FBFE002860D194F86420B4F86630A4F8DA
:1016D000E839A16EA36EC4F8DC09090E04201B0CC6
:1016E00084F8EA2984F8E009A26E84F8EB1984F8FA
:1016F000EC39A16E94F86C0094F86D3084F8EE1912
:10170000120A1B0984F8ED2984F8EF0994F86D207A
:1017100084F8F439216FB4F87600B4F87630C4F860
:10172000F01902F00F02C3F30B1384F8F52943EA12
:101730001023B4F8762003F00F0303F5FA6302F0E8
:101740000F02A4F8F63984F8F82932E7022384F866
:10175000E0392EE7236B002B8DD1D4F8C869D4F87B
:10176000143AC4F8D039072584F8E059002E82D005
:10177000D4F8CC39D4F8BC29D4F8C0190120B0472A
:1017800094F8E0596B1E28E7D4F8143AD4F8D0291D
:101790009B1AC82B7FF66FAFFFF7E0FE94F8E05975
:1017A0001FE7042384F8E0391DE7D4F8D039D4F8D2
:1017B000142A64339342BFF45EAFFFF7CFFED4F830
:1017C000C859002D3FF4F5AE0022D4F8CC39D4F836
:1017D000C0191046A847ECE684F8E00970BDFEF792
:1017E0006BFE00287FF4F6AE94F89030002BA3F146
:1017F0000203B3FA83F308BF01255B0984F8D559C6
:1018000084F8D639FEF758FE00287FF40AAFD4F8E2
:101810008020C4F8E429032384F8E039C9E6C0D164
:10182000FFF792FA94F8E0596B1ED6E610200020DC
:10183000002C01402DE9F0411F4E80460B4696F8E2
:101840006C2D002AFBD19BB343445F1E08F1FF3887
:10185000D6F8703DD6F8742D0133C3F30A039A42CB
:1018600016D10EF0D1FF04460D460EF0CDFF001B41
:1018700061EB0501B0F57A7F71F10001F5D3D6F87F
:10188000703DD6F8742D0133C3F30A039342E8D0B8
:10189000D6F8702DD6F8703D18F8011F3244013388
:1018A000C3F30A03B84582F8781DC6F8703DCFD15E
:1018B0000020BDE8F08100BF1020002090F84820F3
:1018C000531C0244DBB280F8483082F8341090F8A0
:1018D000492052B1132B0CD9002280F8482010B5B2
:1018E0000B4CD4F89C282AB910BD80F84820002B56
:1018F000F5D17047D4F89C28052AF5D11946343023
:10190000D4F8143AFFF796FFD4F8143A10BD00BF8C
:101910001020002010B50A4CD4F89C3803B910BD33
:10192000D4F89C38052BFAD1002A0846D4F8143A8A
:101930001146F4DDFFF77EFFD4F8143A10BD00BF66
:101940001020002090F848100023A0F8483001B97A
:10195000704710B5084CD4F89C381BB1D4F89C38AB
:10196000052B00D010BD3430D4F8143AFFF762FFD5
:10197000D4F8143A10BD00BF102000202DE9F04724
:10198000534E1F4606EB80039C68002C00F09B80A2
:1019900004F13E03A36104F59F73E3614FF4807388
:1019A000C4E904332836236866600546E16094F88C
:1019B0003D00A36391460BF095F8804694F84402ED
:1019C00094F83CA0261D002851D194F8450250BB44
:1019D000D4F840326BBB3A0731D419F0020F49D129
:1019E00019F0010F5AD1D4F8483294F9471294F8FB
:1019F00047221B010029DBB20DDB3649881880F82D
:101A000000335009012302F01F02934041F82030B7
:101A10003046BDE8F087304902F00F0211443046ED
:101A20000B76BDE8F08776F0FFF9D4F84032002B52
:101A3000D1D02A4A116B0B4313633A07CDD5013538
:101A4000EDB2B8F1000F05D040F2067388F80850E7
:101A5000A8F80630FB0694F846222FD417F0200F82
:101A60000CBF3221122140460BF000F8BBE776F0A4
:101A7000DBF9AAE76B1CDBB2B8F1000F05D088F8E0
:101A8000083040F20653A8F8063094F84622404643
:101A900002210AF0EBFF19F0010FA4D050460BF021
:101AA00021F80135EDB218B140F20663C38005722A
:101AB00094F8462202210AF0D9FF94E70221404619
:101AC0000AF0D4FF8FE726463046BDE8F08700BF16
:101AD000503C080800E100E0FCEC00E00038024067
:101AE0002DE9F047038A8489A4B21C4082B047D014
:101AF000814688464FF0004501F14C0701F134065C
:101B0000B4FA84F325FA03F2D24391B2A9F8101083
:101B100014401B3BB8F1000F5FD0042B2ED8DFE838
:101B200003F052483D320300D8F80C30D9F82CA00D
:101B300033B19B6823B11FFA8AF108F1040098477A
:101B4000D8F8243033B19B6823B11FFA8AF108F129
:101B50001C009847D8F83C3033B19B6823B11FFA7A
:101B60008AF108F134009847D8F8543033B19B68B3
:101B700023B11FFA8AF108F14C009847002CBFD11D
:101B800002B0BDE8F087D8F80C30D9F834105B68A3
:101B900008F104009847002CB2D1F1E7D8F82430BE
:101BA000D9F838105B6808F11C009847002CA7D1C1
:101BB000E6E7D8F83C30D9F83C105B6830469847E7
:101BC000002C9DD1DCE7D8F85430D9F840105B6880
:101BD00038469847002C93D1D2E7042B07D8DFE88A
:101BE00003F01903140F0A00D9F83C300193019B4C
:101BF000002C85D1C4E7D9F82C300193019BF7E77D
:101C0000D9F834300193019BF2E7D9F838300193C9
:101C1000019BEDE7D9F840300193019BE8E700BF55
:101C2000F8B5264C94F86C2D012A034603D0022AFD
:101C300009D00020F8BD224ED6F880548DB984F822
:101C40006C5D0020F8BD002540F20112C0E954553A
:101C5000C0E95655A0F8442100F5A27178F0CCFFF8
:101C6000EDE7402D20D94027D4F8741D154AC3F85C
:101C700058710A44C3E9542240F20112A3F84421E6
:101C80000022C3F85C2103F5A271184678F0B4FF76
:101C9000D4F8743D3B44ED1BC3F30A03C4F8743D10
:101CA000C6F880540020F8BDAAB2402A01D02F46C1
:101CB000DAE7022284F86C2DD5E700BF102000205F
:101CC00008310020882D002001EB810138B500EBA0
:101CD000C1010F4DB1F88C1304462846FFF704F8F4
:101CE000E378C4F8A853012083424FF000024FF07C
:101CF0004001C4E9EC12A4F89C0304F56771204686
:101D000008BFC4F8AC5378F077FF002038BD00BF9F
:101D10008C350020F8B52A4CD4F8C4340F2B04D0ED
:101D20005A1CC4F8C4240020F8BD264D95F86C3D1B
:101D30000022C4F8C424002BF5D1D5F8742DD5F8B1
:101D4000703D9A42EFD0D5F8742DD5F8703D9A4287
:101D50002DD8D5F8706DD5F8743DF61A402E2BD8D5
:101D6000B3B2402B13BF3746402702230123D5F8D7
:101D7000742D85F86C3D144BC0F858711344C0E9BC
:101D8000543340F20113A0F844310023C0F85C3111
:101D900000F5A27178F030FFD5F8743D3B44F61B96
:101DA000C3F30A03C5F8743DC4F88064BBE7D5F8F3
:101DB000746DC6F50066D1E701234027D7E700BF61
:101DC0000831002010200020882D002010B5324B53
:101DD00093F8D42493F8E8C4D3F8D034044613B16C
:101DE00052EA0C0231D00123E06984F8463140F216
:101DF0000112A4F8442102682849002AA8BFC2F3AE
:101E000080739B0301EA124143F020030B4363F309
:101E10001F42BCF1020F026000D010BDE278204BDF
:101E2000C4F8A8331F200021C4E9EC01012A4FF0B7
:101E30000101A4F89C1308BFC4F8AC3304F5677122
:101E40002046BDE8104078F0D7BE012178F09EFD15
:101E50000122E06984F8462140F20113A4F84431DC
:101E6000016800290A460CDBC1F380730B4C9B030D
:101E700043F0200304EA11410B4363F31F42026065
:101E800010BD064B03EA114343F4804343F02003A3
:101E900063F31F42026010BD08310020DFBFFFFF67
:101EA000D03500202DE9F041B0F8CC15D0F8CE3572
:101EB000B0F8D255B0F8D085C0F84051012284B0B6
:101EC00080F8112101F01F02012A044600F2CC56CD
:101ED000ADF80810C1F3072ECDF80A30ADF80E505A
:101EE0004FEA134C51D0022A7746C9B29BB210D0A8
:101EF000002A55D1BEF1090F4BD8DFE81EF089004A
:101F0000AD004A00C8004A005C01DF004A0013012E
:101F1000330101F0600120295FFA8CF272D0012FA9
:101F200000F0B881032F00F0A181AFBB90F812310F
:101F3000022B00F0E381032B2BD11CF0800F40F02B
:101F4000E98102EB820200EBC20393F87623003AA8
:101F500018BF0122C24D02234FF48071C4E94E33F1
:101F600084F81131C4F83031A4F81C1105F59F63D1
:101F70000021C4F83411C4E94A3304F58E712046B7
:101F8000C5F8F82478F0D6FD06E090F81231032B5E
:101F90000ED0204678F0C2FC002004B0BDE8F081ED
:101FA00001F0800178F0F2FC002004B0BDE8F0817F
:101FB0005FFA8CFCBCF1010FEBD8D0F8E43502A934
:101FC0009B689847BDF80E30002BE5D1C4E94A3331
:101FD000C4E94C3304214FF4807284F81111A4F841
:101FE0001C2104F58E71204678F0A4FD636D9D4A96
:101FF0001A61E278012ACFD15E614FF08022196820
:102000001A60C9E7D0F8E43502A99B689847C3E78E
:1020100090F81231023B012BBBD8914BD0F818211C
:102020000021C3F8F01412B10222C3F8F0248E4A42
:1020300002234FF480700021C4E94C31A4F81C0144
:10204000C4E94E33C4E94A2284F8113104F58E7193
:10205000204678F06FFD9FE790F81221023A012A9E
:1020600097D8012B98D1D0F8E43500259B68C0F8AB
:10207000185102A9984704224FF48073C4E94A55C5
:10208000C4E94C5584F81121A4F81C31A9E7012BAF
:1020900000F03B81022B7FF47FAF5FFA8CF3002BC3
:1020A0007FF47AAF03694FEA1C22023A5B68032A85
:1020B00000F2BD81DFE802F0B6CED2D01E0A022EB9
:1020C000ADF8065000F08A81032E00F04E81012EFB
:1020D0007FF45FAFD0F8EC3580781B680DF1060116
:1020E0009847BDF80630002B3FF456AFBDF80E20E0
:1020F000002A3FF451AF934228BF13464FF4807239
:102100000221A4F81C210022C4E94A0084F811111C
:10211000C4E94E33C4E94C3204F58E71204678F0A0
:1021200009FD39E7012D7FF434AF90F81231022B0D
:1021300000F00881032B7FF42CAF4FF4807200F580
:1021400088730221A0F81C21002280F81111C0E937
:102150004E55C0E94A33C0E94C5200F58E7178F013
:10216000E9FC19E7DDB23E4F012D87F8E9543FF64F
:1021700010AF90F81231022B00F0D880032B7FF4BF
:1021800008AF002D00F0358190F81011012910D012
:10219000D0F8E4355B68984797F8E914D4F8E4354B
:1021A00084F810111B6820469847D4F8E8359B68DE
:1021B000984700230AE758EA05027FF4EAAE90F850
:1021C000121103293FF4E5AE03F07F0580F81451A6
:1021D0000069114663F30A1103681943042301607F
:1021E00084F811314FF48073C4E94A22C4E94C22C7
:1021F000A4F81C3104F58E71204678F09BFC636DC9
:10220000184A1A61E278012A06D0002D00F0FC80FD
:10221000022384F81231BFE65E614FF08022196814
:102220001A60F2E702210E4861F306130022C0F89B
:10223000F4340423C4E94A22C4E94C2284F811315D
:1022400001224FF4807304F58E7184F81621A4F8EE
:102250001C31C8E60321E6E70521E4E70421E2E7B3
:102260000831002018000860F835002090F812119D
:10227000022943D003297FF48CAE23B9510602D042
:10228000114678F083FBD4F8E4359B6802A9204618
:1022900098478EE790F8121102292FD003297FF476
:1022A00078AE002B7FF478AE12F07F0181D01CF065
:1022B000800F40F0AD8002EB820100EBC10181F89C
:1022C000763381F87533282381F8742303FB0203E6
:1022D00000EB820193F87723496D0B68023A012ADB
:1022E00023F400138CBFC3F30072012262F31C734A
:1022F000D4F8E4250B60936802A9C8E753063FF4BD
:102300004BAE114678F042FB46E6D0F8E425C0F823
:102310001831F0E702F07F0202EB820200EBC20309
:1023200093F81E21003A18BF012213E6002D3FF456
:10233000A2AE01210322D0F8E43580F8101180F814
:1023400012212FE73B4A80F811314FF480710023AE
:10235000A0F81C11C0E94E55C0E94A22C0E94C530F
:1023600000F58E7178F0E6FB16E6DBB2052B3FF642
:1023700010AEDFE803F02B231B130B03D0F8EC3572
:1023800080789B690DF106019847AAE6D0F8EC35F4
:1023900080785B690DF106019847A2E6D0F8EC352C
:1023A00080781B690DF1060198479AE6D0F8EC3564
:1023B0008078DB680DF10601984792E6D0F8EC359D
:1023C00080789B680DF1060198478AE6D0F8EC35D5
:1023D00080785B680DF10601984782E6D0F8E43515
:1023E00080789B6A0DF1060198474670C4F8F005A5
:1023F00077E60222D0F8E43580F8122180F81051F7
:102400005B682946984736E6012384F81231C3E514
:10241000282202FB010080F81C1104EB810180F8E6
:102420001E3180F81DE190F81F21896955E70121CF
:10243000F9E600BFF435002010B5044629B990F83C
:102440001121032A0DD0002010BDD0F8E4359B697E
:10245000002BF8D090F81221032AF4D198470020DD
:1024600010BDD0F890230B46D0F87C138A4219D9BE
:10247000521AC0F8902394F803C0D0F880038A421F
:1024800028BF0A46BCF1010F92B234D0C4E9E2235E
:1024900004F55D71C4F88003A4F87433204678F025
:1024A00049FBD0E7D0F8E4351B691BB190F8122145
:1024B000032A1ED000234FF480720421C4E94A335A
:1024C000C4E94C3384F81111A4F81C2104F58E7171
:1024D000204678F02FFB636D0D4A1A61E278012ADD
:1024E000B1D104F2CC545C614FF0802219681A60BB
:1024F000A9E79847DEE70844C4E9E22304F55D71E3
:10250000C4F88003A4F87433C4F88403C6E700BF9A
:102510001800086038B5044649B990F81131022B0B
:1025200011D094F81631012B39D0002038BDD0F8E5
:10253000E4355B69002BF8D090F81221032AF4D11E
:102540009847002038BDD0F83831D0F82421934284
:102550002FD990F803C09B1ABCF1010F0D46C0F8AB
:102560003831D0F828116ED09BB2C0F830314FF41A
:102570008073C0E94A11C0F8345100F58E71A0F89B
:102580001C3178F0D7FAC4E9E255C4F8805304F559
:102590005D71A4F87453204678F0CCFAC1E73F4B44
:1025A0002269D3F8F4145160002384F81631002016
:1025B00038BDD0F83C31B3FBF2F502FB15350DBB4D
:1025C0009A421FD8D0F8402193421BD24FF4807317
:1025D000A0F81C3100F58E71C0E94A55C0E94C5590
:1025E00078F0A8FAE378C4F84051012BC4E9E25529
:1025F000C4F88053A4F8745308BFC4F8845304F596
:102600005D71C8E7D4F8E435DB681BB194F812219A
:10261000032A15D0E27800230521012A84F811113C
:10262000C4E9E233C4F88033A4F8743304F55D716F
:1026300024D0204678F07EFA636D194A1A6170E75B
:1026400020469847E6E79BB21144C0F830314FF47A
:102650008073C0E94A11C0F8345100F58E71A0F8BA
:102660001C3178F067FAC4E9E255C4F8805304F5E8
:102670005D71A4F87453C4F884538CE7C4F88433B0
:10268000204678F057FA636D0548186104F2CC5281
:102690005A614FF080211A68196042E70831002022
:1026A0001800086070B50B7813F060020D46044600
:1026B00024D0202A04D0204678F030F9022070BDC2
:1026C000CA8848781AB31B0640D5324E3146FEF709
:1026D000CFFAEB884FF480720221A4F81C2100226B
:1026E00084F81111C4E94E33C4E94A66C4E94C3296
:1026F00004F58E71204678F01DFA06E04B780A2B1F
:1027000010D00B2B08D0062BD5D0002070BD022294
:102710001144FEF7ADFAF8E78B78C3BB1E4AC2F846
:10272000FC34F2E7022180F811114FF48071A0F817
:102730001C111A490123C0E94A11C0E94E33C0E90E
:102740004C3200F58E7178F0F5F9DEE71449154B3F
:102750000860E078C3F8A028002103F6A40301284C
:102760004FF00305C4F88C13A4F87413C4E9E422F1
:1027700084F81151C4F88823C4F8803304F55D71DE
:1027800008BFC4F88433204678F0D4F9BDE778F068
:10279000C5F8BAE7B428002008310020043600202C
:1027A0000000002010200020002310B51946044628
:1027B000402278F055F9802120460023402278F00D
:1027C0004FF9D4F8E835A078012284F812215B682B
:1027D0009847002010BD00BF10B5022304464022D8
:1027E000812178F03DF9204602234022012178F032
:1027F00037F9204603230822822178F031F9104B63
:102800000222A3F84C20FEF71FFAE2780D4BC4F821
:10281000A8334021C4F8B013012A4FF000004FF054
:102820000101C4F8B403A4F89C13204604F56771B1
:1028300008BFC4F8AC3378F0DFF9002010BD00BF4A
:10284000000000208C35002030B5812183B0044683
:1028500078F0D6F80121204678F0D2F82A490025F0
:102860000223402281F8185A2046812178F0F8F896
:10287000012102234022204678F0F2F8234BD3F8BE
:10288000002583F8E8541268284690470095009A7E
:10289000E1681F4B42F010020092009A0A610A6937
:1028A0000092013B02D0009AD006F8D40023019395
:1028B000019B43F020030193019A154B012060F323
:1028C0008A120192019A0A610A690192013B02D0BF
:1028D000019A9206F8D4E2780E4BC4F8A8331F2070
:1028E0000021C4E9EC01012A4FF00101A4F89C1376
:1028F000204604F5677108BFC4F8AC3378F07CF962
:10290000002003B030BD00BF10200020083100209F
:10291000410D0300D03500202DE9F843374F8046A4
:10292000894615461C4697F8E01904290BD008295A
:1029300007D1D7F8D839434505D0FEF705FA022864
:10294000F1D0012057E0012387F8C4393B6397F8A1
:102950009030C7F8CC490622022B294CC7F8C08911
:10296000C7F8C859C7F8BC9987F8E02918BF4FEADB
:1029700048280A2640F2FF554FF48B63A5630121D6
:10298000C4F808801820E360FDF7C8FC03464FF048
:10299000000C40F2774201213720A563D3B1A56333
:1029A000C4F808C0E260FDF7B9FC721EA56388B1E7
:1029B00012F0FF06E0D13E63FEF7D0FDD7F8C8491C
:1029C00034B1D7F8CC39D7F8C01932460120A04726
:1029D000032010E00121484675F09EF9084B094993
:1029E00059624FF400729A62DA6A002142F0910251
:1029F000DA620846B962BDE8F88300BF1020002003
:102A0000002C014000E1F5052DE9F04F3F4E9946BD
:102A100096F8E03983B0042B01908846924609D09D
:102A2000082B03D0002003B0BDE8F08FFEF78CF92F
:102A30000228F7D196F890300122022BF26262D080
:102A4000019B4FEA432B324C0021404675F064F95C
:102A50004FF400722F4B6362A262E36A40F2FF57A9
:102A600043F09303E362A763A2604FF48A62E260DB
:102A700001211020FDF752FC0A25A76340F25142C4
:102A8000A7630121C4F808B01120E260FDF746FCFD
:102A900002464FF0000E40F2774301213720A76332
:102AA000DAB1A763C4F808E0E360FDF737FC013D45
:102AB000A76390B115F0FF05E0D1F562B062FEF7B3
:102AC0004DFDD6F8C849002CACD0D6F8CC39D6F894
:102AD000C0192A462846A047A4E7052386F8E0390E
:102AE0000023B362019AD6F8143AC6F8BC890120D3
:102AF000C6F8C029C6F8C8A9C6F8CC99C6F8D03916
:102B000003B0BDE8F08FDDF804B09CE71020002092
:102B1000002C014000E1F5051049114BD1F8882047
:102B200042F4700210B4C1F888201A680D4C0020DD
:102B300042F001021A6098601A6822F0847222F44E
:102B400080321A605C601A68074C22F480221A6096
:102B5000D8608C605DF8044B704700BF00ED00E06A
:102B6000003802401030002400000008704700BF09
:102B70002DE9F84345697DB90768C7F30D08044698
:102B80000E46B8F1000F0AD0D6F80080FDF7F4FE2B
:102B900009283BD06FF001052846BDE8F883514B6A
:102BA0009F422AD303F580439F4224D303F58043F9
:102BB0009F427FD34C4B9F427FD903F580339F4286
:102BC0007ED903F500339F427DD903F500339F4240
:102BD0007CD903F500339F4269D903F500339F4246
:102BE00077D903F580239F4276D9B7F1016F76D369
:102BF00005200DF065FE4FF00808FDF7BDFE092821
:102C000021D04FF0FF352846BDE8F883374E3369B1
:102C100023F440733361336943F4007333613369E0
:102C200043F001033361C7F80080FDF7A5FE336967
:102C3000092823F001033361ACD1236804332360F6
:102C40002846BDE8F883DFF8A490D9F8103023F4C3
:102C50004073C9F81030D9F8103043F40073C9F844
:102C60001030D9F8103023F0F803C9F81030D9F833
:102C7000103043EA080343F00203C9F81030D9F8D2
:102C8000103043F48033C9F81030FDF775FED9F8E1
:102C9000103023F00203C9F81030D9F81030092899
:102CA00023F0F803C9F810303FF46EAFA9E74FF0F6
:102CB0003808A2E74FF010089FE74FF018089CE78C
:102CC0004FF0200899E74FF0280896E74FF03008BA
:102CD00093E74FF0400890E74FF048088DE74FF03A
:102CE00058088AE700400008FFFF0008003C024047
:102CF0000148FDF78DBA00BFD80000200148FDF75C
:102D000087BA00BF240300200148FDF781BA00BF45
:102D1000700500200148FDF77BBA00BFBC0700200A
:102D20002DE9F0410268214D0746002455F8343062
:102D30009A4209D001340E2CF8D11D4A00210520F9
:102D400005F0A4FC002013E01A4B03EB8408D8F82C
:102D500004657EB1797901EB410306EBC3030022E0
:102D60001820C3E9032200FB01609F601A7504303C
:102D7000BDE8F08107216C2005F00EFD0146C8F882
:102D8000040568B131466C227FF034FED8F8046542
:102D900005EBC405C6E90056F6617663F664D9E72B
:102DA000054A052005F072FCCCE700BFAC3C0808E2
:102DB000A0E3080808310020C8E30808704700BFF6
:102DC00030B40C4C0022234604E001320C2A03F1FB
:102DD00014030CD093F804C08445F6D1DD68294271
:102DE00001D10029F1D1142303FB024000E00020AF
:102DF00030BC7047040A002038B5D0E9004007EE27
:102E0000902A0068324A334B2468D3F8F43A246895
:102E1000013990428DB210D002F5806290420CD000
:102E200002F57052904208D002F58062904204D0C0
:102E300002F58062904218BF5B0807EE103AF8EE88
:102E4000677AB8EE477ADFED246A87EE270A30EE1C
:102E5000260A7AF031FD1E492388421E8C4292B226
:102E60009BB21AD01D498C4217D0B4F1804F1FD0AD
:102E7000A1F580318C421BD001F580618C4217D0C6
:102E800001F580618C4213D015498C4219D1238001
:102E90000123E5622285A38238BD23F45C739BB2D3
:102EA00023800023E562228523860123A38238BD87
:102EB00023F45C739BB223800123E5622285A38205
:102EC00038BD08498C42E2D023F440739BB2DEE760
:102ED00000000140000000200AD7233C000401400C
:102EE000001000400014004070B54268937903F070
:102EF000020E13F004033AD175469C469E464FF4E9
:102F0000807001235479032C30D8DFE804F08E62FE
:102F100002361468704E228C22F480721204120C55
:102F20002284228C22F4007212042B43120CA588F6
:102F300042EA0322A38B23F073031B041B0CB4424D
:102F4000ADB243F0600300F09B8006F58066B442AA
:102F500000F09680A580A383E1632284A38B23F0F5
:102F600008031B041B0C43F00803A38370BD00205F
:102F700005464FF0040C0346C4E71268564E148C05
:102F800024F480542404240C1484148C24F4005459
:102F900024042B43240C958844EA0334938B23F4B4
:102FA000E6431B041B0CB242ADB243F4C04375D0E0
:102FB00006F58066B24271D09580938311641484C3
:102FC000938B23F400631B041B0C43F40063938373
:102FD00070BD1468404E228C22F010021204120CB4
:102FE0002284228C22F0200212042B43120CA5888A
:102FF00042EA0312238B23F4E6431B041B0CB44266
:10300000ADB243F4C04359D006F58066B44255D002
:10301000A5802383A1632284238B23F400631B04F4
:103020001B0C43F40063238370BD1268148C24F0DE
:1030300001042404240C1484148C968824F00204C3
:1030400024042B43240C1C43138B234D23F07303C4
:103050001B041B0CAA42B6B243F0600323D005F553
:103060008065AA421FD09680138351631484138B0A
:1030700023F008031B041B0C43F00803138370BDEB
:1030800022F4006242EA0E2222F4806292B225F417
:10309000405542EA0C2245EA00155BE725F48045DD
:1030A00045EA801588E726F4407606434FF6F3702C
:1030B000204040EA0E0040EA0C04D4E722F08002EF
:1030C00042EA0E1222F0400292B225F4406542EA32
:1030D0000C1245EA80059BE70000014042685379E5
:1030E000032B0FD8DFE803F00B080502106840300F
:1030F000704710683C30704710683830704710686F
:103100003430704700207047024B0348D3F8041551
:10311000FEF7E6BC083100200000014010B5064C67
:103120000648D4F80415FEF7DBFCD4F8241504484F
:10313000BDE81040FEF7D4BC08310020000001407B
:103140000040014010B5064C0648D4F80415FEF7BF
:10315000C7FCD4F828150448BDE81040FEF7C0BCF1
:1031600008310020000001400044014010B5064C29
:103170000648D4F80415FEF7B3FCD4F82C1504481F
:10318000BDE81040FEF7ACBC083100200000014053
:1031900000480140034B4FF08040D3F80815FEF77C
:1031A0009FBC00BF08310020024B0348D3F80C1528
:1031B000FEF796BC0831002000040040024B034893
:1031C000D3F81015FEF78CBC083100200008004031
:1031D000024B0348D3F81415FEF782BC08310020D7
:1031E000000C0040024B0348D3F82015FEF778BCD2
:1031F000083100200004014010B5064C0648D4F800
:103200002015FEF76DFCD4F830150448BDE81040D9
:10321000FEF766BC083100200004014000180040A1
:1032200010B5064C0648D4F82015FEF759FCD4F822
:1032300034150448BDE81040FEF752BC08310020A8
:1032400000040140001C004010B5064C0648D4F8AC
:103250002015FEF745FCD4F838150448BDE81040A9
:10326000FEF73EBC08310020000401400020004071
:103270000348D0F8043B13B100F6F8201847704714
:10328000000000200348D0F8243B13B100F61830AA
:1032900018477047000000200348D0F8443B13B1A2
:1032A00000F6383018477047000000200348D0F877
:1032B000643B13B100F658301847704700000020F7
:1032C0000348D0F8843B13B100F6783018477047B4
:1032D000000000200348D0F8A43B13B100F698305A
:1032E00018477047000000200348D0F8C43B13B1D2
:1032F00000F6B83018477047000000200348D0F8A7
:10330000E43B13B100F6D8301847704700000020A6
:103310000348D0F8043C13B100F6F8301847704762
:10332000000000200348D0F8243C13B100F61840F8
:1033300018477047000000200348D0F8443C13B100
:1033400000F6384018477047000000200348D0F8C6
:10335000643C13B100F65840184770470000002045
:103360000348D0F8843C13B100F678401847704702
:10337000000000200348D0F8A43C13B100F69840A8
:1033800018477047000000200348D0F8C43C13B130
:1033900000F6B84018477047000000200348D0F8F6
:1033A000E43C13B100F6D8401847704700000020F5
:1033B00030B44568144CA542144D2C6B0CBF44F43A
:1033C000001444F480042C6390F914C0C16012010D
:1033D000BCF1000F8361D2B20FDB0D4901EB0C038E
:1033E0004FEA5C1083F800230CF01F0C012303FA52
:1033F0000CF330BC41F820307047064B0CF00F0C3A
:1034000063441A7630BC70470060024000380240C6
:1034100000E100E0FCEC00E02DE9F843A8480022C0
:1034200042F2043C510143588CEA030313F47C54E8
:103430000AD00132102AF5D1A24D0023C5F8103A66
:1034400085F8E039BDE8F88301449E4D0B7FC5F84F
:10345000101A002BF1D18F689B4B9F4202D048334A
:103460009F42EAD1994A536A43F4006353620DF0D4
:10347000CBF9064688460DF0C7F9801B61EB0801C1
:10348000B0F57A7F71F10001F5D3904A536A23F4C5
:10349000006353620DF0B8F9064688460DF0B4F9A2
:1034A000801B61EB0801B0F57A7F71F10001F5D363
:1034B000DFF818828648D8F8443043F40063C8F82F
:1034C0004430D8F8303043F48003C8F83030D8F8AE
:1034D000303043F00C03C8F830304FF00D090026AF
:1034E0000C220E21A5F8029D85F8046D09F0BEFAA4
:1034F0007848A5F80E9D0C220E2185F8106D09F074
:10350000B5FA7548A5F81A9D0C220E2185F81C6D98
:1035100009F0ACFA7148A5F8269D0C220E2185F819
:10352000286D09F0A3FA6E48A5F8329D0C220E21F1
:1035300085F8346D09F09AFA0C226A48A5F8629D64
:103540000E2185F8646D09F091FA674B302283F8FB
:1035500031234FF400325A60D8F83030634A43F4D4
:103560008003C8F83030584BC2F83C759F425BD09E
:103570005F4A6049C2F8A060C2F8A8104FF4741105
:10358000D1605D49C2F8A0100721C2F8B4104C4ABE
:103590005A4F33461046114605E00133102B01F116
:1035A000200100F089808E68BE42F6D1544901EBBB
:1035B00043115B01D1F8FC6A52498E426DD0434EF3
:1035C000316B41F48001316303440D2199834B49F0
:1035D00093688B4225D00134102C02F12002F7D1E0
:1035E0000020494900230122FFF7E2FED5F80C3AFA
:1035F0004BB119689A880B691A4204D1002385F8E7
:10360000E039BDE8F883FDF709FE0028F6D1D5F8CA
:10361000142AC5F8D029012385F8E03985F8D409A2
:1036200010E700EB4410DCE7314932488E65244A4C
:103630000866334630484FF074668E608865072010
:10364000C8661046114604E00133102B01F1200139
:1036500032D08E68BE42F7D1294901EB43115B019C
:10366000D1F8FC6A27498E4220D0184E316B41F4C4
:103670008001316303440D219983134993688B4280
:1036800011D00134102C02F12002F7D100201F4983
:1036900000230122FFF78CFEA8E70C4E316B41F4AA
:1036A0000011316390E700EB4410F0E7074E316BF7
:1036B00041F400113163DDE700235B68FFDE00BFEA
:1036C000F80A002010200020586402400038024010
:1036D0000C2D0020182D0020242D0020302D00203E
:1036E0003C2D00206C2D002000E100E0083100207E
:1036F00000640240802C01406054A308A064024092
:1037000000000020006002408D080008C507000886
:1037100070B52D4C636BD9051ED54FF4807340F204
:10372000FF56A363A663E36B284D23F4414323F0C4
:103730003A03E3636B6B9A071FD4012200236A628A
:10374000AB62214A40F2FF539363D36B23F44143AE
:1037500023F03A03D36370BD636B980703D51B4B0B
:1037600002229A62EDE7636B190721D4636B9A0614
:1037700022D5164B06229A62E3E7154BD3F83C2577
:10378000136823F001031360E36A002223F00803A7
:10379000E3622A636B6BDB07CFD540F24C43A66331
:1037A0000121A2600C20E360FCF7B8FDA663C4E72A
:1037B000064B04229A62C4E7636BDB06C1D5034B58
:1037C00005229A62BDE700BF002C014010200020B6
:1037D0000831002002683649002310B422F00102AB
:1037E000212488420260036043608360C3600361F8
:1037F000446138D02F4B98422ED02F4B98423CD06A
:103800002E4B984240D02E4B984232D02D4B9842AE
:1038100041D02D4B984246D02C4B984217D02C4B80
:1038200098423CD02B4B984216D02B4B984224D038
:103830002A4B984228D02A4B98421AD0294B9842BA
:1038400029D0294B98422ED0284B984208D14FF0CE
:103850003D5243F8AC2C03E04FF4746243F8202C43
:103860005DF8044B7047224B5DF8044B3D229A6093
:103870007047204A43F8642CF2E74FF474125DF865
:10388000044B43F8382C70474FF074625DF8044BDA
:1038900043F8502C7047184A43F87C2CE0E73D224F
:1038A00043F8082CDCE7154A43F8942CD8E700BF0E
:1038B00010600240286002404060024058600240B0
:1038C0007060024088600240A0600240B860024020
:1038D0001064024028640240406402405864024080
:1038E0007064024088640240A0640240B8640240F0
:1038F000006002403D000020400F002000003D20FD
:10390000214A936803F00C03042B10B43AD0082B1F
:103910001FD01E4B1C4C0360A1681D4AC1F303114C
:10392000114491F8CC10CB404360A168C1F38221CF
:10393000114491F8CC1023FA01F18160A1685DF87F
:10394000044BC1F342310A4492F8CC20D340C36007
:1039500070475368516813F4800F536814BF0D4AC1
:103960000A4AC3F3881301F03F01B2FBF1F202FBF4
:1039700003F3054A5268C2F3014201325200B3FB1D
:10398000F2F3C7E7034BC5E7003802400024F40018
:10399000503C080800127A0070B5446B8668A38911
:1039A00023F400531B041B0CA381857990F805C0F8
:1039B0002B0303F40051C5F380000CF001032A022D
:1039C0009B001CF0020F4FEA003002F4806218BF27
:1039D00043F0080302431A43238A9BB223F4405363
:1039E0000B432382A38923F4B05323F00C031B045D
:1039F0001B0C1343A381A38A23F440731B041B0CE9
:103A000084B0A3826846FFF77BFF234B9C4205D01E
:103A100003F580639C4201D0029B00E0039BA289D6
:103A20001E49120403EB83034CBF7600B60003EB80
:103A30008303B3FBF6F3A1FB0302A08952096426BA
:103A4000000406FB12334FEA02121CD41B0132336E
:103A5000A1FB0313C3F3431313439BB223812A0730
:103A6000A38A0AD59BB243F00803A382A3899BB221
:103A700043F40053A38104B070BD23F008031B047A
:103A80001B0CA382F2E7DB003233A1FB0313C3F369
:103A900042131343E1E700BF001001401F85EB51C3
:103AA0002DE9F8431D462E4B9DF820609DF824908B
:103AB0009842884617463BD02A4B984240D02A4B22
:103AC000984245D0294B984221D14B46324629464F
:103AD0000520FDF753FF04460023C4E90B87C4E922
:103AE0000733C4E909336671A56084F8069020465F
:103AF000FFF752FFF107626B12D4B3070BD493891F
:103B00009BB243F4005393812046BDE8F883002420
:103B10002046BDE8F883D36843F08003D360EEE726
:103B20004FF6DF731380D36843F02003D360E4E7DC
:103B30004B46324629460020FDF720FF0446CBE7DE
:103B40004B46324629460120FDF718FF0446C3E7DD
:103B50004B46324629460320FDF710FF0446BBE7DB
:103B60000010014000440040004C0040001401409F
:103B7000816011E741710FE781710DE72DE9F04395
:103B8000704F07EBC00985B005464FEAC00899F8A9
:103B9000FC0C08F0A7FF064699F8FD0C08F0A2FF00
:103BA000044699F8FE0C74F03FF96B1CDBB21EB1B1
:103BB00040F60C123372F2801CB1237240F60C23D3
:103BC000E380304604223A2108F050FF04222046C8
:103BD0003A2108F04BFF07EB08025B4BD2F8F84C98
:103BE0009C4200F08E80594B9C4200F09580584BCF
:103BF0009C4200F09C80474497F8FF3C022B32D057
:103C0000032B7CD05349544F012B08BF0F46A68885
:103C10006846FFF775FE26F03F06029B4F4AB3FB4E
:103C2000F7F13604A2FB0323360C46EA9346A6803E
:103C3000228822F001021204120C22808AB2C1F3FF
:103C40000B019B0C09B942F001024FF4967101FB84
:103C500003F34349A1FB03139B0901339BB242F4D5
:103C6000004223841FE0A6886846FFF749FE26F03D
:103C70003F06029A394B3604A3FB0213360C46EA80
:103C80009346A680218821F001010904090C2180B6
:103C900034499209A1FB021292099B0C0133042AB8
:103CA000238438BF0422A28323882F4A9BB243F087
:103CB00001032380238823F4816323F002031B0480
:103CC0001B0C4FF4804143F48063238021812388BF
:103CD00023F080031B041B0C238023889BB202EB80
:103CE000451243F0010323800121002382F840554F
:103CF00082F8411582F8423505B0BDE8F0831B4FCC
:103D000085E703F5F2331A6A42F400121A621A6A5E
:103D100022F400121A626EE703F5F0331A6A42F4D5
:103D200080021A621A6A22F480021A6263E703F5BB
:103D3000EE331A6A42F400021A621A6A22F400028E
:103D40001A6258E70000002000540040005800406C
:103D5000005C0040009F2400804F120083DE1B4364
:103D6000D34D6210632D3E0508310020C0270900A5
:103D70002DE9F047924E90F900108046807806EBCE
:103D8000C1050138CC0090B0D5F8F81C14282DD806
:103D9000DFE810F04C012001150055005F009E0087
:103DA000A600C301B6017A0084003C020402D701D8
:103DB000C000D0002F003700A30195015401888A6C
:103DC0000C8B81B27F4841EA0441884300F0208196
:103DD000D8E90201101A42F2107263EB010190421D
:103DE00071F1000102D3152388F8023010B0BDE84C
:103DF000F08798F813000882C8E90223122088F897
:103E00000200888A0C8B80B240EA04406E4C8443E6
:103E100000F0B28000200E900F9001200F910E90C4
:103E20000E99002900F017820F9914310F910F9904
:103E300009684905CCD5142388F80230D6E798F8EC
:103E4000110000F0FE000882C8E90223052088F86E
:103E50000200888A0C8B80B240EA04405B4C8443A9
:103E600000F0A180002000900190012001910090BD
:103E70000099002900F0FB81019914310191019909
:103E800009684F05D7D4A3E798F8110040F0010066
:103E90000882C8E902230B2088F80200888A0C8B6C
:103EA00080B240EA04404A4C84436DD00020049024
:103EB00005900120059104900499002900F0D1811A
:103EC000059914310591059909684D05B3D47FE72B
:103ED00098F813000882C8E90223072088F8020036
:103EE000888A0C8B80B240EA0440374C84435ED011
:103EF0000020029003900120039102900299002972
:103F000000F0C181039914310391039909684E05AA
:103F100091D45DE7088820F480600004000C0880DC
:103F200098F8110000F0FE000882C8E90223102072
:103F300088F80200888A0C8B80B240EA0440234C47
:103F4000844312D000200C900D9001200D910C9014
:103F50000C99002900F091810D9914310D910D9962
:103F6000096848053FF567AF32E798F81330FF2B33
:103F700006D198F810301BB1132388F8023035E7CA
:103F8000112388F8023031E7D8F81400012800F036
:103F90008F81022800F04382098B0E21C8E9022399
:103FA00088F8021022E7062388F802301EE7D8F8C6
:103FB0001400002800F06D81082388F8023015E70E
:103FC00000000020010003008400070082000700B9
:103FD00002000300088820F400600004000C088040
:103FE000088880B240F480600880088880B240F47D
:103FF00080700880032088F80200888A0C8B81B2C8
:10400000A94841EA04418843C8E902237FF4EEAE9F
:1040100098F81230002B40F0CE8198F81330FF2B27
:1040200000F03F82042388F80230DFE60988890522
:104030003FF5CEAE002388F80230D7E6344494F83A
:10404000FC0C08F04FFD064694F8FD0C08F04AFD04
:10405000964AB2F8A03501339BB28246A2F8A03549
:1040600016B13368B2881A83BAF1000F04D0DAF8B7
:104070000030BAF804201A831121304608F0D2FC2F
:104080001121504608F0CEFC4FF0090965272EB1EA
:104090003368B28819690A4240F02381013F00F079
:1040A0001D810CF0B1FB04460D460CF0ADFB001B6E
:1040B00061EB0501052871F10001F6D3E7E70888F7
:1040C00080B240F4007008804FF6FF3088820121F2
:1040D000C8E9022388F8021088E6D8F814000028FE
:1040E00000F06D81D8F8184014F8016B0E82013889
:1040F0001225C8E90504C8E9022388F8025075E6CC
:10410000888A0C8B81B2684841EA044188437FF475
:104110005FAE0A2388F8023068E6088880B240F46F
:1041200080700880092088F80200888A0C8B81B290
:104130005D4841EA04418843C8E902237FF456AE52
:10414000E7E7002401250A940B940B910A950A983D
:10415000002800F047810B9814300B900B980068F2
:1041600046077FF535AED8F81400032800F06D81BE
:10417000022800F24381088820F480600004000CCB
:104180000880088880B240F400700880098A88F8A6
:104190001C40C8E9022388F8025027E600200124C9
:1041A00008900990099108940898002800F014815B
:1041B0000998143009900998006847077FF508AE00
:1041C000EFF31185102080F31288088880B240F444
:1041D00000700880D8F818000E8A471CC8F81870BC
:1041E000EDB2067085F311880D8AD8F818106FF0BB
:1041F00001004E1CC8F818600D70C8E90223C8F809
:10420000140088F81C4088F80240EFE50020069072
:104210000790012007910690069C002C00F0E88092
:10422000079C14340794079C246864067FF5D0AD7E
:104230000C8AD8F818104D1CC8F818500C70D8F813
:10424000141088F81C000139C8E90223C8F81410BA
:1042500088F80200CAE50F9918310F910F99096883
:10426000B6E505991831059105990968B0E50199F8
:104270001831019101990968AAE50D9918310D913C
:104280000D990968A4E50399183103910399096808
:104290009EE5088880B240F4007008800121C8E9DA
:1042A000022388F80210A1E5010003000831002074
:1042B000088820F480600004000C0880EFF311846B
:1042C000102080F31288088B088880B240F40070B8
:1042D000E4B2088084F311880C215FE616B13368DC
:1042E000B2885A830CF090FA04460D460CF08CFA12
:1042F000001B61EB0501052871F10001F6D316B131
:104300003368B2881A830CF07FFA04460D460CF02D
:104310007BFA001B61EB0501052871F10001F6D362
:10432000B9F101097FF4B2AE16B13368B2885A838D
:104330000CF06AFA04460D460CF066FA001B61EBBD
:104340000501052871F10001F6D3BAF1000F04D080
:10435000DAF80030BAF804205A830CF055FA044613
:104360000D460CF051FA001B61EB0501052871F1B7
:104370000001F6D316B13368B2881A830CF044FA00
:1043800004460D460CF040FA001B61EB05010528C0
:1043900071F10001F6D3BAF1000F04D0DAF8003061
:1043A000BAF804201A8398F90000441C3FF442AE86
:1043B000FFF7E4FB3EE60F2388F8023016E5088895
:1043C00080B240F4007008800121C8E9022388F817
:1043D0001C1088F8021009E509991831099109990A
:1043E0000968F5E40B9918310B910B990968EFE412
:1043F00007991831079107990968E9E4D8F8180076
:10440000098A441CC8F818400170D8F81410C8F87C
:1044100008200139C8F81410C8F80C30E6E4088800
:1044200080B240F400600880EFF31184102080F324
:104430001288088B088820F480600004000CE4B225
:10444000088084F311880D21A8E5088820F4806095
:104450000004000C0880EFF31184102080F3128810
:10446000D8F818000D8A461CC8F81860057008882E
:1044700080B240F40070E4B2088084F31188D8F868
:104480001800098A441CC8F818400170D8F81410A4
:104490000C200239C8E90223C8F8141088F8020079
:1044A000A4E498F81030002B3FF4BCAD31E600BF17
:1044B00038B5184D9DF814E005EB40144FEA401C48
:1044C00094F8410500B938BD490084F85325C4F873
:1044D000543584F851150023049984F850E50222DC
:1044E00005F5A86584F85235C4F8581584F85C358C
:1044F00084F8422565440CF087F902460B462846AD
:10450000FFF736FC94F84235002BF4D194F85C05A3
:1045100038BD00BF0831002038B5184D9DF814E0B3
:1045200005EB40144FEA401C94F8410500B938BD32
:1045300084F85325C4F8543501220023490005F5B9
:10454000A86584F8522584F85C35049A84F850E50F
:10455000022384F85115C4F8582584F8423565447F
:104560000CF052F902460B462846FFF701FC94F87E
:104570004235002BF4D194F85C0538BD0831002099
:10458000F0B589B00023904A02930393136843F473
:104590008033136003E0029BB3F5A04F09D013688A
:1045A00003F400330393029B01330293039B002B1C
:1045B000F1D0854B1B6813F4003318BF012303931C
:1045C000039B012B01D000BFFDE77F4B7F491A6C95
:1045D0007F4842F080521A640A6842F440420A60FE
:1045E0009A689A609A6842F400429A609A6842F423
:1045F000A0529A6058601A6842F080721A601A6875
:104600009001FCD5734A40F205711160996821F060
:1046100003019960996841F00201A2F580629960F6
:10462000936803F00C03082BFAD1936803F00C0392
:10463000042B00F0C680082B00F0AB80664A624B6A
:1046400066499868664D674E674FC0F30310014492
:10465000002491F8DC10CA406449E9606449586F4D
:10466000A960596BC6F8F42A21F080015963596F8B
:10467000604A614841F080715967196B0A431A63B7
:104680005A6B5A639A6B9A631A6C5C490A431A64B0
:10469000596C5B4A0A435A6448F2FF71234622462A
:1046A000CDE9004476F044FE5648234622464FF6B4
:1046B000FF71CDE9004476F03BFE53482346224685
:1046C0004FF6FF71CDE9004476F032FE4F482346A5
:1046D00022464FF6FF71CDE9004476F029FE4C48A2
:1046E000234622464FF6FF71CDE9004476F020FEC6
:1046F0004848234622464FF6FF71CDE9004476F044
:1047000017FE4548234622464FF6FF71CDE9004487
:1047100076F00EFE4148234622464FF6FF71CDE962
:10472000004476F005FE234622464FF6FF713C48D2
:10473000CDE9004476F0FCFD04A8FFF7E1F8D5F8D8
:10474000FC200499D6F8F43A364842F08072C5F855
:10475000FC20354AC2F8B00F5460106840F00100E8
:1047600010604FF47A72B3FBF2F3013BB3F1807F38
:104770002E4AB1FBF2F2C7F8A42508D24FF0E0228E
:10478000F0215361072385F823109461136109B068
:10479000F0BD5168536852684902C2F388124CBF99
:1047A00023490D4903F03F03B1FBF3F303FB02F28E
:1047B000054B5B68C3F3014301335B00B2FBF3F2CB
:1047C0003DE71B4A3BE700BF003802400070004055
:1047D00008544007003C02400024F400503C080804
:1047E00000ED00E000000020083100200003FA0581
:1047F00000000008FF91670000000240FFC9FE10A2
:10480000335707000004024000080240000C024039
:10481000001002400014024000180240001C024038
:104820000020024055CEACC5001000E040420F0011
:1048300000127A0082B0064B002201920193019B84
:1048400003EB80030193019B196002B0704700BF26
:104850005028004010B51C2008F044F911210446EE
:1048600008F0E0F8204605F077F8C8200BF0FAFFD2
:104870002046BDE8104005F069B800BF704700BF92
:10488000704700BF704700BF10B5104C94F8B235A8
:1048900023B90F4B4FF480225A6110BD4FF0E02234
:1048A000D2F8103D23F00603C2F8103DFEF734F9AC
:1048B000D4F8B8359B68DB07EBD5D4F8B426136879
:1048C00023F0030161F307031360E2E708310020DE
:1048D000003C01402DE9F04FA34CD4F8B4355A699F
:1048E000D5078BB002D50BB0BDE8F08F5A699B6934
:1048F00012EA0301F7D0C1F307430803019300F163
:10490000E180019B5D073FD48807CEB203D5D4F880
:10491000B43502225A610029C0F24A820A05C1F365
:10492000072500F19981370708D5904B9048D3F8B7
:104930001C3D9847D4F8B43508225A61F60600F1B8
:104940000F82E80600F1BE81A80600F11781019BE5
:10495000DA0609D5854B8648D3F82C3D9847D4F81C
:10496000B4354FF480125A61019B9B06BBD57F4B37
:104970007F48D3F8303D9847D4F8B4354FF400124F
:104980005A610BB0BDE8F08FD4F8B8359E69DB6989
:104990001E40B6B2002EB7D0754D4FF0000B05F19A
:1049A00018080F46F00740F18280D4F8B815D8F8FF
:1049B000002008694B6B23FA0BF3DB01DBB20343E6
:1049C0009068034013F00109D8B200F00F824B6BDE
:1049D000012000FA0BF023EA00034B6301239360EC
:1049E000624B6348D3F8143D5FFA8BF1984794F813
:1049F000AB35012B00F07E8219F0800F57D0D5E93E
:104A00004CC1D5F82431D8F800E0ACEB0102934258
:104A1000DEF8180028BF134680B20333B0EB930FC3
:104A200045D9D4F8B83594F8AB95CDE9026BBA46C0
:104A300067469C46B94237D2D5F82431781A984255
:104A400028BF184600F1030BD5F828314FEA9B0B1D
:104A5000B9F1000F10D182B203329210D8F8B860C9
:104A60000AD04946013153F8047B37608A42F9D1B4
:104A7000D5E94C71D5F82831014403448F42C5F87B
:104A80002831C5F83411DEF818300AD195F81C0128
:104A9000012202FA00F0DCF8342022EA0002CCF80D
:104AA00034209BB29B45C5D3DDE9026B574676089F
:104AB0000BF1010B05F1280508F104087FF472AF32
:104AC000394621E7D4F8B8359D69DB691D402D0CC6
:104AD0003FF417AF04F5B568DFF890B0029104F227
:104AE000FC5600274FF00109C24608E06D0807F1A7
:104AF000010706F1040608F1280800F09181EA0791
:104B0000F4D53068D4F8B815836849690B40D9B238
:104B1000DB0740F1708194F8AB35C0F80890012BA9
:104B200007D10169D8F87C33C1F312015B1AC8F8C8
:104B30008C33DBF8103DF9B25046984794F8AB350A
:104B4000012BD3D1002FD1D194F8B936052BCDD17B
:104B5000D4F8FC35074919610749596119684FF0C4
:104B600080211960C2E700BF08310020000000204A
:104B7000B0360020180008607C3C0020D4F8B855FE
:104B8000D4F8C025AB68C3F34103022B136814BFEC
:104B90000021032161F30A0313606B6843F48073FF
:104BA00006A86B60FEF7ACFED4F8B425079ED36868
:104BB00023F47053D360A86810F0060FC0F34101CE
:104BC00000F03C819F49A0483144814240F2AE81CF
:104BD0009E48A6F57401A1F51051814240F2AA81C8
:104BE0009B499C4831448142C0F0A8819A48A6F173
:104BF0008C71A1F54341814240F2A48197499848C4
:104C000031448142C0F0A2819649974831448142A3
:104C1000C0F0A0819548A6F1B771A1F55851814225
:104C2000C0F0A0819249934831448142C0F09681FE
:104C3000914892493044884234BF062005204025DF
:104C4000012160F38D23D3604FF4005384F8AA153B
:104C5000A4F8AC5553617AE600238DF8133094F82C
:104C6000BA368DF81330864B8648D3F8243D9847E2
:104C7000D4F8B835D4F8B425986894F8B2354FF420
:104C800000615161002B3FF44EAEC3077FF54BAE80
:104C900094F8BD36012B7FF446AE9DF81330032BFC
:104CA0007FF441AED4F8B43677491A6842F0010275
:104CB0001A601A6842F003021A600B6943F0060397
:104CC0000B6130E6D4F8B865D4F8B41573680027E2
:104CD00023F0010373600597059B43F020030593C0
:104CE000059B67F38A130593059B0B61674BBC46D5
:104CF0000A690592013B02D0059A9206F8D494F80D
:104D0000A92552B1624B03EB820EFF2253F8040F28
:104D10008260D86B73458260F8D10B2363F3070779
:104D200063F3070C4FF0FF33B3614FF00113F361EE
:104D30007761C6F810C03368564823F4FE633360C9
:104D400094F8AB25D4F8FC35012A18616FD04FF4E4
:104D500080534B614A4B4B48D3F8203D9847F3E5CD
:104D6000D4F8B4359A6922F010029A611A6AC2F333
:104D70004340022802F00F0100F09080062812D173
:104D800001EB810104EBC101D4F87866D1F8340954
:104D9000C2F30A1210443268C4F8742B3268C4F8A3
:104DA000782BC1F834099A6942F010029A61C8E57B
:104DB00094F8B2353BB1D4F8B426136823F003005D
:104DC00060F307031360D4F8B8252D4B2D48D3F8B2
:104DD000285D5368029123F001035360A847D4F87B
:104DE000B43502994FF000425A6197E5010707D5A3
:104DF000082393605BE68A0707D50223836075E684
:104E0000C3060FD51023936051E60B077FF56EAEF6
:104E1000DBF8183D5046984733680821996065E6ED
:104E200002996EE5410679D5402393603FE61A4A20
:104E30005A611A684FF080221A6088E74FF40075B3
:104E40000920FEE6401E1BFF3F420F00DFC8100096
:104E50002013FBFE20D61300FF69180000D3CEFEFE
:104E600040771B00C05BB3FEC091210040AC27001F
:104E7000C01D6AFE40E13300803C36FEE09C4100EC
:104E800000000020B036002000ED00E0410D0300DE
:104E9000C4360020180008607C3C002047F6F07003
:104EA000104280D0C2F30A1201EB810004EBC00073
:104EB00002F1030C5FEAAC0CD0F82869D4F878E66C
:104EC0004FEA810818BF002006D00130DEF80070DC
:104ED00046F8047B8445F8D1414404EBC101D1F884
:104EE00028091044C1F82809D1F834091044C1F840
:104EF000340958E7BBF1000F7FF47EAD94F8B93662
:104F0000042B7FF479ADD4F8FC35184A1A61184A9D
:104F10005A611A684FF080221A606DE5830758BF06
:104F200081467FF569AD02239360C0E501214025EC
:104F30000E2086E6012140250D2082E60121402534
:104F40000C207EE6012140250B207AE60121402538
:104F50000A2076E601214025092072E6012140253C
:104F600007206EE60121402508206AE61800086047
:104F70007C3C002002784368022A11D00C49026967
:104F8000D1F8180210B41840D1F81042D1F80C1220
:104F9000931E400A04FB030008445DF8044B70476D
:104FA000034AD2E9802102EB410202EB5320704711
:104FB000DC5C00202DE9F04F12F0020A884E83B02D
:104FC0009B4601D000286FD0D6F80852002D58D14A
:104FD0004FF0FF3C834C844FCDF804C0E046E646DA
:104FE000002300922268A57B904200F09E80002D55
:104FF00040D003F58179012D07EB09190AD199F801
:105000000750EA0706D415F07E0F03D1ED0900F032
:1050100090809E460133082B04F11004E2D1BCF1CC
:10502000000F009A04DABEF1000FC0F29280F4463D
:105030006D4CD6F8983004EB0C1741F2180E013382
:1050400047F80E0041F21C0E0CF5817547F80E3042
:105050002F01C6F89830E35104EB051300275F6079
:1050600004EB05139B79042B7AD8DFE803F0294081
:10507000194043009C460133082B04F11004B1D1C0
:10508000CDE7D6E9833404FB05339842A0D396F8E4
:10509000B43113B9012386F8B431534B01225A704D
:1050A000002003B0BDE8F08F96F8B431A6F5805427
:1050B000002B59D001230220637003B0BDE8F08FAC
:1050C00012F0010776D104EB0513D01093F807E036
:1050D000BBF1030F60F3C71E83F807E068D94FF6F2
:1050E000FF735B4528BF5B4604EB05108380BAF174
:1050F000000F49D1500705D504EB0510C37943F0E3
:105100000103C371D30608D504EB0515EB79C3F38E
:105110004502013262F34603EB71344B012003EB8D
:105120004C230B6003B0BDE8F08F009A05BB9C4692
:105130007EE7A568019A954238BF984603F10103BE
:1051400038BF2A46082B019204F110047FF44AAFBD
:1051500065E7B8F1000FA8BFC446BFF669AF9FE787
:1051600096F8B431002BA5D1012386F8B431A1E71C
:10517000D6F898701C4C03F581759C462B010137BD
:10518000E750C6F898706BE7D6F89830D6F89C00D0
:1051900001330130C6F89830C6F89C0004EB0C10BF
:1051A00041F21C06835104EB051304209871A1E71A
:1051B0003B4699E70E4BD3F8683D002B3FF470AFA8
:1051C0000A495E680B4A01EB4C210023B0470028D6
:1051D0003FF466AF04EB05150223AB7160E700BF37
:1051E000DC5C0020F45C0020DC4C0020F44C00204F
:1051F00010200020F90D000870B5104E3378022BF6
:105200000F4B0BBF020AC0F3D412C4B200F07F04EC
:10521000D3F8000282B010440D460023032201A9F6
:10522000FFF7C8FE012807D13378019A022B0CBF83
:1052300022F8145042F8245002B070BDDC4C00201B
:10524000DC5C00202DE9F04FDFF820910D4699F845
:1052500000102B68032985B0164640D0022966D17C
:105260004FEA132A5FFA83F84FF4807B421E012A2B
:1052700024D801249E421CD901288CBF002201227F
:10528000394F0192D7F878211AB1D7F89411994281
:1052900050D0D7F8000200235044092203A9FFF799
:1052A00089FE012824D0022815D020B12B689E4207
:1052B000E8D82E60032005B0BDE8F08FB8F1000FEC
:1052C00014D0294B93F8B42112B9012283F8B421E8
:1052D000012389F80130022005B0BDE8F08F4FF0BE
:1052E000800BC3F3D41A03F07F08BFE75C46C1E725
:1052F00099F80010022916D00329ECD1039B53F82A
:10530000282022F07042019BD5F800C0B2FA82F248
:1053100052099A4220D0A0440CEB0403D8452B60DC
:105320001DD20229EAD1039B33F81820EBE74FF492
:10533000807BD6E7D7F81012013A02EB41224902EE
:10534000B2FBF1F21344B3FBF4F204FB12320AB1E4
:1053500023449B1A2B60AAE76645ACD8A9E70AF15B
:10536000010A4FF00008A2E7DC5C0020DC4C0020C2
:105370002DE9F04FDFF850910B6899F800C01746FF
:1053800009F58052BCF1020FD2F8005283B08B466F
:10539000824640F08180DEB2A6EB030805EB1325C0
:1053A000B8444FF480729044BB4208F1FF38B8FB18
:1053B000F2F843D2A844BCF1030F06EB0704A4EBB8
:1053C000030414BF4FF4807280229442A8EB0503BB
:1053D00028BF1446B6BB944234BF0B220A2201A94F
:1053E0002846FFF7E7FD012829D199F800C0DBF82E
:1053F0000000BCF1020F00F1010325D0A64210D23B
:10540000019906F18042013A01EB8202043901EB75
:10541000840142F8043F8A4203F10103F9D1DBF829
:105420000000A31B0344BAF1010FCBF8003023D0D6
:105430009F4205F101054FF00006BCD8012003B0E2
:10544000BDE8F08F0B22CAE7A642EAD2019906F125
:105450000042013A01EB4202023901EB440122F819
:10546000023F8A4203F10103F9D1A31B0344BAF1BD
:10547000010FCBF80030DBD1BB42D9D1BCF1020F18
:10548000019B18D004F18044013C4FF0FF3243F8F7
:105490002420DBF80030CBE703F07F06C3F3D412FF
:1054A000BCF1030FA6EB03081544B84414BF4FF436
:1054B0008072802277E704F10044013C4FF6FF72CE
:1054C00023F814200120BAE7DC4C002030B5044654
:1054D000C06983B010B9012003B030BD0D46002370
:1054E000032201A9FFF766FD0128F5D1B4F92020B8
:1054F000002A19DB019B012D4FEA421103EB4212F6
:1055000003D0022D1BD1E5205854A368D361237822
:10551000032B04D10023137753779377D377636AF0
:1055200053831B0C9382D6E7064A92F8B41109B94B
:1055300082F8B401044B01225A700220CCE7E368E0
:10554000E4E700BFDC5C0020DC4C00202DE9F043E8
:10555000814683B00E4699F83C30042B00F28980D6
:10556000DFE803F02F03704F3F00434DDFF8108159
:105570004FF6F77705F5805418E0BA4260D872F01C
:10558000A1FB01284FF0000138D1D9F83000FFF716
:1055900033FE012832D1019AD4F81412C9F8302010
:1055A000531E8B4228BF0B46C4F814322A78D9F810
:1055B0003030032A01A918469AB2DED14345DED91C
:1055C0003EE0710001F0FE014846FFF77FFF012831
:1055D00043D1D9F83430002B18BF022089F83C00A1
:1055E000B9E799F82830042B04BF002389F8283044
:1055F000D9F838300BB148469847012003B0BDE8D0
:10560000F0831E48D9F82C20D0F89431C0F89421AA
:105610009B1AD0F8102202FB03F3D0F8782102EB9A
:105620004322C0F87821D0F87C2102EB4322C0F855
:105630007C21002100F5B870FFF748FF01280CD14C
:105640000420CBE7D9F8342009F130010020FFF71E
:105650008FFE012801D10320C0E70228CED199F89E
:105660002830042B04BF002389F8283003B0BDE89C
:10567000F0830220F3E700BFDC4C0020DC5C00205C
:10568000F7FFFF0F38B5044694F83430052B58D88F
:10569000DFE803F0372B2319100394F82830082B88
:1056A00004BF002384F82830274B012283F8B5215A
:1056B000022038BD94F82830082B04BF002384F85A
:1056C0002830012038BD00212046FFF7FFFE0128C9
:1056D00037D1042084F83400D6E7D4E90B01FFF772
:1056E0008BFD01282DD10320F4E7206B4FF0FF3113
:1056F000FFF782FD012824D1E36A002BF3D00220BA
:10570000E8E7114DD5F8082204F1300101200232FA
:10571000FFF798FD012805D00238C0B2012810D843
:105720000520D7E7E368D5F81012226BC5F81422DC
:1057300003EB4123C4E90332E36A002BCAD162625E
:10574000C8E7002038BD00BFDC5C002070B504460F
:1057500094F83830032B4BD8DFE803F01F170B0207
:1057600000212046FFF7B2FE431EDBB2012B40D9D9
:1057700070BD626B04F130010120FFF7F9FD0128D3
:10578000F2D1032384F83830E2E71F480021FFF705
:105790009DFE0128E8D10223F4E71C4AE56802F5E2
:1057A00080531278D3F81012D3F89401032A14BF4F
:1057B0004FF48072802202FB01F105EB4125C4E920
:1057C0000350D3F87851A5EB4125C3F87851D3F8AD
:1057D0007C51861AA5EB41210244C3F89421C3F8F9
:1057E0007C11E36AC4E90C025BB960620123C9E77A
:1057F000022094F82830062B04BF002384F82830B8
:1058000070BD2663F2E700BF4C5E0020DC4C002038
:105810002DE9F0434368C3F308020A44B2F5007F60
:1058200083B005460C4605D223446B60012003B0CB
:10583000BDE8F08390F91A20501C0AD0464902F5C1
:10584000817201EB0212D17921F00101D171FF22A5
:10585000AA7695F91B20511C16D03F4E02F5817295
:1058600006EB021106EB0212C979D079C1F34501AA
:10587000012986BF01F1FF3101F03F010021FF2620
:1058800061F34600D071EE762A78022ACCD0324EEF
:1058900006F58058D8F81022B4EB422F4FEA42297F
:1058A0002BDCD8F818721F407A42A24225DCE2199C
:1058B0004A45286913D32A7E120729D5D8F894219E
:1058C000411C8A421BD300D100214B44DB1BA4EBBB
:1058D0000909686109EB070429616B600846002823
:1058E000A4D03278032A31D080B24FF6F7729042BA
:1058F0009CD81A4614446C6098E7002097E798F803
:10590000B42102BB012388F8B43173706B68DCE703
:1059100001A972F0D7F90128EFD16B6829782869BD
:105920006861A4EB09049944A9EB070301986B6033
:1059300002293C4428611A46D1D1D8F82012B3EB91
:10594000412FD7D372E701227270BEE7034A90421B
:105950003FF66CAFCDE700BFDC4C0020F7FFFF0F38
:105960002DE9F047044682B094F83830032B00F25A
:10597000AB80DFE803F09A170C02236C002084F858
:10598000280003B19847022002B0BDE8F087236CDD
:10599000002284F828200BB120469847012002B04D
:1059A000BDE8F08723786668484F022B1CBF474B41
:1059B000D3F81832204618BF1E40FFF7DBFAC6F3B3
:1059C0004F26361A0546B6B2A7F5805811E0D7F82B
:1059D00010325A1E914557D2FFF71AFF40B997F877
:1059E000B43113B9012387F8B431012388F80130A9
:1059F000013506EB050C022201A9002328461FFAF7
:105A00008CF9FFF7D7FA01284FF400724FF000012C
:105A1000BAD101987CF0EEFFE3694FF400712046A3
:105A2000002BD4D06368002BD1D1019B4FF02032E2
:105A30004FF02E0C4FF0100EC3F80120C3F80520D4
:105A4000A3F8092083F800C042F62E6AD4F824C0D7
:105A5000A3F820A083F80BE0C3F82220C3F8262087
:105A600083F82A20E26BA3F81AC05A872CFA0EFC9E
:105A700022FA0EF283F82BE09A86A3F814C0D7F826
:105A800010325A1E9145A7D3C3EBC353590201F5F7
:105A900000712046FFF7BCFE28B997F8B4317BB1FE
:105AA0000B4B01225A70022007E02046FFF7EAFD67
:105AB000012802D0022807D1032084F8380053E7D8
:105AC000012387F8B431EBE700205DE7DC5C0020C0
:105AD000DC4C00202DE9F041B1F904300F2B82B0ED
:105AE0000E460446174632D02046FFF743FA94F993
:105AF0001B80B8F1FF3F3BD05C4B41F2180203EB37
:105B000008118A58904211D1183303EB4825B38805
:105B100001331BB205EB4315B38020463D60FFF710
:105B200029FA3060012002B0BDE8F08103F580520F
:105B300092F8B41100295CD001225A702378022B0C
:105B40004CD02269002A60D100233B60EAE74FF481
:105B50000071FFF75DFE002847D04FF6FF73B3805A
:105B60002046FFF707FA94F91B80B8F1FF3FC3D135
:105B70002378022B41D02269002AE5D03B4B1B78C9
:105B8000032B69D093B24FF6F7718B4294BF002379
:105B90000123002BD6D138B9354B93F8B421002A14
:105BA0004DD0324B01225A700023112201A9FFF778
:105BB00001FA012810D1019D2E4BEB1A48BF03F2C8
:105BC000FF13B3F5805F4FEA63222DD24FFA82F8BC
:105BD00084F81B80002D9AD12378B0E7244A6368AB
:105BE000D2F82022B3EB422FAED2002002B0BDE8A3
:105BF000F081012182F8B4119EE71D4BD3F82022D9
:105C00006368B3EB422FC6D39EE7184B1B78032B78
:105C100019D093B24FF6F772934294BF0023012339
:105C2000002B91D10020E1E7114B93F8B42112B978
:105C3000012283F8B4210D4B01225A70C8E70122DA
:105C400083F8B421ADE70C4B9A4294BF00230123A3
:105C5000002B7FF479AFE5E7074B9A4294BF00230E
:105C60000123002B7FF46EAF95E700BFDC4C0020D2
:105C7000DC5C0020F44C0020F7FFFF0F2DE9F0431F
:105C8000044689B094F83030042B11D8DFE803F0D3
:105C9000501361035A00237E9A0640F1FA80E069AE
:105CA0000023112204A9FFF785F9012800F0F180F3
:105CB00009B0BDE8F083C64D03AE04F11C073246BF
:105CC00039462846FFF706FF012800F0FD8002282C
:105CD000EED1C04901F5805595F9D2315A1C0AD050
:105CE00003F5817301EB0313DA7922F00102DA7113
:105CF000FF2385F8D23195F9D3315F1C16D003F517
:105D0000817301EB031201EB0313D279D979C2F34A
:105D10004502012A86BF02F1FF3202F03F02002253
:105D200062F34601FF22D97185F8D321042306E0EE
:105D3000A74872F0FDF84FF6FF720123228484F821
:105D400030309FE70020E36A207009B0BDE8F043DF
:105D50001847A14D95F8E031002BA9D104F11C079B
:105D600003AE05F5DC78324639464046FFF7B2FE11
:105D7000012840F01A81039B002B00F0F4801A7870
:105D8000E52A01D0002AEED19449591A48BF01F200
:105D9000FF11B1F5805F4FEA612280F050818D499B
:105DA00012018F480244907B04280CD0D5F898004B
:105DB0000130C5F89800506004209073D5F89C20FD
:105DC0000132C5F89C2095F9D221561C0AD002F563
:105DD000817201EB0212FF2085F8D201D07920F008
:105DE0000100D07195F9D321501C18D002F58170B3
:105DF00001EB001201EB0011D279C2F34502012A36
:105E00004FF0FF0088BF02F1FF3285F8D301C87957
:105E10008CBF02F03F02002262F34600C8711846B0
:105E2000202200217CF0E6FDD4F83120D4F8351092
:105E300041600260B4F8392094F83B10817202810D
:105E4000627EC272019005A802F0CAFF019B002881
:105E500000F0DE809DF816009DF817209DF81910BF
:105E600042EA4012BDF81400A0F2BC7042EA40229F
:105E70009DF81A00490141EA50019DF8180041EAD5
:105E8000C02192B288B2D9811A821A83D8820323A0
:105E900055E7204672F04CF82369002B00F08A8009
:105EA000237E03F0F70213F00403227640F09A8079
:105EB000122A00F0B080E36A0022204684F82820ED
:105EC00009B0BDE8F0431847DDF80C80B8F1000FC9
:105ED00000F0C18098F80030002B00F0BC8098F8EA
:105EE0000B9019F0080F7FF4EAAE0B2204F1310198
:105EF00040467BF0D9FB00287FF4E1AE637E89EA5F
:105F00000303D90640F1E680324901F5805595F941
:105F1000D2315A1C0AD003F5817301EB0313FF221F
:105F200085F8D221DA7960F30002DA7195F9D3218C
:105F3000571C3FF4FBAE02F5817201EB021301EB3B
:105F40000212DB79D179C3F34503012B86BF03F13C
:105F5000FF3303F03F03002363F34601FF23D171B6
:105F600085F8D331E2E695F8B831022B4FF00902FB
:105F70003FF4DCAE95F8E031002B7FF4D7AEC5E9F5
:105F80007D3385F8F03185F8EC31D5F8CC31C5F8A2
:105F9000E4310F48D5F8143285F8E021C5F8E8312E
:105FA000FFF7DEFC01283FF4DEAE02287FF480AE6E
:105FB0000423C4E6237E1B077FF57DAF064B93F8D1
:105FC0009821002A7FF474AE072283F8982172E7A3
:105FD000945E0020DC4C0020DC5C0020F44C0020AF
:105FE000F45C0020A568E66A002384F8283029467E
:105FF0002046FFF70DFC002866D194F82830002BCE
:106000007FF456AE0223C4E90B6584F828304FE6CE
:1060100044F2817238E7626AE16AA163042084F87D
:1060200028002046C4E90B22C4E9023384F83C303E
:106030006363636209B0BDE8F04371F079BF95F81E
:10604000B42112B9012285F8B421454901224A70D0
:106050006FF00F02A5E6424901F5805595F9D2315E
:106060005F1C0AD003F5817301EB0313DA7922F088
:106070000102DA71FF2385F8D23195F9D3315E1C24
:1060800016D003F5817301EB031201EB0313D279F0
:10609000D979C2F34502012A86BF02F1FF3202F02C
:1060A0003F02002262F34601FF22D97185F8D32115
:1060B000237ED8067FF53AAE2A4871F039FF4FF6B5
:1060C000FF72022322843AE6002E3FF4F1AD20460F
:1060D00033463AE6B8F81420B8F81A30224D43EAAD
:1060E00002436362D5F81022D8F81C30A360520234
:1060F000B3FBF2F102FB113109B113445B1AE36007
:1061000084F8199095F9D23115495E1C0AD003F52F
:10611000817301EB0313DA7922F00102DA71FF23B4
:1061200085F8D23195F9D321501C3FF4B0AE02F579
:10613000817201EB021301EB0212DB79D179C3F317
:106140004503012B86BF03F1FF3303F03F03002318
:1061500063F34601FF23D17185F8D33197E600BF81
:10616000DC4C0020945E0020DC5C002070B50378DD
:10617000017E023B012B044602D911F0060F68D1C3
:106180008D0643D494F91A30581C0AD0374A03F5C7
:10619000817302EB0313FF20DA7922F00102DA7136
:1061A000A07694F91B305A1C16D0304803F5817242
:1061B00000EB021300EB0210DB79C279C3F3450355
:1061C000012B86BF03F1FF3303F03F03002363F38A
:1061D0004602FF23C271E3760B070ED5244B93F8DA
:1061E0009821072A06D093F8B421002A38D01F4AF4
:1061F00001215170002283F89821E26A0023237064
:1062000084F8283022B3BDE87040104700231948B5
:10621000E5691A018258954206D00133082BB1D0A6
:106220001A0182589542F8D1104803F5817300EBAA
:106230000312D279C2F34502012A15D9013A02F0BC
:106240003F0200EB0313D87962F34600D87199E757
:1062500070BD0121FFF73AF90128F9D1217E8FE7BE
:10626000012283F8B421C2E70022EAE7DC4C0020D7
:10627000DC5C0020F45C002038B5184D05F5805436
:10628000014694F8E00120B961B191F8283013B1CA
:1062900038BD002038BD04F5DC7044227BF088FA5C
:1062A000012038BD44220E487CF0A4FB2B78D4F8A2
:1062B0001C12C4F8DC1103224FF6FF70022B18BF2A
:1062C0001346A4F8D20184F8D021054884F8B831E7
:1062D000102284F8D12171F02BFEE1E7DC4C002084
:1062E000945E00204FF0FF3C2DE9F041344A354DDB
:1062F0006446002304E00133082B02F1100216D09B
:1063000010780428F7D103F5817005EB0010C179EE
:10631000CE07F0D4601C52F80A1C01D08C45EAD993
:106320001C460133082B8C4602F11002E8D1002CE8
:1063300002DA0120BDE8F081224DDFF8948004F5F7
:10634000817705EB07139988D8F8683DF9B92601DC
:10635000D8F8683DDFF87C802E4441F2180208EB43
:106360004421B058EBB1DC68174A0023A047C0B104
:1063700002280AD108F6E87805EB0715D8F89C3012
:106380000122013BC8F89C30AA710020D2E705EB3E
:10639000041041F218022601805813B19B689847F7
:1063A000D6E70A4BD3F89C2005EB07150320013AEA
:1063B0000121C3F89C20A87183F8A010E5E700BF75
:1063C000025D0020DC4C00206D0E0008DC5C00202B
:1063D00010200020F44C00202DE9F04390F82830E4
:1063E000013B83B00446082B0BD8DFE803F0393DAE
:1063F0001F24052A0A2F34000121FFF7A7F80128DE
:1064000002D003B0BDE8F0832378216C002284F829
:106410002820002BF5D0D4E9010383424FF003027A
:1064200038BF0346A36084F82820E162204603B009
:10643000BDE8F0439AE6002103B0BDE8F043FFF762
:1064400085B803B0BDE8F043FFF780B903B0BDE8FD
:10645000F043FFF717B903B0BDE8F043FFF780BA88
:1064600003B0BDE8F04309E4534F4368D7F818522E
:10647000026BD7F8101290F800C01D4005EB020E19
:10648000BEEB412F4FEA4126184645D3A7F5805968
:106490004FF6F778BCF1020F14D0216908460029A5
:1064A0005ED16068A368E26A834238BF0346002178
:1064B000A36084F82810002AA3D0204603B0BDE8CA
:1064C000F04310476068D7F82012B0EB412F68D234
:1064D0002069217E090735D5D7F8941100F1010E06
:1064E00071452BD297F8B41100294BD1012387F8BD
:1064F000B43189F8013094F800C06368226B921BB4
:106500002A4433445B1B9642C4E904E0636022637F
:1065100018464FF00005BDD9BCF1020F41D02169EA
:106520000029BFD0254B1B78032B40D089B24FF6F2
:10653000F7739942B6D810446060B3E7DFD14FF0EB
:10654000000EDCE701A971F0BDFB01287FF459AF13
:106550002069DDF804E094F800C06368226BCEE7A0
:1065600099F800E0BEF1030F12D01FFA81FEC64574
:1065700094BF4FF0000E4FF0010EBEF1000FA8D0F7
:106580006068CDE7012189F8011094F800C0B6E7F2
:10659000DFF82CE0714594BF4FF0000E4FF0010E74
:1065A000EBE7D7F82032B0EB432FC4D37AE7044BA4
:1065B00099423FF677AFBEE7DC5C0020DC4C002060
:1065C000F7FFFF0F70B5194D194BC5F89C3B194BE0
:1065D00085F8A81B002683F8186A05F69C33C0E9E5
:1065E00054330D23C0F8583140F201130446C0F86B
:1065F0005C6100F5A271A0F8443174F0FDFA1F232C
:10660000C4E9EC36E378012205F599659342C4F8B4
:10661000A853A4F89C2308BFC4F8AC5304F56771D1
:106620002046BDE8704074F0E7BA00BF0831002092
:106630005553425310200020F0B50B7813F0600240
:1066400083B004462BD0202A30D14A78FE2A39D094
:10665000FF2A2DD14A88002A3BD1CA88002A38D186
:106660001F0636D46148624B80F8182AC4F8B42358
:10667000E278012183F8E814A4F89C1303F59963E8
:106680001F21012AC4F8B013C4F8A83304F56771B8
:1066900008BFC4F8AC33204674F0AEFA06E04B787D
:1066A0000A2B1AD00B2B08D0012B2AD0002002E095
:1066B00074F034F9022003B0F0BD4D4B4A8883F8E2
:1066C000AD2BF3E74F8827B9CD88012D01D11B06EB
:1066D00042D4204674F022F9ECE7022180F811112F
:1066E0004FF48071A0F81C1142490123C0E94A11FE
:1066F000C0E94E33C0E94C3200F58E7174F01AFADD
:10670000D4E78B88C0681E06DDB244D40192019A9A
:10671000394B42F010020192019A02610269019222
:10672000013B02D0019AD206F8D4314E29462046C8
:1067300074F066F9294696F8E85402234022204670
:1067400074F08EF9022DB1D18121204674F01EF92A
:10675000002386F8E834A9E7254ED6F800359B6972
:106760009847C0B286F8AC0B0028B2D0022306F6D8
:10677000AC3684F811314FF48073C4E94E55C4E946
:106780004A66C4E94C57A4F81C3104F58E712046C2
:1067900074F0D0F98AE70092009A174B42F0200279
:1067A0000092009A65F38A120092009A02610269CF
:1067B0000092013B02D0009A9106F8D40C4E294673
:1067C000204674F01DF9294696F8E8540223402229
:1067D000204674F045F9022DB6D0012D3FF466AF86
:1067E00001212046FFF7EEFE60E700BF10200020E9
:1067F00008310020B53C0020410D030010B50D4BC1
:1068000093F8183A022B07D0033B012B02D8002142
:10681000FFF7D8FE002010BD074B93F8D5140446AF
:1068200074F09EFA0028F5DA01212046FFF7CAFE2F
:10683000F0E700BF1020002008310020F8B53F4CE1
:1068400094F8186A05467EB1012E01D00020F8BDEB
:106850003B4B93F8D51474F083FA0028F6DA3146EE
:106860002846FFF7AFFEF1E7354FB0F8B433D7F85D
:10687000D024C7F8A42B1F2BD7F8CC24C7F8A02B03
:1068800008D1304BD7F8C8249A4203D197F8D514D1
:10689000012919D997F8AE3B5A1CD2B207EBC303B2
:1068A000042A18BF1646052283F8B02B4FF4005275
:1068B0002846C3F8B42B022387F8AE6B87F8E83478
:1068C000FBF784FA0020F8BD97F8D634013B0F2B74
:1068D000E0D874F045FA002827DB94F8183A013B19
:1068E000022BB3D9B7F8D03B1BB3042284F8182A83
:1068F000154AC5F85C61C5E95422D7F8D02487F859
:10690000A86B934228BF1346D7F8A42BC5F858317B
:1069100040F20111A5F84411D21A05F5A2712846DA
:10692000C7F8A42B74F068F990E72846FBF74EFAF5
:106930008CE719462846FFF745FE87E71020002020
:106940000831002055534243DC3C002000207047B2
:10695000704700BF704700BFD0ED007AD0ED036AEA
:1069600030EE677AE6EE877AB0EE670AC0ED007A1D
:10697000704700BF90ED017AB5EE407AF1EE10FA63
:10698000F0EE407A09D19FED0D7A60EE870AF7EEBE
:10699000006A86EEA07A80ED017A31EE077A90EDFA
:1069A000000A80ED021AC1EE076A77EEC07AC0EDE8
:1069B000036AA6EEA70A80ED000A7047DB0FC94004
:1069C000D0ED056AD0ED017A90ED066AD0ED025A5D
:1069D00090ED035AC0ED066AB0EE407A26EEA70AA3
:1069E000D0ED007A80ED057AA7EE870AD0ED077A20
:1069F000A5EE860A90ED086AD0ED045AC0ED087A3B
:106A0000A5EE670AA5EEC60A80ED070A704700BF2B
:106A1000F0EE406AD0ED007A90ED050A90ED037A31
:106A200090ED016AD0ED025AA7EEA60AD0ED047AE5
:106A300027EE407A67EEC07AA6EE267AE5EEA67AD1
:106A400090ED066AC0ED067A36EE076A80ED056ABB
:106A5000704700BF03685A1C02601970704700BF7E
:106A60002DE9F04FD0E9003185684A1C00EB810424
:106A7000F1EE407A92FBF3F6002D03FB1622426002
:106A800089B084ED200AC4ED407A40F346815A185B
:106A90009FEDA46A0692591E6A1C079200F18009B4
:106AA00000F5807BF0EE466A02224FF0010A88462C
:106AB00006998C1A94FBF3F103FB1144611C91FBC2
:106AC000F3F003FB101101EB0A0009EB840E0BEB52
:106AD000840C924590FBF3F49EED007ADCED007A95
:106AE00003FB1400A3EB020680F2CD80CDE901EC9C
:106AF000CDE9032637460C460546059031E0A34212
:106B000009EB850C0BEB850605F1010531DD09EB81
:106B100084000BEB840E2246013490ED006AD6ED22
:106B2000005ADEED006AB4EEC76AF1EE10FA07DD36
:106B30009CED005AB4EEC56AF1EE10FA00F38680BF
:106B4000F4EEE76AF1EE10FA04DDF4EEE56AF1EE38
:106B500010FA13DC01374745B0EE467A2EDAF0EE34
:106B6000667AAB42CBDCA3425E46CC464FF00105D1
:106B7000CDDCDE46484601240022CEE7F4EEE75A9B
:106B8000F1EE10FA58BFF0EE657ABAF1010FCEEDD2
:106B9000007A18BF01200CD00132934200F10100AD
:106BA000CEBF0BEB82065E4600228245C6ED007A20
:106BB000F2D101374745B0EE677AD0DBDDE901EC71
:106BC000DDE903260598DEED006A9CED006A30E001
:106BD0008B4209EB800C0BEB800700F1010030DDEC
:106BE00009EB81050BEB810E0C46013195ED007A26
:106BF000D7ED005ADEED007AB4EEE67AF1EE10FA47
:106C000006D59CED005AB4EEC57AF1EE10FA4DD4DB
:106C1000F0EE476AF4EEC67AF1EE10FA04D5F4EE1F
:106C2000E57AF1EE10FA5DD4B0EE676A0136B04550
:106C300029DD8342CCDC8B425F46CC464FF001001D
:106C4000CEDCDE464D4601210024CFE7B4EEC75A24
:106C5000F1EE10FA58BFB0EE457ABAF1010F80EDAF
:106C6000007A3FF46DAF104601260130834206F1F1
:106C70000106CEBF09EB800CCC46002056458CEDBA
:106C8000007AF2D15CE707990AF1010A8A4502F11C
:106C9000020208F1FF387FF40BAF76EEC66AF6EE1B
:106CA000007A26EEA70A09B0BDE8F08FB4EEE65AE6
:106CB000F1EE10FAD8BFF0EE456ABAF1010FC5ED5A
:106CC000006AA7D0254601270135AB4207F101072D
:106CD000CEBF09EB850CCC4600255745CCED006AAC
:106CE000F2D197E7F4EEC65AF1EE10FAD8BFB0EE43
:106CF000656ABAF1010F8EED006A97D00125013463
:106D0000A34205F10105CEBF0BEB84075F460024CB
:106D1000554587ED006AF2D188E79FED020A09B078
:106D2000BDE8F08F0000000003685A1C0260197073
:106D3000704700BF024B186803681B68184700BF04
:106D4000005F0020007970470079C0F34010704761
:106D500000794009704700BF90F83C20034602F0DC
:106D6000FF0012B1002283F83C2070474FF480539B
:106D7000838170474FF40063838170474FF4006351
:106D8000838170474FF40063838170474FF4006341
:106D9000838170474FF40063838170474FF4006331
:106DA00083817047074B10B403F11001002453F89E
:106DB000042B824208BF43F8044C8B42F7D15DF8A4
:106DC000044B7047045F002070B5374C608CA38A79
:106DD000B4F92C50B4F92660B4F91AC01B1A208CEF
:106DE00000FB03F3B4F92A0005EBE335C00290FB86
:106DF000F5F000EBE330A0F57A6EB4F924302063AF
:106E00000EFB0EF52D1305FB06F605FB03F3B4F997
:106E10001C500EFB0CFC0EFB05F51B1403EB65333D
:106E20004FEAEC2CB4F918500CEBE62C0CEB850C6B
:106E30000233B4F93450A66BE48B9B1003F5004386
:106E40000CFA05FC04FB03F30CF1020C4CF2503479
:106E5000A6EBAC0C2C4104FB0CF4002C4FEAD33312
:106E6000ABBF6400B4FBF3F3B4FBF3F35B0089B195
:106E70001C120E4D04FB04F440F6DE3606FB04F44F
:106E800003FB05F5241404EB254404F6CF6403EB5F
:106E900024130B602AB100EB800040000830001181
:106EA0001060012070BD00BF005F002043E3FFFFC2
:106EB00001207047012070472DE9F04F734DE86BBA
:106EC000B5F84030B5F94CE0B5F948C0B5F84680A2
:106ED000B5F94E6085B0C3EB2014009204FB04F4B6
:106EE000B5F94420CDF80CE0241302FB04F45B0058
:106EF000B5F942200296C3EBE00302FB03F3A413AF
:106F000004EBE324EB6D0193A4F5FA30B5F94A30B4
:106F1000AC6580FB00EA4FEAE37B03FB0AF98CFBDC
:106F200000C20EFB0B99A3FB0E3BCB4412031B0AC2
:106F300042EA1C5243EA0B634FEA0C3C13EB0C038E
:106F400042EB2B22A3FB083C02F5004208FB02CCDB
:106F50004FEAEC734FEA6C0953EA6C0C0F46B5F933
:106F6000501000F09180029E019A86FB0008C2F545
:106F7000801C01FB0AFA4A464FEA48484FEAE17989
:106F800048EAD0380EFB09A94004A1FB0E1E4118A7
:106F9000F14449EB080900200CF00048039E411819
:106FA00048EA5C084FEACC7CBCEB010C09EBC60953
:106FB00068EB09081CEB0C0E48EB08011EEB0C0EED
:106FC00048EB010188014FEA8E1940EA9E601EEBF2
:106FD000090E41EB0001890041EA9E714FEA8E0ED5
:106FE0001EEB0C0E48EB01014FEA8E00890010EBFE
:106FF0000C0041EA9E7148EB010175F0D3FCB5F934
:1070000056304FEA61384FEA503E4EEAC14EDA1729
:1070100003FB08F984460EFB0299B5F95400B5F953
:107020005220A3FB0E35A94403FB08F50EFB0955BE
:10703000A3FB0E3E75445B0E43EAC51313EB0C0332
:1070400041EB65654FEAE07E00FB01F10EFB0C11A0
:10705000A0FB0C0C6144C00C40EA41301B1845EB0E
:10706000E1451B0A43EA056303EB02130FB11B0A58
:107070003B60009B23B104EB8404803424121C6029
:10708000012005B0BDE8F08F0023EFE7005F00208E
:1070900031B10A4BD3ED1F7AFDEEE77AC1ED007AEC
:1070A00052B1064B9FED067AD3ED207A67EE877AD0
:1070B000FDEEE77AC2ED007A01207047005F002004
:1070C0000000C8422DE9F04F614DB5F89230D5F877
:1070D0008400B5F890E0B5F88E40B5F8946085B0BE
:1070E0001B02C01A67EB0707B5F88C300191AEFBA5
:1070F000001C0EFB07CCC9091B0441EA4C61C918EE
:107100009346A4FB003EB5F88A2004FB07EE4FEA45
:1071100013234FEAC23243EA0E634FEAEC1C4CF1F0
:10712000000C9B18A6FB002406FB07444FEAD25232
:1071300042EA44224FEA2E2E4EF1000EE41512F5DB
:10714000FA6944F10006B9F5FA6F029676F1000685
:1071500032DAA2FB02A802FB04F6039408EB460411
:107160004FEA84084FEA8A0616EB0A0648EA9A783C
:1071700044EB08084FEA560A4AEAC87AB608B1EB67
:107180000A0A46EA8876334C6CEB680C9E1B334641
:10719000029E6EEBA80EA1454FF0FF34A64151466A
:1071A00027DB00FB07F7A0FB000202EB4702C00F42
:1071B00040EA4200B9EB0009019C8CB1D5F8980077
:1071C000A0FB033200FB0E225B0D43EAC2235B1AD5
:1071D0004FEA625262EB0C02DB0B43EA424323604C
:1071E000BBF1000F01D0CBF80090012005B0BDE845
:1071F000F08F40F6AC56039C921944F1000402FB58
:1072000004F4A2FB026202EB44024FEAC208F4005B
:10721000341B48EA567862EB080864184CEB080CFB
:107220002146B41942EB0208A41942EB08084FEAC0
:10723000880848EA9478A400A41B68EB0208620856
:1072400042EAC8729A1A6EEB680E1346A9E700BFAD
:10725000005F002024FAFFFF0120704710B40F4B9D
:107260000F4C1B68D4F89C001B1AFA2B0BD811B1D9
:10727000D4F8A4300B6012B1D4F8A8301360012008
:107280005DF8044B7047074A1368002023F004039D
:1072900084F8A00013605DF8044B7047242A002096
:1072A000005F002000000010064B00220021C3F800
:1072B000AC20C3F8B020C3F8B420C3F8B810012044
:1072C000704700BF005F0020104B114A1B68D2F8C6
:1072D000B8105B1AFA2B16D8D2ED2B6A92ED2C7AE5
:1072E000D2ED2D7AFDEEE66ABDEEC77A16EE903A43
:1072F000FDEEE77AC38617EE103A038717EE903A51
:107300004387012070470020704700BF242A0020D7
:10731000005F002030B50F4A83B092F8BC50019155
:10732000B5B9D2F8C0509DB12B681A6882B19B687C
:1073300073B104462846984750B12B6801992246FC
:107340001C6828460B46214603B0BDE8304008477C
:1073500003B030BD005F00200B4B70B5D3F8C460A4
:107360008EB133681A6872B19B6863B105463046C6
:107370000C46984738B133682A4619683046234688
:10738000BDE87040084770BD005F0020024BD3F895
:10739000C8305B68184700BF005F0020024BD3F87D
:1073A000C83008309B681847005F002001207047F4
:1073B0000120704738B51446002944D0344BDFED26
:1073C000355AD3ED337AB3F9E82093ED360AB8EEA7
:1073D000E77A05EE102AC7EE256AB3F9E4200D46D8
:1073E000D3ED347A06EE102AF8EEE77AB3F9E62008
:1073F000C7EEA54A05EE902AB3F9E22007EE102A5F
:10740000F8EEE55AB3F9E020B8EEC77A07EE902A15
:10741000A6EEA57AB8EEC55AB8EEC66AF8EEE77AD7
:10742000A6EE856AE6EE877A93ED377AB8EEC77AEC
:10743000B8EEC00AA6EE867AA6EE870AA4EEA70AE0
:1074400076F03AFA28600CB3114B9FED126AD3ED37
:10745000347AB3F9D620B3F9D430F8EEE76A07EE00
:10746000102A86EE860A07EE903AB8EEC77AF8EE52
:10747000E77A20EE070AB6EE006AA7EE860ADFED8D
:10748000066A20EE260A76F017FA2060012038BD41
:10749000005F00200000F04A0000C8422DE9F041E2
:1074A0000446D0E90030134483421DD80D4601EB59
:1074B0000208B2B104F10C07002601E0A84510D083
:1074C00023695A1C2261234415F8011B1973042AED
:1074D000F4D139462046FBF74BFBA845C4E90460CC
:1074E000EED16069BDE8F0814FF0FF30FAE700BFF0
:1074F000034690F910002DE9F04116469A68224C97
:1075000000EB8000920754F8208009D5404674F0C3
:107510009FF93146404674F09BF90120BDE8F081A7
:107520005D69084615B12B68AA885A83174B184F16
:107530001C68184B7A684FEAC40CA3FB0C3C4FEA5A
:107540009C1C7B689B1A9C45FBD20146404674F00C
:107550007FF93146404674F07BF90E4B78680C4950
:107560004FF4FA7204FB02F2A3FB023292094B6859
:107570001B1A9A42FBD2002DCFD02B68AA881A83FF
:107580000120BDE8F08100BF400D0020AC36002096
:10759000001000E0D34D621000680379012B0AD07F
:1075A000022B01D0002070478368DB074FF0F00208
:1075B00018D5FF219CE700B5826890F910C0417C86
:1075C00085B002F0010201920DF10F0200926046B7
:1075D000FF224FF0F00C8DF80FC0FCF79DFF05B0B7
:1075E0005DF804FB7F2183E700680379CA4341EA21
:1075F0000211012BCAB208D0022B01D00020704723
:107600008368DB0716D5D22172E700B585B090F903
:1076100010C08DF80F208268417C02F001020DF14C
:107620000F00CDE90002D2226046FCF775FF05B0DD
:107630005DF804FB52215BE700680379012B0AD057
:10764000022B01D0002070478368DB074FF0B402A3
:1076500018D5FF214CE700B5826890F910C0417C35
:1076600085B002F0010201920DF10F020092604616
:10767000FF224FF0B40C8DF80FC0FCF74DFF05B0A2
:107680005DF804FB7F2133E700680379012B09D003
:10769000022B01D0002070478368DB070A4616D50D
:1076A000A52125E700B5826890F910C085B002F0E9
:1076B00001028DF80F10417C0DF10F00CDE90002A1
:1076C000A5226046FCF728FF05B05DF804FB2521E4
:1076D0000EE700BF00680379012B0AD0022B01D00E
:1076E000002070478368DB074FF0960218D5FF2112
:1076F000FEE600B5826890F910C0417C85B002F0CA
:10770000010201920DF10F0200926046FF224FF03C
:10771000960C8DF80FC0FCF7FFFE05B05DF804FB7A
:107720007F21E5E600680379012B09D0022B01D007
:10773000002070478368DB070A4616D58721D7E605
:1077400000B5826890F910C085B002F001028DF892
:107750000F10417C0DF10F00CDE900028722604639
:10776000FCF7DAFE05B05DF804FB0721C0E600BFB8
:1077700000680379C901012BCAB205D0022B01D0E0
:10778000002070477821B3E600B585B090F910C0AD
:107790008DF80F208268417C02F001020DF10F008C
:1077A000CDE9000278226046FCF7B6FE05B05DF830
:1077B00004FB00BF00680379012B0AD0022B01D023
:1077C000002070478368DB074FF0550218D5A521CC
:1077D0008EE600B5826890F910C0417C85B002F059
:1077E000010201920DF10F0200926046A5224FF0B6
:1077F000550C8DF80FC0FCF78FFE05B05DF804FB4B
:10780000252175E600680379012B0AD0022B01D0EF
:10781000002070478368DB074FF02E0218D5F42153
:1078200066E600B5826890F910C0417C85B002F030
:10783000010201920DF10F0200926046F4224FF016
:107840002E0C8DF80FC0FCF767FE05B05DF804FB49
:1078500074214DE6144B00689A8E037992013432FC
:10786000012BD2B208D0022B01D0002070478368D0
:10787000DB0716D5F4213BE600B585B090F910C0C2
:107880008DF80F208268417C02F001020DF10F009B
:10789000CDE90002F4226046FCF73EFE05B05DF83B
:1078A00004FB742124E600BF005F002000B50068DF
:1078B0000379012B85B012D0022B03D0012005B033
:1078C0005DF804FB8368DB074FF031024CBFF42105
:1078D0007421FFF70DFE012005B05DF804FB8268FE
:1078E00090F910C0417C02F0010201920DF10F02EB
:1078F00000926046F4224FF0310C8DF80FC0FCF777
:107900000BFE012005B05DF804FB00BF00680379A1
:10791000012B06D0022B01D00020704701225821F4
:10792000E6E500B5826890F910C0417C85B002F0B0
:10793000010201920DF10F020092604658228DF86B
:107940000F30FCF7E9FD05B05DF804FB0068037932
:10795000012B06D0022B01D00020704701224821C4
:10796000C6E500B5826890F910C0417C85B002F090
:10797000010201920DF10F020092604648228DF83B
:107980000F30FCF7C9FD05B05DF804FB0068037912
:10799000012B06D0022B01D0002070471A46082187
:1079A000A6E500B5826890F910C0417C85B002F070
:1079B000010201920DF10F020092604608224FF081
:1079C000020C8DF80FC0FCF7A7FD05B05DF804FBB5
:1079D00000680379012B06D0022B01D000207047EC
:1079E0000122082184E500B5826890F910C0417C2D
:1079F00085B002F0010201920DF10F020092604683
:107A000008228DF80F30FCF787FD05B05DF804FB08
:107A10002DE9F0410C4E356873691D4011D0DFF837
:107A20002C800127B5FA85F4C4F11F0408EB840308
:107A300007FA04F4D3F8EC0003689847A54374618F
:107A4000F0D1BDE8F08100BF003C0140005F0020A4
:107A50002DE9F04F604BD3F82C9191B0B9F1000FA4
:107A600004D05E4A03214846FBF7C6F90021484688
:107A7000FBF73AFAD9F80430594DD3F800801F6962
:107A80000022560105EB4210A959794011F47C54AB
:107A900002F1010208D0102AF3D10023C9F80C30FA
:107AA000002011B0BDE8F08F027FC9F80C00002A59
:107AB000F6D1B8F84420DFF840A16FEA42426FEAFD
:107AC000524292B2A8F84420B8F8002092B242F094
:107AD0008002A8F8002093F805B09B791AF80B10E3
:107AE000B8F820205B074CBF042301238B409BB2D6
:107AF00092B222EA0302A8F82020B8F820203949DF
:107B000092B21343A8F82030B8F8003042689BB214
:107B100043F00103A8F80030334B9A42334A136B09
:107B20000CBF43F4001343F48003136306F11802FF
:107B30004FF0070C354421F802C04B462C49032274
:107B4000FBF736FCAD682846FBF744FE2B6823F0B4
:107B500001032B602846FBF73DFE0023CDE90C33E3
:107B6000CDE90E3306930A93BBF1030F05D8DFE886
:107B70000BF0302D022A08F13C04FFB20AEB870A11
:107B800040F62B4205921B48DAF8043001934FF47B
:107B900080614FF48042079109924FF48051402256
:107BA000CDE9030208914FF40033284601A90B9355
:107BB000029470F00DF92B68012043F010032B6044
:107BC00011B0BDE8F08F08F14004D6E708F13804A1
:107BD000D3E708F13404D0E7005F0020009F2400C1
:107BE000F80A0020FC0A0020006002400038024031
:107BF000A1020008447500205C3D080838B5104D0E
:107C0000D5F82C4124B10F4A64212046FBF7F4F843
:107C100000212046FBF768F96368012285F83021CE
:107C20001A68B2F844306FEA43436FEA53439BB299
:107C3000A2F8443013889BB243F00103138038BD8F
:107C4000005F0020009F240010B54FEA511E02443F
:107C500000EB8E0C624529D901F01F034FF0FF3471
:107C600050F82E1004FA03F30B4093FAA3F3B3FA7F
:107C700083F3DBB2202B16D10CF104018A4202D827
:107C800017E08A4212D98C460431DCF8003093FAAE
:107C9000A3F3B3FA83F3DBB2202BF2D0ACEB000CEE
:107CA00003EBCC0010BD03EB4E1010BD4FF0FF30C6
:107CB00010BD204610BD00BF0369416890ED067AF3
:107CC000F0B4C56A394E876853EA010204BF3168CF
:107CD00041606A1C30EE077A0133012A80ED067A92
:107CE0000361C26240D090ED075AD0ED096A346852
:107CF00007EE902A70EE455AB8EEE76A611AC5EEB3
:107D0000867AB94277EE857A30EE670AC0ED087A56
:107D1000E5EE806AC0ED077AC0ED0A6AC0ED096A37
:107D200001D8F0BC7047012A29DD07EE905AF8EE21
:107D3000E77A86EEA76AB5EEC06AF1EE10FA1EDBAE
:107D4000F1EEC67AF4EE677AF1EE10FA17D6D0EDBE
:107D5000056AF4EEE76AF1EE10FA13D5037BEBB196
:107D60000323F0BC03707047326880ED080A521A92
:107D7000BA424FF0000180ED070A4162D1D9DFED30
:107D80000C7AE4E707EE903AF8EE677A0223C7EE42
:107D9000276AF0BC0370C0ED066A70473168416025
:107DA000002203618261C362BBE700BF242A002076
:107DB00000000000DFED4F4A10B5844600F1480E88
:107DC0000346B1EC017AD3ED067ADA6A77EE877A68
:107DD0000132012AC3ED067ADA6254D093ED075AD4
:107DE00093ED096A07EE902A77EE455AF8EEE77AA6
:107DF000C5EEA76A76EE857AF0EE466A37EE677AC8
:107E0000C3ED087AE5EE876AC3ED0A6AC3ED077A27
:107E1000C3ED096A18337345D3D1374C41682268E2
:107E20000369521A816801338A4203612AD990EDAD
:107E3000056A00F1300EDCF82C20DCED0A6A012A1C
:107E400002F1FF3126DD07EE901AF8EEE77A86EEB2
:107E5000A77AB5EEC07AF1EE10FA1BDBF1EEC77A25
:107E6000F4EE677AF1EE10FA14D6E645B4EEE76A5E
:107E70000CF1180C16D0F1EE10FADCD5037B6BB3C5
:107E80000323037010BDF0EE477AF0EE646A83EDD1
:107E9000087ABBE7DFED177AE645B4EEE76A0CF146
:107EA000180CE8D1F1EE10FAE8D407EE903AD0EDD4
:107EB000066A90ED0C7AD0ED125AF8EE677A02233A
:107EC00086EEA76A0370C7EE276A85EEA77A80ED73
:107ED000066AC0ED0C6A80ED127A10BD002221689E
:107EE000416003618261C362026343648264C3656B
:107EF00010BD00BF00000000242A0020B0EEC06AC0
:107F0000F0EEE05AF4EEC65AF1EE10FAF0EE407AD6
:107F10000EDCB5EE400AF1EE10FA4BD0F4EEC65A84
:107F2000F1EE10FAF0EE466A50D5B0EE655A03E075
:107F3000F0EE656AB0EE465A85EE267A9FED252A68
:107F40009FED253A9FED254ADFED254ADFED252AF5
:107F5000DFED253ADFED256AA7EE023AE7EE223A99
:107F6000A7EE034AB7EE005AE7EE044AA7EE235AFB
:107F7000E7EE246AF4EEC65AB1EE667A87EE050A99
:107F8000F1EE10FA48BF9FED1A7AF5EEC00A48BF2D
:107F900037EE400AF1EE10FA48BF9FED167AF5EE83
:107FA000C07A48BF37EE400AF1EE10FA48BFB1EE92
:107FB000400A7047DFED107A9FED100AF5EEC00A17
:107FC000F1EE10FA58BFB0EE670A7047B0EE465AAD
:107FD000B2E700BF39094E3DE3B59EBE88FA16BE32
:107FE00045FE7FBF99FB243F69A2163EA7DFA8B4D8
:107FF000DB0FC93FDB0F4940A7DFA834DA0F494048
:1080000091ED007AD0ED047A90ED054AD0ED064A64
:1080100090ED075AD0ED085A90ED096AD0ED0A6A42
:10802000E7EE077AF7EE003AC0ED047A91ED007AB8
:10803000D1ED017AA7EE274A90ED0B7A80ED054A43
:1080400091ED024A91ED003AD0ED0C7AE3EE044A4C
:10805000C0ED064AD1ED004A35EE245A80ED075AAC
:10806000D1ED014A91ED005AE4EE855AC0ED085A6F
:10807000D1ED015AA5EEA56A80ED096AD1ED015A4C
:1080800091ED026AE5EE866AC0ED0A6AD1ED016AF9
:1080900037EE267A80ED0B7AD1ED026A91ED007A07
:1080A000E6EE877AC0ED0C7A91ED026AD1ED016AB5
:1080B000D0ED0D7A90ED0E7A90ED0F4AD0ED104A8A
:1080C00090ED115AD0ED135AE6EE267A75EEA35ACA
:1080D000C0ED0D7AD1ED026AD0ED127A90ED006A12
:1080E000A6EEA67AD0ED016A80ED0E7A91ED027AC5
:1080F00034EE074A90ED027A80ED0F4A91ED004A86
:1081000074EE844AC0ED104AD1ED014A35EE245A8E
:1081100080ED115A91ED025AC0ED135A77EE857A2F
:10812000C0ED127AD1ED017AD1ED005A91ED025AEB
:1081300067EEA77AE5EEA57AE5EE057AA5EEA76AE1
:1081400080ED006A91ED016AE6EE276AC0ED016AF2
:10815000D1ED026AA6EEA77A80ED027A90ED037A5D
:1081600077EE277AC0ED037A704700BF2DE9F04F14
:108170004FF0000989B0864600F110050646034617
:1081800000F13008074648462C46CDF80CE08B46F7
:108190009C46B24600283CD10CF1040CA445FBD10E
:1081A000032800F1010151D09C46AA46029398B1E0
:1081B000DCED047A0192AAEB0903B6467246F3ECB1
:1081C000016A92ED007AE6EEC77A53450EF1100E81
:1081D000CCED047AF2D1019ADCED046A15ED047A53
:1081E000C6EE877A0CF1100CC4450AF1100ACCEDEA
:1081F000007ADCD1029B04361433084608F10408E7
:1082000014351034103709F104099C46B246002891
:10821000C2D0DCED007A0192D64639467246F1ECC6
:10822000016A92ED007AE6EEC77A99420EF1100EDD
:10823000CCED007AF2D10CF1040CA445019A0AF1BC
:10824000040AE6D1032800F10101ADD1DDF80CE00C
:108250000023594604930593069307937646774681
:1082600004AD0020F2EC017AE5EC017AB0B104AC87
:108270003B46B4EC017AF3EC016AE6EEC77AB3420E
:1082800045ED017AF5D1013004280BD0F2EC017AEA
:1082900010371436E5EC017A0028E8D1103714368F
:1082A0000120DFE708AD75ED017A10310EF1400EC7
:1082B00004287446A1F1040241ED017A1ED07346F0
:1082C000F3EC016AB1EC017AE6EEC77AA342C2EDA3
:1082D000007AF5D15EED016A87EEA67A013882ED6B
:1082E000007A17D0AEF1140E103C114675ED017AEC
:1082F0000428A1F1040241ED017AE0D15EED016AAA
:1083000087EEA67A103CAEF1140E032001ED017A3F
:108310001146EBE709B0BDE8F08F00BFDFED297A29
:10832000B4EEE70AF1EE10FA28DD9FED277A30EE81
:10833000470AB4EEE70AF1EE10FAF8DCDFED237A33
:10834000B4EEE70AF1EE10FA2FDD30EE670A37EEF1
:10835000C00A60EE007A9FED1E7A9FED1E6ADFED87
:108360001E6AA7EE876A9FED1D7AE7EE866A60EEC9
:10837000275AA7EEA67AA5EE870A7047DFED187A8E
:10838000B4EEE70AF1EE10FAD8D59FED0F7A30EE91
:10839000070AB4EEE70AF1EE10FAF8D4DFED0B7A33
:1083A000B4EEE70AF1EE10FACFDC9FED0E7AB4EEF0
:1083B000C70AF1EE10FA44BF30EE270A37EE400A42
:1083C000C7E700BFDB0F4940DB0FC940DB0FC93FE8
:1083D0009A7C2E36FAAF4FB93587083CA4AA2ABE3C
:1083E000DB0F49C0DB0FC9BF10B5404CB4FBF2F442
:1083F000A14219D3DFED3E7AF7EE005AB0EE677A6C
:10840000B0EE676AF0EE676A0023C0ED005AC0ED77
:10841000017A80ED027A80ED036AC0ED046A83611F
:1084200043610362C36110BD07EE902AB8EE677A1C
:10843000DFED307A27EE277AB7EE006AC6EE076ADC
:1084400007EE901A9FED2C7AF8EE677AB0EE405A5C
:1084500067EE877AC7EEA64AFDEEE47A17EE902A19
:108460002032402A3FD8B0EE640AFFF757FFB0EE43
:10847000404ADFED227A34EEA70AFDEEC07A17EE0D
:10848000902A2032402A29D8FFF748FFF8EE006AE8
:1084900060EE266A012B1CD0B7EE006A36EE406A09
:1084A000F6EE004A66EE244A35EE055AF7EE007AFB
:1084B00084EE057A77EE275A37EEC75A84EEA57A0E
:1084C000C6EE257A86EEA56AC5EE256AF0EE475A15
:1084D0009AE7B0EE666AF7EE004AE5E7DFED086A74
:1084E0009FED030AD6E79FED024AC2E720A10700ED
:1084F00000000000BD378635DB0FC940DB0FC93FE8
:1085000000000080DFED077A30EE270AFDEEC07A2A
:1085100017EE903A2033402B00D8FFE69FED020A79
:10852000704700BFDB0FC93F000000002DE9F84F86
:10853000DDF82CB09DF828408946002C1BF8011B63
:108540000CBF4FF020084FF030081C1E05461746A0
:1085500008463ADB00295CD0002C55D04FF0000AC9
:108560005B4600E064B313F8016B013C002EF9D1C7
:10857000BAF1000F2FD1264644B14D454146284659
:1085800000D2B847013CF8D10B9B18780146A0B146
:108590004FF0FF344FF0000A00E09B464D4528465F
:1085A00000D2B8475B4613F8011B0029F5D10B9B9D
:1085B000F61A5E44BAF1000F10D13046BDE8F88FCC
:1085C000BAF1000F1BD15646E0E7634229B31C46BF
:1085D0004FF0010AC4E70028E0D10646002C04F160
:1085E000FF3AEADD54464D454146284600D2B84799
:1085F000013CF8D2013656443046BDE8F88F0646B5
:108600000028DAD02646C9E72646A2464FF0FF34B6
:10861000C4E72646002CB0D1CFE76FEA040A0E4625
:10862000E0E700BF0FB430B583B006AB0A4C53F897
:10863000042B0193D4E9D30173F04CF9054620686B
:1086400003685B6998470028F9D0284603B0BDE865
:10865000304004B0704700BF005F00200EB410B57A
:1086600083B005AB044653F8042B0749009301A8D7
:10867000019473F02FF9019B00221A7003B0BDE83A
:10868000104003B0704700BF296D00080CB4F0B56E
:108690003C4CD4F85433ADF5277D002B6DD094F8C5
:1086A0005C3399420BD9D4F86023012383401342F1
:1086B00005D10DF5277DBDE8F04002B07047324B83
:1086C000324A1B68A2FB030292094FF47A7101FB44
:1086D000123306A82E49FFF7C1FF06AB03442D490C
:1086E000AC9A01930646ADAB01A8009373F0F2F883
:1086F000019B0A22591C01911A70019B0022591CEE
:1087000001911A70D4F85453ADB12B685B6A1BB158
:1087100028469847D4F854539DF818100029C8D01B
:108720000DF119042B6828461B68984714F8011BA3
:108730000029F7D1BDE7D4F85873002FB9D03044E1
:1087400026AB841CFD2206A9ADF81020184622464F
:10875000CDF81250ADF8165079F02AF802220346EF
:10876000044402A93846CDE9023438F0C1FF0DF5C2
:10877000277DBDE8F04002B07047D4F85833002B95
:108780008DD196E7005F0020242A0020D34D62108F
:10879000F0E30808556A0008184A10B5D2F8644397
:1087A000033004EB9003B3F5007F18D802EB81018E
:1087B000C2F8643302F55A7202EB8404D1F8682BD4
:1087C00020F003001044C3F50073C1F8680B0C4A95
:1087D0009B0004210020FFF759FF204610BD002117
:1087E0000846084AFFF752FF074AD2F8B030002483
:1087F00043F00073C2F8B030204610BD005F002087
:10880000FCE3080820E408080000001038B50568FB
:10881000EB690446F3B1987800B938BDB3F90A2082
:1088200007EE902AF8EEE77A0120C4ED057AB3F955
:108830000C2007EE902AF8EEE77AF1EE677AC4EDA5
:10884000047AB3F90E3007EE903AF8EEE77AC4ED09
:10885000067A38BD09211420FFF79EFF0346E86120
:10886000D9E700BF38B50568EB690446E3B19878ED
:1088700000B938BDB3F9042007EE902AF8EEE77A84
:108880000120C4ED047AB3F9062007EE902AF8EE31
:10889000E77AC4ED057AB3F9083007EE903AF8EEBE
:1088A000E77AC4ED067A38BD09211420FFF774FF7A
:1088B0000346E861DBE700BF38B50568EB690446AD
:1088C000E3B1987800B938BD9A88D2BA07EE902AF9
:1088D000F8EEE77A0120C4ED047ADA88D2BA07EE1E
:1088E000902AF8EEE77AC4ED057A1B89DBBA07EE29
:1088F000903AF8EEE77AC4ED067A38BD09211420E3
:10890000FFF74AFF0346E861DBE700BF38B50468BC
:10891000E3690D467BB1987800B938BD5B89094A97
:10892000DBBA82FB0312DB17C3EB221303F26D13D6
:108930002B80012038BD09211420FFF72DFF0346AD
:10894000E061E8E7797878782DE9F04103EB4306B8
:10895000964602EB460612F9067B86B0034675463C
:1089600092F80080A3EB0804A3EB070C002CB8BF1F
:108970006442BCF1000FB8BFCCF1000C6445B8BF35
:10898000154602F10602B8BF4FFA88F7B242E7D1A6
:108990006A889EF80000B842144614D1BEF802005E
:1089A000A1EB0008A1EB020CB8F1000FB8BFC8F1B1
:1089B0000008BCF1000FB8BFCCF1000CE045BEBF11
:1089C0007546024604460EF1060E7645E1D16A79F7
:1089D00004922A79CDE902422878054ACDE90010AF
:1089E00003210120FFF752FE284606B0BDE8F081C2
:1089F00030E408084B1EDBB2062B9CBF214A02EB79
:108A0000430330B598BF9D8E1F4BA3F1580488BF18
:108A10004FF48075002808BF1C46A44620893CF806
:108A2000082B87B04FFA82FE90B1A5EB0E022B1AED
:108A3000002AB8BF5242002BB8BF5B429A42C4BF63
:108A400064464FFA80FE3CF8080F0028EDD12288DA
:108A50000E4B0F4893F8F0CBA3790593A3880493AA
:108A60000C4BBCF1000F18BF0346A078CDE90015F0
:108A7000CDE902200321084A0120FFF707FE204626
:108A800007B030BD5C3D0808A0160020005F002044
:108A9000BCF608080CE308086CE4080803685A1CD4
:108AA00002601878704700BF03681A46591C0160BD
:108AB00012F8021B0260587841EA0020704700BF9C
:108AC00010B402681346511C016013F8021B0360C6
:108AD000D31C5478036093781B0443EA0423141DC9
:108AE0000460D0785DF8044B0B4343EA00607047A4
:108AF00012B370B50446864604E0981B17D114EBF8
:108B00000C0C15D01EF8013BA3F14100192811F8F7
:108B1000010BA0F1410598BF2033192DA2EB0E0CDB
:108B200000F12006E9D91B1A04D10028E7D170BD55
:108B3000604670BD184670BD1046704710B402887C
:108B40008378184C02F0030101EB4101013B03EB78
:108B5000810304EB4303C178B3F84430A2F5FA6211
:108B6000920840F2B55404FB02334A1E13440179C3
:108B700042798479008903EB430301EBC301C1EB24
:108B80000111094B02EB8102C2EB0212234403EBF9
:108B9000820300214FF47A72C3FB02015DF8044B9B
:108BA000704700BF5C3D080880436D38F8B5164635
:108BB0001F460446394630464FF47A72002373F05C
:108BC000F1FE3C4D3C4B054483FB05602844E9170E
:108BD000C1EB601183FB01030B44384EC817C0EB97
:108BE000631086FB003CC317354EC3EBAC0386FB1A
:108BF00003764FEAE37ECEEBE61EC1EB0116A5EB52
:108C0000860CC0EB0015A1EB8501617103EB4301FC
:108C1000A0EBC10040F2B55101FB1E33B3F5896FE3
:108C200084F806C020714FEA8E0637DA40F2DA2166
:108C30008B4239DCB3F5B77FB4BF4FF0000E4FF075
:108C4000010E20490EEB4E0001EBC0017546B1F854
:108C50005A004FEA4E071C4907EB0E0C01EBCC0CF7
:108C60000CF1160C0B2101E03CF8020D984212DDCC
:108C70000139F9D11349774401EBC701B1F8440038
:108C80000121013306F5FA6E1B1A7544A170E370D9
:108C900022812580F8BD0131C9B2F2E7032540F2F7
:108CA0009650AE460627D6E7022540F22940AE464A
:108CB0000427D0E780BC92C789888888ABAAAA2AF3
:108CC00073B06D165C3D0808A03D080830B52F4C08
:108CD00086460D460FCC8DB0EC46ACE80F000FCCAD
:108CE000ACE80F0094E80F001EF0030F8CE80F00B3
:108CF0000FD1274B274A03FB0EF3B2EBB30F43D33D
:108D0000254AB2EB331F34BF01220022C2F11D02FB
:108D100000E01C220EF1FF33002B019240F26D1295
:108D2000194602FB0EF2B8BF0EF1020102EBA102DE
:108D30001A491B4C81FB0301DB17A3EB61100244B2
:108D4000C3EBE1131A44253284FB02311144D317DB
:108D5000C3EBA103C3EBC303D31AADF10402EE4688
:108D600002EB85015EF8040FC21884FB023C9444B8
:108D7000D317C3EBAC03C3EBC3037145A2EB0303EF
:108D8000F0D1C01A0DB030BD1D22C3E7003E080867
:108D9000295C8FC2285C8F020AD7A3001F85EB5184
:108DA000932449920C4B10B553E9024354EA030251
:108DB00009D1014640F201130020C1F80230887148
:108DC0000880088110BD054A1268121943F100039A
:108DD000FFF7ECFE012010BD006B0020242A0020CC
:108DE00030B5144DD5F8F81BD5F8FC3B51EA030219
:108DF00083B0044609D1002040F201132080C4F85A
:108E00000230A071208103B030BD0B4A12685218A5
:108E100043F10003FFF7CAFEB5F8003CADF8063099
:108E200020460DF1060221466EF0ACFE012003B093
:108E300030BD00BF005F0020242A002088422DE9B9
:108E4000F0414FF001043DD301FB04F4B0FBF4FC0E
:108E50008C45F9D23CB3002616E0BCF1090F274639
:108E600098462C4623DD002A0CBF4FF0570E4FF0DA
:108E7000370EF444B94288F800C003F1010306F14B
:108E8000010610D8B0FBF5FCB4FBF1F504FB1C00A7
:108E9000002EE2D1BCF1000FDFDCA1420AD90CF1B7
:108EA000300C03F801CB00221A70BDE8F0814FF0BE
:108EB000300EDEE7B0FBF5FC2C4605FB1C00B5FBD5
:108EC000F1F5E7E78446C6E72DE9F0410446944210
:108ED0001546084609D2B4FBF2F6154B05FB1644BD
:108EE0001B5D00F8013BBDE8F081B4FBF2F6964251
:108EF000B6FBF2F70CD20E4B05FB176705FB1644C9
:108F0000DA5D00F8012B1B5D00F8013BBDE8F08144
:108F1000BA42B7FBF2F807D9054B05FB187813F8EE
:108F2000082000F8012BE7E74046FFF7CDFFF3E705
:108F3000B8E40808B5EEC00ADFED347AF1EE10FAB5
:108F4000CCBF30EE270A30EE670ADFED317A20EE33
:108F5000270A30B5FDEEC07A87B017EE904A054675
:108F600084EAE470002303A9A0EBE470CDE90033A8
:108F700002936EF07BFF002CB4BF2D23202303A8A7
:108F80008DF8003072F0F4FE012829D0022833D089
:108F900003281DD003A968467AF0E4FB684672F006
:108FA000E7FEC41EE4B222466946284678F000FC7B
:108FB00000232B55284672F0DBFE2E232B54013064
:108FC0000DEB040128447AF042FC284607B030BD7E
:108FD000302303A968468DF801307AF0C3FBDDE742
:108FE00043F23002302303A96846ADF801208DF822
:108FF00003307AF0B7FBD1E743F2300303A96846A8
:10900000ADF801307AF0AEFBC8E700BF6F12033A4B
:1090100000007A440278202A034600F10100F9D0CA
:10902000092AF7D02D2A29D02B2A03BF5A78B7EE68
:10903000000A0346B7EE000AA2F13001C8B20928BF
:10904000DFED4C7A10D8F2EE046A07EE101AB8EE93
:10905000C77A13F8012FA7EEA67AA2F13001C8B2A1
:109060000928F0EE477AF0D92E2A49D0197801F074
:10907000DF01452907D020EE270A70475A78BFEE56
:10908000000A0346D8E710B459782D2962D02B295D
:1090900054D0A1F13002092A03F1010355D800246C
:1090A000002202EB820201EB420213F8011FA1F140
:1090B00030000928A2F13002F3D9B2F59A7F1346A5
:1090C00028BF4FF49A73072A50D9DFED2B6A1A464E
:1090D000B7EE007A083A072A27EE267AFAD803F084
:1090E00007032BB1F2EE046A013B27EE267AFBD18F
:1090F0006CB3C7EE877A5DF8044B20EE270A704701
:109100005978A1F13002D0B2092803F10103AED899
:10911000F2EE046AF0EE665A07EE102AB8EEC77A4D
:1091200013F8011F87EE266AA1F13002D0B2092898
:1091300066EEA56A77EE867AEED998E79978A1F17E
:109140003002092A03F10203A9D9B7EE007A67EECB
:10915000877AD0E79978A1F13002092A03F1020356
:1091600088BFB7EE007AC4D8012499E7B7EE007A39
:10917000B7E700BF0000000020BCBE4C0378202BE6
:10918000024600F10100F9D0092BF7D02D2B08BFC2
:109190005378A3F13001CBB206BF02464FF0FF3C3B
:1091A0004FF0010C092B4FF0000000D9704712F866
:1091B000013F00EB800001EB4000A3F13001CBB296
:1091C000092BF4D90CFB00F0704700BF70B5344D8B
:1091D0002B787E2B01D0002070BD08224FF4FC4379
:1091E00041F2210019B200294FEA4303B6BF80EAD9
:1091F00041019BB28BB2013AF4D1B5F8011069B3C9
:109200002848294CA042E6D206384618A642E2D2A7
:1092100041F2210C0529DED9864214D0013806F12D
:10922000FF3E10F8012F082183EA02231AB2002A18
:109230004FEA4303B6BF8CEA42029BB293B20139B4
:10924000F4D17045EDD1318849B1B21DA242C2D2EC
:109250007218A2423046BED21646DBE7134E741E89
:1092600041F22100A44614F8012F082183EA0223C9
:109270001AB2002A4FEA4303B6BF80EA42029BB209
:1092800093B20139F4D16645ECD17288D01A084AFC
:10929000331D5B1BB0FA80F04009A2F8043C70BD9E
:1092A00000000E0807000E080000100801000E085C
:1092B000005F00202DE9F04F914B924A8BB00020C7
:1092C000D21ACDE90600CDE90800D11805928E4AE0
:1092D0000393049110690028C0F281818A4AF32027
:1092E000D060002008908948012288428DF824200F
:1092F00000F271817E2007928DF818004FF4FC4235
:10930000082041F2210514B2002C4FEA4202B6BFF8
:1093100085EA440492B2A2B20138F4D17C48ADF897
:1093200002207C4A90427CD2804641F22105B8F866
:109330000200B8F80020C0F30B07C2F30B04120BB5
:10934000BE1D4FF000098DF808200204ADF804603E
:10935000ADF806408DF8099000F1C38006338B42CA
:1093600000F2398101AE0DF10A0B344601E0A3454C
:1093700013D0079B14F8011B03F128026A44013340
:10938000042B079302F8101CF1D106A903A8F9F7E2
:10939000EFFBA345CDE90790EBD1089B002BC0F272
:1093A0001A81BDF8024016F8013B082284EA032422
:1093B00023B2002B4FEA4404B6BF85EA4303A4B2AC
:1093C0009CB2013AF4D1B345EDD1D8F804603A46E5
:1093D000314603A8FEF762F80028C0F2FC80F019BD
:1093E000864213D0711E013811F8013F082284EA29
:1093F000032423B2002B4FEA4404B6BF85EA43039B
:10940000A4B29CB2013AF4D18142EDD1DDE903026C
:10941000ADF8024011463F4A08F114089045034652
:1094200085D302334FF000089942ADF80480C0F0B4
:10943000D28001AD2E460DF106042F4601E0BC425C
:1094400013D0079B17F8011B03F128026A4401336C
:10945000042B02F8101C0793F1D106A903A8F9F711
:1094600087FBBC42CDE90780EBD1089B002BC0F203
:10947000B280BDF8023041F2210016F8012B83EAD8
:109480000223082219B200294FEA4303B6BF80EA3B
:1094900041019BB28BB2013AF4D1B442EDD10399B0
:1094A000ADF80230049B0231994200F294800DF134
:1094B0000206144602E0B54200F08A80079B16F8C7
:1094C000011B03F128026A440133042B02F8101C2B
:1094D0000793F0D106A903A8F9F74AFBCDE90740A5
:1094E000E9E7CB460BF1010B06335FFA8BFB9942A0
:1094F0008DF809B06FD301AE0DF10A0A34460DE0C4
:1095000000000E0800001008003C024001000E0898
:109510008061090834670908A24515D0079914F835
:1095200001CB01F128030DEB030001310429079160
:1095300000F810CCF0D106A903A8F9F719FB002315
:10954000A24508900793E9D1089A002A43DBBDF8A9
:10955000024016F8012B082184EA022422B2002AD4
:109560004FEA4404B6BF85EA4202A4B294B201397C
:10957000F4D1B245EDD1D8F8041001EB09063A4612
:10958000314603A8FDF78AFF002824DBF019864244
:1095900013D0711E013811F8013F082284EA032418
:1095A00023B2002B4FEA4404B6BF85EA4303A4B2BA
:1095B0009CB2013AF4D18142EDD1DDE90302BBF165
:1095C000030FADF8024003461146B9448AD121E7A2
:1095D000089B002B09DA00200BB0BDE8F08F15487E
:1095E000506000F18830506078E6079840B9124921
:1095F0000A6942F000420A61B3FA83F04009EBE7DE
:10960000DDE9033203449342E5D806ABC0F104021E
:109610000021184479F0EEF906A903A8F9F7A8FA91
:10962000002803460890D6DB9DF82420002AE3D0CA
:10963000DDE700BF23016745003C024008B5FFF7A6
:1096400039FE40B9FFF736FE28B9FFF733FE10B9EF
:10965000052007F035F9FFF7B9FD0028F8D008BD5F
:10966000034AD2F8083C23EA0003C2F8083C7047DA
:10967000005F002070B545880B460446C5F30B0516
:109680002A460021184679F0B5F90A4A2169914223
:10969000034606D3084A914206D3BDE870401846F7
:1096A00008470029F9D170BD2A46BDE8704078F01E
:1096B0007FB800BF34670908576C090810B50379F3
:1096C000012B84B08E460ED0022B02D0002004B0B5
:1096D00010BD8368DB0758BF01F07F0104B0BDE80F
:1096E0001040FDF705BF144682688DF80F4002F068
:1096F000010201920DF10F020092417C90F91000DD
:109700007246FAF709FF04B010BD00BFF8B5782221
:10971000074600210068FFF7D1FF052607F074F81F
:1097200004460D4607F070F8001B61EB0501B0F52B
:109730007A7F71F10001F5D3013EEFD13868202224
:109740000121FFF7BBFF052607F05EF804460D4632
:1097500007F05AF8001B61EB0501B0F57A7F71F153
:109760000001F5D3013EEFD1324638680221FFF700
:10977000A5FF642607F048F804460D4607F044F8B4
:10978000001B61EB0501B0F57A7F71F10001F5D3A3
:10979000013EEFD10120F8BDF8B5072207460A21A6
:1097A0000068FFF78BFF052607F02EF804460D46EC
:1097B00007F02AF8001B61EB0501B0F57A7F71F123
:1097C0000001F5D3013EEFD1386824224121FFF793
:1097D00075FF052607F018F804460D4607F014F843
:1097E000001B61EB0501B0F57A7F71F10001F5D343
:1097F000013EEFD13868C0224221FFF75FFF052606
:1098000007F002F804460D4606F0FEFF001B61EB70
:109810000501B0F57A7F71F10001F5D3013EEFD17A
:109820000120F8BD10B50446002221210068FFF791
:1098300045FF2068FC222021FFF740FF20684022DE
:109840002421FFF73BFF20680C222321FFF736FF7E
:10985000206800222221FFF731FF012010BD00BF48
:10986000F8B50122074610210068FFF727FF00B96D
:10987000F8BD142606F0C8FF04460D4606F0C4FFE6
:10988000001B61EB0501B0F57A7F71F10001F5D3A2
:10989000013EEFD13868A022BDE8F84011210DE764
:1098A00010B5044600680379012B84B011D0022B57
:1098B00002D0002004B010BD01220B21FDF718FEDC
:1098C0000028F6D020681D22092104B0BDE8104010
:1098D000F4E6826890F910C0417C8DF80F3002F0F8
:1098E000010201920DF10F02009260460B22FAF77D
:1098F00013FEE5E710B50446C06900B110BD0921AB
:109900001420FEF749FFE06110BD00BF0C4B0D496C
:109910001A680D4B10B44FF4FA7404FB02F2A3FB67
:1099200002324C6892094B681B1B9A42FBD2436976
:1099300013B11A689B8813835DF8044B704700BF0E
:10994000AC360020001000E0D34D621010B1036867
:1099500082881A83704700BF10B1036882885A83D7
:10996000704700BF10B5174C04EB8000406830B35F
:1099700000EB400004EB800393F90DCCBCF1FF3FFA
:109980001ED093F8150CD0B104EB0C0293F8140C14
:1099900092F860EC8C23142103FB0CFC00220CEBEE
:1099A000000304EB43030139B3F8643C704412FA3A
:1099B00083F2F4D1044BA3FB0230C0F30F1010BDAF
:1099C000002010BD005F0020CDCCCCCC30B50320F2
:1099D00083B00D461446FFF7C5FF01909DB107EE19
:1099E000900A9FED0B7AF8EE677AF0EE006A67EE68
:1099F000877AB8EE047AA7EEA67ADFED067A67EEEC
:109A0000277AC5ED007A0CB1034B236003B030BD5B
:109A10006740533A00007A443313904370B5104BBB
:109A2000104CA3421AD2054602E00C33A34215D2D1
:109A300093F805C08C45F8D193F804C0AC4501D02B
:109A4000002DF2D1D8799042EFD1186890F804E057
:109A5000E645EAD106689E42E7D170BD002070BDA0
:109A6000586C0908146E09080379022B00D070475E
:109A700010B490F910201C4C1C4883B00831694484
:109A800002EB8202009450F8222011F8084C184989
:109A90008A4224D0A1F578418A4222D001F5806122
:109AA0008A4218D1118821F04001090403EB830395
:109AB000090C118000EB83001388C16823F0380380
:109AC00031F824101B041B0C0B43138013889BB22A
:109AD00043F04003138003B05DF8044B704700234C
:109AE000E0E70123DEE700BF00010203400D002094
:109AF00000300140F8B50468002107462046FFF712
:109B0000B3FFB62214212046FFF7D8FD642606F0E5
:109B10007BFE04460D4606F077FE001B61EB050157
:109B2000B0F57A7F71F10001F5D3013EEFD18122CA
:109B300010213868FFF7C2FD06F066FE04460D46A8
:109B400006F062FE001B61EB0501B0F57A7F71F152
:109B50000001F5D3802215213868FFF7AFFD06F02C
:109B600053FE04460D4606F04FFE001B61EB050157
:109B7000B0F57A7F71F10001F5D338680321BDE8B3
:109B8000F84071E7F8B50468002107462046FFF762
:109B90006BFFB6227E212046FFF790FD642606F07B
:109BA00033FE04460D4606F02FFE001B61EB050157
:109BB000B0F57A7F71F10001F5D3013EEFD1324665
:109BC00038687C21FFF77AFD642606F01DFE044606
:109BD0000D4606F019FE001B61EB0501B0F57A7F1A
:109BE00071F10001F5D3013EEFD1386804227D21E7
:109BF000FFF764FD642606F007FE04460D4606F0F6
:109C000003FE001B61EB0501B0F57A7F71F10001E5
:109C1000F5D3013EEFD18C2240213868FFF74EFD8D
:109C200006F0F2FD04460D4606F0EEFD001B61EB6A
:109C30000501B0F57A7F71F10001F5D302224121CF
:109C40003868FFF73BFD06F0DFFD04460D4606F0E1
:109C5000DBFD001B61EB0501B0F57A7F71F10001BE
:109C6000F5D338680221FFF7FFFE4FF40063BB8194
:109C7000F8BD00BF2DE9F041076882B08046B622EA
:109C80007E213846FFF71AFD642606F0BDFD044626
:109C90000D4606F0B9FD001B61EB0501B0F57A7FBA
:109CA00071F10001F5D3013EEFD102213846FFF7F3
:109CB000DBFE7B6913B11A689B88538306F0A4FD11
:109CC00004460D4606F0A0FD001B61EB0501B0F552
:109CD0007A7F71F10001F5D37B6913B11A689B8813
:109CE00013830A2606F090FD04460D4606F08CFD0F
:109CF000001B61EB0501B0F57A7F71F10001F5D32E
:109D0000013EEFD132467C213846FFF7D7FC06F002
:109D10007BFD04460D4606F077FD001B61EB050157
:109D2000B0F57A7F71F10001F5D300225921384650
:109D3000FFF7C4FC06F068FD04460D4606F064FD1E
:109D4000001B61EB0501B0F57A7F71F10001F5D3DD
:109D500097F91030BA688D4903EB83035E209207B0
:109D600051F823408DF8070040F1E48001230DF104
:109D700007020021204671F01BFD4FF4A473844AB2
:109D80002046002171F014FDBB689B0740F1E5807F
:109D90000A2606F039FD04460D4606F035FD001B87
:109DA00061EB0501B0F57A7F71F10001F5D3013E59
:109DB000EFD1012259213846FFF780FC06F024FD3F
:109DC00004460D4606F020FD001B61EB0501B0F5D1
:109DD0007A7F71F10001F5D38C2240213846FFF7DC
:109DE0006DFC06F011FD04460D4606F00DFD001B4E
:109DF00061EB0501B0F57A7F71F10001F5D3032223
:109E000041213846FFF75AFC06F0FEFC04460D4699
:109E100006F0FAFC001B61EB0501B0F57A7F71F1E9
:109E20000001F5D35B4CD8F8382098F83500B4FB26
:109E3000F2F2032391B2584AFEF786FD4388B4FB41
:109E4000F3F4C8F840400279422142F0C00238469B
:109E5000FFF734FC06F0D8FC04460D4606F0D4FCAF
:109E6000001B61EB0501B0F57A7F71F10001F5D3BC
:109E7000082243213846FFF721FC06F0C5FC0446C2
:109E80000D4606F0C1FC001B61EB0501B0F57A7FC1
:109E900071F10001F5D3042258213846FFF70EFC7A
:109EA00006F0B2FC04460D4606F0AEFC001B61EB6A
:109EB0000501B0F57A7F71F10001F5D30A22532133
:109EC0003846FFF7FBFB06F09FFC04460D4606F004
:109ED0009BFC001B61EB0501B0F57A7F71F100017D
:109EE000F5D300227C213846FFF7E8FB06F08CFC16
:109EF00004460D4606F088FC001B61EB0501B0F539
:109F00007A7F71F10001F5D306227D213846FFF7F3
:109F1000D5FB06F079FC04460D4606F075FC001BE7
:109F200061EB0501B0F57A7F71F10001F5D302B064
:109F3000BDE8F0817B6913B11A689B885383174B86
:109F400017491A68174B4868D200A3FB02329209DE
:109F50004B681B1A9A42FBD208E7104B10491A684B
:109F6000104B48684FF4FA7404FB02F2A3FB023270
:109F700092094B681B1A9A42FBD27B69002B3FF473
:109F800007AF1A689B88138302E700BF400D0020CB
:109F9000303E080840420F00783F0808AC360020E9
:109FA000001000E0D34D62102DE9F041836B07688B
:109FB0005A4A5B4DB5FBF3F10446062389B290F88B
:109FC0003500FEF7C1FC00214388B5FBF3F5804660
:109FD00025643846FFF748FD80226B213846FFF79D
:109FE0006DFB642606F010FC04460D4606F00CFCE2
:109FF000001B61EB0501B0F57A7F71F10001F5D32B
:10A00000013EEFD1032268213846FFF757FB642653
:10A0100006F0FAFB04460D4606F0F6FB001B61EB6A
:10A020000501B0F57A7F71F10001F5D3013EEFD162
:10A0300001226B213846FFF741FB0F2606F0E4FBB7
:10A0400004460D4606F0E0FB001B61EB0501B0F590
:10A050007A7F71F10001F5D3013EEFD118221B2167
:10A060003846FFF72BFB0F2606F0CEFB04460D46C5
:10A0700006F0CAFB001B61EB0501B0F57A7F71F1B8
:10A080000001F5D3013EEFD118221C213846FFF71D
:10A0900015FB0F2606F0B8FB04460D4606F0B4FB90
:10A0A000001B61EB0501B0F57A7F71F10001F5D37A
:10A0B000013EEFD198F804201A213846FFF7FEFA46
:10A0C0000F2606F0A1FB04460D4606F09DFB001B83
:10A0D00061EB0501B0F57A7F71F10001F5D3013E26
:10A0E000EFD198F8052019213846FFF7E7FA6426E2
:10A0F00006F08AFB04460D4606F086FB001B61EB6A
:10A100000501B0F57A7F71F10001F5D3013EEFD181
:10A1100038460321BDE8F041A6E400BF8C3F0808A3
:10A1200040420F002DE9F041836B0768654A664D98
:10A13000B5FBF3F10446062389B290F83500FEF72B
:10A1400003FC00214388B5FBF3F5804625643846BF
:10A15000FFF78AFC80226B213846FFF7AFFA6426AE
:10A1600006F052FB04460D4606F04EFB001B61EB69
:10A170000501B0F57A7F71F10001F5D3013EEFD111
:10A18000072268213846FFF799FA642606F03CFB5F
:10A1900004460D4606F038FB001B61EB0501B0F5E7
:10A1A0007A7F71F10001F5D3013EEFD132466B2188
:10A1B0003846FFF783FA642606F026FB04460D4670
:10A1C00006F022FB001B61EB0501B0F57A7F71F10F
:10A1D0000001F5D3013EEFD101226B213846FFF794
:10A1E0006DFA0F2606F010FB04460D4606F00CFB38
:10A1F000001B61EB0501B0F57A7F71F10001F5D329
:10A20000013EEFD118221B213846FFF757FA0F26DF
:10A2100006F0FAFA04460D4606F0F6FA001B61EB6A
:10A220000501B0F57A7F71F10001F5D3013EEFD160
:10A2300018221C213846FFF741FA0F2606F0E4FAEF
:10A2400004460D4606F0E0FA001B61EB0501B0F58F
:10A250007A7F71F10001F5D3013EEFD198F8042027
:10A260001A213846FFF72AFA0F2606F0CDFA0446DF
:10A270000D4606F0C9FA001B61EB0501B0F57A7FC7
:10A2800071F10001F5D3013EEFD198F805201921B5
:10A290003846FFF713FA642606F0B6FA04460D4670
:10A2A00006F0B2FA001B61EB0501B0F57A7F71F19F
:10A2B0000001F5D3013EEFD138460321BDE8F0415E
:10A2C000FFF7D2BB8C3F080840420F002AE700BFCF
:10A2D000F0B5046883B0074600212046FFF7C4FBB1
:10A2E0000C2225212046FFF7E9F90A2226213868A9
:10A2F000FFF7E4F9002263213868FFF7DFF93868D7
:10A3000081222721FFF7DAF9142606F07DFA0446A8
:10A310000D4606F079FA001B61EB0501B0F57A7F76
:10A3200071F10001F5D3013EEFD10C2225213868EF
:10A33000FFF7C4F90A2226213868FFF7BFF90F2278
:10A3400063213868FFF7BAF9386881222721FFF7BF
:10A35000B5F90A2606F058FA04460D4606F054FAF6
:10A36000001B61EB0501B0F57A7F71F10001F5D3B7
:10A37000013EEFD1032301AA102138466DF03CF8CD
:10A380000A2606F041FA04460D4606F03DFA001B87
:10A3900061EB0501B0F57A7F71F10001F5D3013E63
:10A3A000EFD19DF804009DF805109DF806202C4B78
:10A3B000803080318032A3F8AC0FA3F8AE1FA3F831
:10A3C000B02F25210C223868FFF778F90A222621C0
:10A3D0003868FFF773F9324663213868FFF76EF982
:10A3E000386881222721FFF769F90A2606F00CFA5E
:10A3F00004460D4606F008FA001B61EB0501B0F5B6
:10A400007A7F71F10001F5D3013EEFD10DF1030226
:10A410000123022138466CF0EFFF01230DF1030206
:10A42000092138466CF0E8FF38680C222521FFF737
:10A4300045F938680A222621FFF740F938681222C8
:10A440006321FFF73BF9812238682721FFF736F9AE
:10A4500038680321FFF708FB012003B0F0BD00BFFF
:10A46000005F00202DE9F04105461F4695F91030A8
:10A47000234803EB8303164650F82380AB689A0702
:10A480000ED5404671F0E4F93B4632460021404685
:10A4900071F08EF9AB689B0718D50120BDE8F081FB
:10A4A0006B6913B11A689B885383164B164A1B6855
:10A4B0004FEAC30E154BA2FB0E2E5A684FEA9E1EA2
:10A4C0005C68A4EB020CE645FAD2DAE70D4B0F49C3
:10A4D0001A680D4B4FF4FA7000FB02F2A3FB023234
:10A4E000486892094B681B1A9A42FBD26B69002B91
:10A4F000D3D01A689B8813830120BDE8F08100BF88
:10A50000400D0020AC360020D34D6210001000E05A
:10A5100030B50579012D83B08E460DD0022D02D0C5
:10A52000002003B030BD8468E40758BF41F08001CB
:10A5300003B0BDE8304095E714468268009402F00D
:10A540000102417C90F9100001927246F9F7E4FF94
:10A5500003B030BD2DE9F04105461F4695F9103096
:10A56000234803EB8303164650F82380AB689A0711
:10A570000ED5404671F06CF93B460022314640460C
:10A5800071F016F9AB689B0718D50120BDE8F08182
:10A590006B6913B11A689B885383164B164A1B6864
:10A5A0004FEAC30E154BA2FB0E2E5A684FEA9E1EB1
:10A5B0005C68A4EB020CE645FAD2DAE70D4B0F49D2
:10A5C0001A680D4B4FF4FA7000FB02F2A3FB023243
:10A5D000486892094B681B1A9A42FBD26B69002BA0
:10A5E000D3D01A689B8813830120BDE8F08100BF97
:10A5F000400D0020AC360020D34D6210001000E06A
:10A6000030B50579012D83B08E460DD0022D02D0D4
:10A61000002003B030BD8468E40758BF41F08001DA
:10A6200003B0BDE8304095E714468268009402F01C
:10A630000102417C90F9100001927246F9F738FF4F
:10A6400003B030BD2DE9F043836B0768804A814C2D
:10A65000B4FBF3F185B08046062389B290F835004B
:10A66000FEF772F900214388B4FBF3F48146C8F881
:10A6700040403846FFF7F8F980226B213846FFF753
:10A680001DF8962606F0C0F804460D4606F0BCF804
:10A69000001B61EB0501B0F57A7F71F10001F5D384
:10A6A000013EEFD1032268213846FFF707F89626CE
:10A6B00006F0AAF804460D4606F0A6F8001B61EB6A
:10A6C0000501B0F57A7F71F10001F5D3013EEFD1BC
:10A6D00003226B213846FEF7F1FF06F095F8044699
:10A6E0000D4606F091F8001B61EB05010F2871F192
:10A6F0000001F6D310226A213846FEF7DFFF06F08C
:10A7000083F804460D4606F07FF8001B61EB050157
:10A710000F2871F10001F6D300226C213846FEF7B4
:10A72000CDFF06F071F804460D4606F06DF8001BEB
:10A7300061EB05010F2871F10001F6D399F80520AE
:10A7400019213846FEF7BAFF06F05EF804460D46BA
:10A7500006F05AF8001B61EB05010F2871F10001AA
:10A76000F6D318221B213846FEF7A8FF06F04CF856
:10A7700004460D4606F048F8001B61EB05010F2862
:10A7800071F10001F6D318221C213846FEF796FF1E
:10A7900006F03AF804460D4606F036F8001B61EB69
:10A7A00005010F2871F10001F6D399F804201A2150
:10A7B0003846FEF783FF06F027F805460C4606F0FC
:10A7C00023F88C4208BF8542F9D003213846FFF7B1
:10A7D0004BF9D8F800000623432102AAFFF710FF27
:10A7E00028B3BDF80810BDF80A30BDF80C20C9BA6E
:10A7F00007EE901ADBBAD2BAF8EEE76A07EE102A33
:10A8000007EE903AB8EEC77AF8EEE77AC8ED076A35
:10A81000C8ED087A88ED097AFDEEE77ACDED017A88
:10A820009DF90430013305D005B0BDE8F083D8EDC3
:10A83000087AF1E7D8ED077AFDEEE77ACDED017AF7
:10A840009DF904300133EFD1062006F039F800BF3E
:10A850008C3F080840420F0010B504460068037999
:10A8600082B0022B0CBF4321032106236A46FFF767
:10A87000C7FE68B1BDF80010BDF80220BDF8043075
:10A8800049BA52BA5BBAE1866287238702B010BD2B
:10A89000C4F83600608702B010BD00BF2DE9F04754
:10A8A000164F97F8B93F824689466BB9DAF800002F
:10A8B00097F8BA3F00244A46492187F8B94FFFF775
:10A8C0009FFE0120BDE8F08705F09EFFD7F8C03F4E
:10A8D000C51AC5F5FA55002DE8DD05F095FF4FEADC
:10A8E000E57804460E4605F08FFF001B61EB06017C
:10A8F000A84271EB0801F6D3D8E700BF005F002043
:10A900002DE9F041624C0546D4F8C80FC5F8360071
:10A9100094F8B83FB4F8CC2F6A87012B82B076D078
:10A92000022B0FD0002B69D10122022128466DF0A5
:10A93000CBFB012394F8CE6F84F8B83F304602B0C9
:10A94000BDE8F08194F8B93F05F1360804F6C87700
:10A95000002B6ED169462846FFF7A0FF9DF8063010
:10A96000064600284AD01B0748D4B4F8AC2FBDF8DF
:10A97000003013FB02F3474A93427DDBB3F5000F2F
:10A980006FDA002BB8BFFF331B125B421BB2B4F867
:10A99000AE2FEB86BDF8023013FB02F33D4A934223
:10A9A0006EDBB3F5000F6FDA002BB8BFFF3343F354
:10A9B0000F23B4F8B02F2B87BDF8043013FB02F33C
:10A9C000344A93425ADBB3F5000F5BDA002BB8BF71
:10A9D000FF331B125B421BB2D5F83600C4F8C80F18
:10A9E0006B87B8F80430BB8000220123304684F81E
:10A9F000B82F84F8CE3F02B0BDE8F0810026304683
:10AA000084F8B86F84F8CE6F02B0BDE8F08194F896
:10AA1000B93F94F8CE6FD3B969462846FFF73EFF99
:10AA20009DF8003008B19A071DD1002384F8B83F83
:10AA300084E705F0E9FED4F8C03FC01AB0F5FA5F2C
:10AA400088DA94F8CE6F304602B0BDE8F08105F0A8
:10AA5000DBFED4F8C03FC01AB0F5FA5FFFF66EAF68
:10AA6000DAE70D4B93E70722032128466DF02CFB14
:10AA7000022384F8B83F61E7084B88E7074BABE750
:10AA8000064B96E7044BA7E747F6FF7391E700BF35
:10AA9000005F002001FF7FFF0180FFFF0080FFFFBC
:10AAA00010B5044600680179012984B02AD0022932
:10AAB00002D0002004B010BD836813F0010F02AA79
:10AAC0004FF0060308BF8221FFF744FD0028F0D0B5
:10AAD000BDF9083006EE903ABDF90A3007EE103A9B
:10AAE000BDF90C3007EE903AF8EEE66AB8EEC77A98
:10AAF000F8EEE77AC4ED076A84ED087AC4ED097AC6
:10AB000004B010BD8368417C90F9100003F001038C
:10AB1000019302AB009302220623F9F7C9FCD5E7A3
:10AB200030B5044600680379012B85B014D0022BA0
:10AB30000FD1826802AD12F0010F18BF03212A461F
:10AB400008BF8321FFF706FD18B19DF90930002BDE
:10AB500010DB002005B030BD8368417C90F9100007
:10AB600003F0010302AD0193009502230322F9F7DC
:10AB70009FFCE9E7206807232A461221FFF740FDE2
:10AB80000028E6D09DF90A209DF809309DF90C10A7
:10AB900043EA022313EB430248BF03329DF80B3014
:10ABA000921043EA012307EE902A13EB4302F8EEDA
:10ABB000E77A48BF03329DF90E109DF80D30C4EDC1
:10ABC000047A921007EE902A43EA012313EB430321
:10ABD000F8EEE77A48BF03339B10C4ED057A07EE21
:10ABE000903AF8EEE77AC4ED067AB3E770B50668F6
:10ABF000F46982B00546002C3FD03379012B04F173
:10AC000004022DD0022B26D1B36813F0010F4FF0B0
:10AC10000C03304614BF19468C21FFF79BFCA07033
:10AC2000D8B1B4F9043007EE903AF8EEE77AC5ED02
:10AC3000077AB4F9063007EE903AF8EEE77AC5EDF8
:10AC4000087AB4F9083007EE903AF8EEE77AC5EDE5
:10AC5000097A02B070BD0023A370002002B070BD5D
:10AC6000B368717C96F91000009203F00103019320
:10AC70000C231A46F9F71CFCD1E709211420FDF733
:10AC80008BFDF06104462E68B7E700BF70B506681B
:10AC9000F46982B00546002C3FD03379012B04F1D2
:10ACA00003022DD0022B26D1B36813F0010F3046DA
:10ACB0004FF00D0314BF0C218C21FFF74BFCA0704B
:10ACC000D8B1B4F90A3007EE903AF8EEE77AC5ED5C
:10ACD000077AB4F90C3007EE903AF8EEE77AC5ED52
:10ACE000087AB4F90E3007EE903AF8EEE77AC5ED3F
:10ACF000097A02B070BD0023A370002002B070BDBD
:10AD0000B368717C96F91000009203F0010301937F
:10AD10000C220D23F9F7CCFBD1E709211420FDF714
:10AD20003BFDF06104462E68B7E700BF10B5006830
:10AD30000379012B84B00C461AD0022B02D00020DC
:10AD400004B010BD836813F0010F03AA4FF0030392
:10AD500014BF2221A221FFF7FDFB0028EFD0BDF98F
:10AD60000D3003EB83031B12E633238004B010BDC8
:10AD70008368417C90F9100003F00103019303AB59
:10AD8000009322220323F9F793FBE6E710B504466C
:10AD900000680379012B84B02DD0022B01D0002054
:10ADA00027E0836813F0010F02AA4FF0060314BFD7
:10ADB0001F219F21FFF7CEFB0028F0D0BDF808101F
:10ADC000BDF80A20BDF80C30C9BA07EE901AD2BA05
:10ADD000F8EEE76A07EE902ADBBAB8EEE77A07EEFC
:10ADE000903AF8EEE77AC4ED046A84ED057AC4ED92
:10ADF000067A04B010BD8368417C90F9100003F01E
:10AE00000103019302AB00931F220623F9F750FBC5
:10AE1000D2E700BF10B5044600680379012B84B067
:10AE20002DD0022B01D0002027E0836813F0010F02
:10AE300002AA4FF0060314BF2521A521FFF78AFBC4
:10AE40000028F0D0BDF80810BDF80A20BDF80C307D
:10AE5000C9BA07EE901AD2BAF8EEE76A07EE902A5E
:10AE6000DBBAB8EEE77A07EE903AF8EEE77AC4ED8F
:10AE7000076A84ED087AC4ED097A04B010BD8368CE
:10AE8000417C90F9100003F00103019302AB0093A1
:10AE900025220623F9F70CFBD2E700BF10B50068A6
:10AEA0000379012B84B00C4625D0022B01D0002061
:10AEB0001FE0826812F0010F18BF1D2103AA08BF0E
:10AEC0009D21FFF747FB0028F1D0BDF80C309FED26
:10AED000116ADFED116ADBBA07EE903AB8EEE77A55
:10AEE000C7EE067A77EEA67AFDEEE77A17EE903A8D
:10AEF000238004B010BD8368417C90F9100003F0FA
:10AF00000103019303AB00931D220223F9F7D0FA4A
:10AF1000D9E700BFCFF7534100007A4370B5066808
:10AF2000F46982B00546002C3FD03379012B04F13F
:10AF300004022DD0022B26D1B36813F0010F304646
:10AF40004FF00E0314BF3B21BB21FFF703FBA070A2
:10AF5000D8B1A389DBBA07EE903AF8EEE77AC5EDEF
:10AF6000077AE389DBBA07EE903AF8EEE77AC5EDA7
:10AF7000087A238ADBBA07EE903AF8EEE77AC5ED55
:10AF8000097A02B070BD0023A370002002B070BD2A
:10AF9000B368717C96F91000009203F001030193ED
:10AFA0003B220E23F9F784FAD1E709211420FDF79B
:10AFB000F3FB0446F061B8E700B500680379012BA4
:10AFC00085B011D0022B01D000200AE003AAF6219F
:10AFD000FFF7C0FA0028F7D0BDF80C30094A5BBA79
:10AFE000938205B05DF804FB8368417C90F9100002
:10AFF00003AA03F00103CDE900230223F622F9F7A7
:10B0000057FAE7E7005F002000B500680379012BDD
:10B0100085B01ED0022B01D0002017E0032303AA25
:10B02000F621FFF797FA0028F6D09DF80D309DF82D
:10B030000CC00F499DF80E201B0243EA0C4313433A
:10B04000B1F93420C2F10802D3408B6305B05DF83A
:10B0500004FB8368417C90F9100003AA03F001030C
:10B06000CDE900230323F622F9F722FADBE700BF3C
:10B07000005F002000B500680379012B85B033D054
:10B08000022B0AD01F49D1F8D03FD1F8D42FCA6380
:10B090000020CB6505B05DF804FB062302AAF7216A
:10B0A000FFF758FA0028EDD09DF809309DF808C048
:10B0B0009DF80C209DF80A109DF80BE01B0143EA57
:10B0C0000C3312019DF80DC043EA111342EA0E320F
:10B0D0000C4942EA1C12C1F8D03FC1F8D42FCA6310
:10B0E000CB6505B05DF804FB8368417C90F91000E6
:10B0F00002AA03F00103CDE900230623F722F9F7A2
:10B10000D7F9CFE7005F002000B500680379012B75
:10B1100085B01ED0022B10D09DF80D309DF80C008C
:10B120009DF80E10124A1B0243EA00430B43012014
:10B13000C2F8843005B05DF804FB836813F0010F9A
:10B1400003AA4FF0030314BF00218021FFF702FA86
:10B15000E2E78368417C90F9100003AA03F0010341
:10B16000CDE9002303230022F9F7A2F9D4E700BFB9
:10B17000005F002000B500680379012B85B01ED068
:10B18000022B10D09DF80D309DF80C009DF80E108C
:10B19000124A1B0243EA00430B430120C2F89830D5
:10B1A00005B05DF804FB836813F0010F03AA4FF0AC
:10B1B000030314BF00218021FFF7CCF9E2E7836885
:10B1C000417C90F9100003AA03F00103CDE90023AC
:10B1D00003230022F9F76CF9D4E700BF005F0020D9
:10B1E00010B500680379012B84B029D0022B01D05F
:10B1F000002023E0836813F0010F4FF0030303AA3C
:10B2000014BF19468321FFF7A5F90028F0D09DF857
:10B210000C309DF90C109DF80D209DF80EC01B04FC
:10B22000002943EA0223A8BF00210C4AB8BF4FF00F
:10B230007F4143EA0C030B43C2F8D03004B010BD89
:10B240008268417C90F9100002F0010203AC0323F4
:10B25000CDE900421A46F9F72BF9D6E7005F002046
:10B2600000B500680379012B85B02AD0022B01D0EC
:10B27000002023E0836813F0010F03AA4FF00303BB
:10B2800014BF00218021FFF765F90028F0D09DF858
:10B290000C309DF90C109DF80D209DF80EC01B047C
:10B2A000002943EA0223A8BF00210D4AB8BF4FF08E
:10B2B0007F4143EA0C030B43C2F8CC3005B05DF884
:10B2C00004FB8368417C90F9100003AA03F001039A
:10B2D000CDE9002303230022F9F7EAF8D5E700BF00
:10B2E000005F002010B5044600230068C4F8363023
:10B2F00063870379012B84B022D0022B01D0002078
:10B300001CE0836813F0010F02AA4FF0060314BF7C
:10B3100003218321FFF71EF90028F0D0BDF90A3080
:10B32000BDF80810BDF80C205B4201EB410103EBB6
:10B33000430302EB4202E1862387628704B010BD1B
:10B340008368417C90F9100003F00103019302AB84
:10B35000009303220623F9F7ABF8DDE700B5006898
:10B360000379012B85B00DD0022B07D1012303AA4D
:10B37000FF21FFF7EFF805B05DF804FB002005B0F2
:10B380005DF804FB8268417C90F9100002F0010234
:10B39000019203AA0092FF22F9F78AF805B05DF83E
:10B3A00004FB00BF70B50446224894F9103003EB4B
:10B3B0008303154650F82360A3689A070DD53046DD
:10B3C00070F046FA012300222946304670F0F0F969
:10B3D000A3689B0716D5012070BD636913B11A6875
:10B3E0009B885383144B154A1B6850684FEAC30C63
:10B3F000134BA3FB0C3C4FEA9C1C53681B1A9C4547
:10B40000FBD2DCE70C4B0D491A680D4B4FF4FA7078
:10B4100000FB02F2A3FB0232486892094B681B1A38
:10B420009A42FBD26369002BD5D01A689B8813839C
:10B43000012070BD400D0020AC360020001000E05F
:10B44000D34D621010B50379012B82B08E460DD01A
:10B45000022B02D0002002B010BD8368DB0758BF6A
:10B4600041F0800102B0BDE810409BE714468268BD
:10B47000009402F00102417C90F9100001927246A2
:10B48000F9F716F802B010BD70B505682B79012BDD
:10B4900084B004460E4616D0022B02D0002004B021
:10B4A00070BDAB68E122DB074CBF11466121284625
:10B4B000FCF71EF80028F1D020683246FF2104B0C6
:10B4C000BDE87040BEE7AA68697C95F9100002F0FB
:10B4D00001020DF10F0501920095E1228DF80F2078
:10B4E000F9F71AF8E6E700BF70B505682B79012B6C
:10B4F00084B004460E4617D0022B02D0002004B0C0
:10B5000070BDAB68DB074FF0C3024CBFE121612186
:10B510002846FBF7EDFF0028F0D020683246FF21D7
:10B5200004B0BDE870408DE7AA6895F91000697C09
:10B5300002F0010201920DF10F020092C3228DF878
:10B540000F20E122F8F7E8FFE5E700BF70B50568D6
:10B550002B79012B84B004460E461CD0022B02D05E
:10B56000002004B070BDAB68DB074FF0F0024CBFA9
:10B57000E12161212846FBF7BBFF0028F0D02246DD
:10B58000FF2152F8040BFFF75DFF0028E8D0237974
:10B59000337004B070BDAA6895F91000697C02F0A0
:10B5A000010201920DF10F020092F0228DF80F209E
:10B5B000E122F8F7B1FFE0E7F0B5046883B00021BD
:10B5C00007462046FEF750FA15227E212046FEF758
:10B5D00075F8642605F018F904460D4605F014F9CF
:10B5E000001B61EB0501B0F57A7F71F10001F5D325
:10B5F000013EEFD1386811227E21FEF75FF8052663
:10B6000005F002F904460D4605F0FEF8001B61EB5B
:10B610000501B0F57A7F71F10001F5D3013EEFD15C
:10B6200038680DF107020321FFF70CFF9DF8073082
:10B6300003F03C03142B40F09B800C22402138681F
:10B64000FEF73CF805F0E0F804460D4605F0DCF89E
:10B65000001B61EB0501B0F57A7F71F10001F5D3B4
:10B66000BB6B454C454AB4FBF3F197F83500032317
:10B6700089B2FDF769F9034642215A88B4FBF2F416
:10B680003C641A793868FEF719F805F0BDF80446ED
:10B690000D4605F0B9F8001B61EB0501B0F57A7FA6
:10B6A00071F10001F5D3082241213868FEF706F850
:10B6B00005F0AAF804460D4605F0A6F8001B61EB5C
:10B6C0000501B0F57A7F71F10001F5D30022432125
:10B6D0003868FDF7F3FF05F097F804460D4605F0CE
:10B6E00093F8001B61EB0501B0F57A7F71F1000161
:10B6F000F5D3102251213868FDF7E0FF05F084F8FA
:10B7000004460D4605F080F8001B61EB0501B0F51D
:10B710007A7F71F10001F5D30A2253213868FDF7D1
:10B72000CDFF05F071F804460D4605F06DF8001BDD
:10B7300061EB0501B0F57A7F71F10001F5D380224C
:10B7400056213868FDF7BAFF05F05EF804460D464D
:10B7500005F05AF8001B61EB0501B0F57A7F71F135
:10B760000001F5D338680321FEF77EF903B0F0BD80
:10B77000062005F0A5F800BF40420F00B03F0808C2
:10B780002DE9F043836B0768A04AA14CB4FBF3F1A9
:10B7900083B08046052389B290F83500FDF7D4F8D0
:10B7A00000214388B4FBF3F48146C8F84040384692
:10B7B000FEF75AF9002276213846FDF77FFF0F2267
:10B7C0004E213846FDF77AFF0F2605F01DF8044696
:10B7D0000D4605F019F8001B61EB0501B0F57A7F05
:10B7E00071F10001F5D3013EEFD199F805204F2109
:10B7F00002F00F023846FDF761FF0F2605F004F84E
:10B8000004460D4605F000F8001B61EB0501B0F59C
:10B810007A7F71F10001F5D3013EEFD199F805204F
:10B82000502102F00F023846FDF748FF0F2604F0C2
:10B83000EBFF04460D4604F0E7FF001B61EB05013A
:10B84000B0F57A7F71F10001F5D3013EEFD1FF220F
:10B8500052213846FDF732FF0F2604F0D5FF04468B
:10B860000D4604F0D1FF001B61EB0501B0F57A7FB6
:10B8700071F10001F5D3013EEFD198F83510072999
:10B8800041D0644D95F8F00BFDF7B4F80446012261
:10B8900076213846FDF712FFA2780C213846FDF7D5
:10B8A0000DFF22790D213846FDF708FFA279A38804
:10B8B000120142EA1322D2B20E213846FDF7FEFEF3
:10B8C0004FF4807195F8F00BFDF794F804460222CE
:10B8D00076213846FDF7F2FEA2785200032102F0ED
:10B8E000FE023846FDF7EAFE227904213846FDF7CC
:10B8F000E5FEA279A388120142EA13220521D2B201
:10B900003846FDF7DBFE002276213846FDF7D6FEED
:10B91000032214213846FDF7D1FE0F2604F074FFF0
:10B9200004460D4604F070FF001B61EB0501B0F505
:10B930007A7F71F10001F5D3013EEFD132466321E8
:10B940003846FDF7BBFE642604F05EFF04460D4654
:10B9500004F05AFF001B61EB0501B0F57A7F71F12D
:10B960000001F5D3013EEFD1082265213846FDF7ED
:10B97000A5FE64210DF107023846FFF763FD9DF82F
:10B98000072022F0100242F06002642138468DF850
:10B990000720FDF793FE0F2604F036FF04460D4600
:10B9A00004F032FF001B61EB0501B0F57A7F71F105
:10B9B0000001F5D3013EEFD10DF106024D213846CD
:10B9C000FFF740FD9DF8062002F03F0242F04002E2
:10B9D0004D2138468DF80620FDF770FE0F2604F045
:10B9E00013FF04460D4604F00FFF001B61EB050139
:10B9F000B0F57A7F71F10001F5D3013EEFD103215B
:10BA00003846FEF731F803B0BDE8F083C43F0808BC
:10BA100040420F00005F0020F0B583B015460DF1E5
:10BA200007021C4606460F46FFF70CFD9DF807204F
:10BA300005EA0203A34201D103B0F0BD22EA0502E8
:10BA400022433946304603B0BDE8F040FDF736BE2C
:10BA500010B582B004466A4600680821FFF7F2FC80
:10BA60009DF80030DB0602D4002002B010BD206833
:10BA700006236A460021FEF7C3FD0028F4D09DF896
:10BA800001309DF800109DF802209FED4A6A1B02CC
:10BA900003EB01439DF804101C029DF803401A4477
:10BAA0004FEA01219DF8053001EB044148BF02F146
:10BAB0007F420B4407EE902A090248BF03F17F43FF
:10BAC000B8EEE77A07EE903AF8EEE77AC7EE066A44
:10BAD000394BB3F96C20B3F9721093F8D84F112C8D
:10BAE000C7EE863A07EE102A93ED1A6AB3F96E2074
:10BAF000D3ED197AF8EEC65A06EE102AB3F9702083
:10BB000005EE102AB3F9742004EE901A04EE102A00
:10BB1000B8EEC77AF8EEE77AB8EEC66AB8EEC55A5C
:10BB2000F8EEE44AB3F97610B3F97820B8EEC44AD7
:10BB300027EE237A26EEA32A23D0A6EE845AA6EE79
:10BB4000A46AE5EE265AE5EEA67A77EE877AE6EE67
:10BB5000027AB3F9622007EE102AB3F96020C3ED30
:10BB60001F7A06EE902AB8EEC77AF8EEE66A27EE5C
:10BB7000237AB6EE006AA6EE867A83ED207A02B0CA
:10BB800010BD03EE102AF8EEC32A03EE101AA6EE3B
:10BB9000A24AB8EEC33AA4EE265AE6EE834AE5EE90
:10BBA000265AA4EEA66AE5EEA67A77EE877AE6EE46
:10BBB000027ACEE700007848005F0020F0B5044626
:10BBC00083B00D461746061D20680379012B1AD055
:10BBD000022B02D0002003B0F0BD8368DB073246A1
:10BBE0004FF0FF015CBF3246FF21FFF7DBFB00286F
:10BBF000F0D015B12379DB07E6D4002FEBD0237901
:10BC00003B7003B0F0BD8268417C90F9100002F0F7
:10BC10000102CDE90062FF22F8F74AFCE7E700BF26
:10BC200030B50446051D20680379012B83B017D079
:10BC3000022B02D0002003B030BD8368DB072A4608
:10BC40004FF0FF015CBF2A46FF21FFF7ABFB002846
:10BC5000F0D02379DB07EED520680379012BE7D1FB
:10BC60008268417C90F9100002F00102CDE9005297
:10BC7000FF22F8F71DFCEAE730B50246044652F809
:10BC8000040B0379012B83B00ED0022B01D00020CE
:10BC900008E0FF21FFF786FB0028F8D02079C04399
:10BCA00000F0010003B030BD8568417C90F91000C0
:10BCB000009205F001050195FF22F8F7F9FBEBE78B
:10BCC00030B5B42283B00446FF210068FDF7F6FCCE
:10BCD00010B9002003B030BD20680379012B04F1B6
:10BCE000040514D0022BF4D18368DB072A464FF0F9
:10BCF000FF015CBF2A46FF21FFF754FB0028E8D074
:10BD00002379DB07E6D520680379012BEAD1826825
:10BD1000417C90F9100002F00102CDE90052FF22AF
:10BD2000F8F7C6FBEAE700BF30B50A4683B0044621
:10BD3000A5210068FDF7C2FC10B9002003B030BD9A
:10BD400020680379012B04F1040514D0022BF4D1EF
:10BD50008368DB072A464FF0FF015CBF2A46FF21BC
:10BD6000FFF720FB0028E8D02379DB07E6D5206821
:10BD70000379012BEAD18268417C90F9100002F02E
:10BD80000102CDE90052FF22F8F792FBEAE700BF7B
:10BD900070B582B0CDE900230446FFF791FF10B9DA
:10BDA000002002B070BD20685522A521FDF786FC59
:10BDB0000028F5D0251D20682A46FF21FFF742FB09
:10BDC0000028EDD02379DB07F5D40DF1FF350DF117
:10BDD000070615F8011F2046FFF7A6FF0028DFD051
:10BDE000B542F6D1DDE700BF002A35D0F0B50446F4
:10BDF00083B00E468F18051D16F8012B2068A5216B
:10BE0000FDF75CFC90B9002003B0F0BD8268417C76
:10BE100090F9100002F00102CDE90052FF22F8F77C
:10BE200047FB0028EFD02379DB0710D52068037982
:10BE3000012BEBD0022BE6D18368DB072A464FF0BB
:10BE4000FF015CBF2A46FF21FFF7ACFAE9E7B742E2
:10BE5000D2D1012003B0F0BD0120704770B5962209
:10BE600082B004460E460068FF21FDF727FC10B99A
:10BE7000002002B070BD251D20680379012B1FD062
:10BE8000022BF5D18368DB072A464FF0FF015CBF28
:10BE90002A46FF21FFF786FA0028E9D02379DB073D
:10BEA000EAD4E12220681146FDF708FC0028DFD023
:10BEB00020683246FF2102B0BDE87040FFF7C2BAE9
:10BEC0008268417C90F9100002F00102CDE9005235
:10BED000FF22F8F7EDFADFE7002A43D0F0B5044679
:10BEE00083B00E468F18051D20689622FF21FDF7AE
:10BEF000E5FB90B9002003B0F0BD8268417C90F969
:10BF0000100002F00102CDE90052FF22F8F7D0FA4A
:10BF10000028EFD02379DB0710D520680379012BA7
:10BF2000EBD0022BE6D18368DB072A464FF0FF01F6
:10BF30005CBF2A46FF21FFF735FAE9E7E1222068D6
:10BF40001146FDF7BBFB0028D4D020683246FF2104
:10BF5000FFF778FA0028CDD00136B742C4D10120CE
:10BF600003B0F0BD0120704770B505460B4604468E
:10BF7000164655F8040B82B087211A46FDF79EFB42
:10BF800020680379012B1AD0022B02D0002002B0C6
:10BF900070BD8368DB072A464FF0FF015CBF2A466D
:10BFA000FF21FFF7FFF90028F0D02379DA07E7D463
:10BFB000002EECD0C3F34013337002B070BD826822
:10BFC000417C90F9100002F00102CDE90052FF22FD
:10BFD000F8F76EFAE7E700BF70B5782182B0044643
:10BFE000164600680022FDF769FB10B9002002B078
:10BFF00070BD251D20680379012B14D0022BF5D1CB
:10C000008368DB072A464FF0FF015CBF2A46FF2109
:10C01000FFF7C8F90028E9D02379DA07EAD45B09E9
:10C02000337002B070BD8268417C90F9100002F05C
:10C030000102CDE90052FF22F8F73AFAEAE700BF21
:10C0400030B5CC2283B00446A5210068FDF736FB4D
:10C0500010B9002003B030BD20680379012B04F132
:10C06000040514D0022BF4D18368DB072A464FF075
:10C07000FF015CBF2A46FF21FFF794F90028E8D0B2
:10C080002379DB07E6D520680379012BEAD18268A2
:10C09000417C90F9100002F00102CDE90052FF222C
:10C0A000F8F706FAEAE700BF30B5B42283B00446D9
:10C0B000FF210068FDF702FB10B9002003B030BD7E
:10C0C000251D20680379012B22D0022BF5D183682E
:10C0D000DB072A464FF0FF015CBF2A46FF21FFF72E
:10C0E00061F90028E9D02379DA07EAD4CC21204687
:10C0F000FFF71AFE0028E0D002E02379DB07DDD548
:10C1000020682A46FF21FFF79DF90028F5D1D4E7E2
:10C110008268417C90F9100002F00102CDE90052E2
:10C12000FF22F8F7C5F9DCE72DE9F04F8BB0CDE938
:10C1300007230446002004908A460390251D049B93
:10C14000079A2046DE0002EBC30BFFF7B9FD20B9CA
:10C1500035E0237913F0010207D020682A46FF2139
:10C16000FFF770F90028F4D129E005929A070990A9
:10C1700040F1D880F0212046FFF7D6FDF8B1079BAB
:10C18000DDF81480083E3344012606933746BAF1A1
:10C19000000F54D0082F52D807F1FF394AFA09F995
:10C1A00009F0010920684FEAC9127821FDF786FAE3
:10C1B00028B120680379012B50D0022B06D0002033
:10C1C000089B049A1A700BB0BDE8F08F8368DB07F8
:10C1D0002A464FF0FF015CBF2A46FF21FFF7E2F835
:10C1E0000028ECD0237913F00102E2D1C3F3801CC4
:10C1F000D9099B0646D5BCF1000F60D1BAF1000FFA
:10C200005AD0082F58D8894540F08880B9F1000FDE
:10C2100048D01BF8083033430BF80830760001375C
:10C2200016F0FF06FFB2B2D108F101085FFA88F8F4
:10C23000B8F1080F43D00126BAF1000FAAD1049B30
:10C24000C3B1039BBB4215D9069B13F808301E42AD
:10C2500014BF4FF001094FF00009A3E78268417C49
:10C2600090F9100002F00102CDE90052FF22F8F728
:10C270001FF9B5E7039BA3EB0709B9FA89F94FEA60
:10C2800059198FE7BAF1000F13D0082F11D889453B
:10C2900096D1B9F1000FBCD1059BBCF1000F08BFCE
:10C2A0003B4605931BF8083023EA06030BF80830D9
:10C2B000B4E70029ADD1EFE70029AAD1F2E7402F7A
:10C2C00006D8089B049A1B7893423FF638AF77E76D
:10C2D0009BF807700BF1FF360BF1060B16F801CF38
:10C2E000082182EA0C0343F30003013923F07303AE
:10C2F00083EA520211F0FF01D2B24FEA5C0CF0D196
:10C30000B345EBD19742DCD1049B0133DBB20493FC
:10C31000059B002B3FF454AF0393D2E7DDF8248054
:10C3200040464DE7804640464AE700BF10B5044608
:10C3300086B0006800238DF80F300379012B31D0CF
:10C34000022B02D0002006B010BD8368D9070DF182
:10C350000F024CBF2721A721FFF724F80028F1D0B6
:10C360009DF80F301B07EDD52068062304AA28216D
:10C37000FEF746F928B3BDF91030BDF91220002BA5
:10C38000B8BF03339B10E386BDF91430002AB8BF51
:10C390000332002BB8BF033392109B1022876387B0
:10C3A00006B010BD826890F910C0417C02F0010215
:10C3B00001920DF10F02009260462722F8F778F8FB
:10C3C000CCE7C4F8360060870020BCE730B50446EF
:10C3D0004FF0000C0068C4F836C0A4F83AC00379E6
:10C3E000012B87B02AD0022B02D0002007B030BD2D
:10C3F0008368D9070DF10F024CBF61468021FEF71B
:10C40000D1FF0028F1D09DF80F301B07EDD5206833
:10C41000062304AA0121FEF7F3F80028E5D0BDF8B1
:10C420001430BDF81010BDF812205BBA49BA52BAE8
:10C430005B42E1862287638707B030BD8568417C17
:10C4400090F9100005F0010501950DF10F05624608
:10C450000095F8F72DF8D4E710B5044600230068DE
:10C46000C4F8363063870379012B86B023D0022BC2
:10C4700002D0002006B010BD8368D9070DF10F026D
:10C480004CBF06218621FEF78DFF0028F1D09DF8D4
:10C490000F305B07EDD52068062304AA0021FEF7C4
:10C4A000AFF80028E5D0049ABDF81430C4F836205F
:10C4B000638706B010BD826890F910C0417C02F01D
:10C4C000010201920DF10F02009260460622F7F779
:10C4D000EFFFDAE710B50368DA6B82B0044612B1F9
:10C4E000904740B123685B6B1BB1214601A8984778
:10C4F00018B9FF23E38202B010BDBDF80630013B3E
:10C500009BB2F7E7F0B5044683B018460D461646D1
:10C510001F466FF02DFC2844D4F800C0A073E673CA
:10C52000204600240094DCF814403B46324629465D
:10C53000A04703B0F0BD00BF38B58B68016004466A
:10C540000D46984700230B4A226123752B6B13B1CC
:10C55000204698472075084B93F8DC3F1BB1237D9C
:10C5600023F0010323750023E3822046BDE8384011
:10C57000B0E700BF0001FF00005F002010B5154BC1
:10C58000D3F8E04F84B084B12379012B10D0022B73
:10C590000BD1A16811F00101024618BF802120468D
:10C5A00004B0BDE81040FAF7A3BF002004B010BDEE
:10C5B000A268617C8DF80F0002F0010294F910006E
:10C5C0000DF10F04CDE900428022F7F7A5FF04B07A
:10C5D00010BD00BF005F0020F0B5294BD3F8E05F2D
:10C5E00085B09DB1B02280212846FDF767F8402232
:10C5F00080212846FDF762F8002280212846FDF7B9
:10C600005DF8102280212846FDF758F84FF4806429
:10C610002DB9013CA4B2002CFBD105B0F0BD002720
:10C620000DF10F062B79012B08D0022B04F1FF32FC
:10C6300017D094B2002CF0D0012BF6D1AA6895F94E
:10C640001000697C8DF80F7002F00102013CCDE909
:10C650000062A4B24022F7F75FFF002CE2D105B0E0
:10C66000F0BDAA68013C12F0010218BF002240216F
:10C670002846A4B2FAF73CFF002CD3D105B0F0BD98
:10C68000005F00200B4B10B5D3F8E04F8CB1503851
:10C69000C2B280212046FDF711F8002280212046F9
:10C6A000FDF70CF820461022BDE810408021FDF770
:10C6B00005B810BD005F0020F0B5264B264CD3F81E
:10C6C000E05F203800EB8000661D85B0044406441E
:10C6D00025B90134A642FCD105B0F0BD0DF10F071C
:10C6E0002B792278012B1BD0022B0AD00134A642D1
:10C6F000F7D100224021284605B0BDE8F040FCF704
:10C70000DDBFAB68DB074FF04001284619D5013487
:10C71000FAF7EEFEA642E3D1002DEAD105B0F0BD56
:10C720008DF80F20AA6895F91000697C02F00102CB
:10C73000CDE9007201344022F7F7EEFEB442CFD1CA
:10C74000D7E70134FAF7D4FEB442C9D1002DE5D0C1
:10C75000CFE700BF005F0020E43F0808F0B5754B4D
:10C76000D3F8E05F85B0002D00F09680D4228021C0
:10C770002846FCF7A3FF802211462846FCF79EFFBF
:10C78000A82280212846FCF799FF3F2280212846D5
:10C79000FCF794FFD32280212846FCF78FFF00226C
:10C7A00080212846FCF78AFF402280212846FCF79A
:10C7B00085FF8D2280212846FCF780FF14228021EE
:10C7C0002846FCF77BFFA12280212846FCF776FF54
:10C7D000C82280212846FCF771FFDA2280212846F2
:10C7E000FCF76CFF122280212846FCF767FF8122AC
:10C7F00080212846FCF762FFCF2280212846FCF7E3
:10C800005DFFD92280212846FCF758FFF1228021C4
:10C810002846FCF753FFDB2280212846FCF74EFF19
:10C82000402280212846FCF749FFA4228021284687
:10C83000FCF744FFA62280212846FCF73FFFAF22E9
:10C8400080212846FCF73AFFA62280212846FCF7E3
:10C8500035FFAE2280212846FCF730FF20228021C0
:10C860002846FCF72BFF002280212846FCF726FFF4
:10C87000B02280212846FCF721FF40228021284653
:10C88000FCF71CFF002280212846FCF717FF10222E
:10C8900080212846FCF712FF4FF4806435B9013C33
:10C8A000A4B2002CFBD1012005B0F0BD00270DF192
:10C8B0000F062B79012B2AD0022B04F1FF3214D062
:10C8C00094B2002CF6D1812280212846FCF7F6FE96
:10C8D000C82280212846FCF7F1FEAF22802128469D
:10C8E000FCF7ECFE012005B0F0BDAA68013C12F097
:10C8F000010218BF002240212846A4B2FAF7F8FD31
:10C90000002CD6D1002DDED1012005B0F0BDAA68E3
:10C9100095F91000697C8DF80F7002F00102013C5E
:10C92000CDE90062A4B24022F7F7F6FD002CC0D199
:10C93000C9E700BF005F0020FBF76AB8FBF768B8E3
:10C94000FBF766B8FBF764B8FBF762B8FBF760B8B3
:10C9500001207047034620B1026812B1D26902B1CA
:10C96000104793ED017A084BB8EEC77AD3ED016A10
:10C97000F6EE007AE7EE267AFDEEE77A17EE900AF9
:10C9800000F30B00704700BFE46E0020034620B1A7
:10C99000026812B1126A02B1104793ED027A084B95
:10C9A000B8EEC77AD3ED026AF6EE007AE7EE267AA1
:10C9B000FDEEE77A17EE900A00F30B00704700BF18
:10C9C000E46E0020034628B102681AB1516A09B129
:10C9D0009369184793ED037A074BB8EEC77AD3ED06
:10C9E000036AF6EE007AE7EE267AFDEEE77A17EEB6
:10C9F000900A00F30B007047E46E002010B5044667
:10CA000030B1036823B1DB6813B1BDE810401847AB
:10CA100003F0FAFED4E904239042994134BF012087
:10CA2000002010BDF8B170B506680F4B06F13F420B
:10CA300002F57E0203EB92230C4682B0054693F882
:10CA40002C056BF0F1F9C4F34112C4F30013A9886B
:10CA50003046CDE90032C4F3810304F003026EF0E6
:10CA600067FC02B070BD70475C3D0808B0B3F0B51C
:10CA700007681B4B144607F13F4202F57E0203EBA9
:10CA80009223054683B093F82C050E466BF0CCF943
:10CA9000A988B1FA81F3C3F11F03C3F3CC0207EBFA
:10CAA000820203F00703156A4FF00F0C9B009C40B5
:10CAB0000CFA03F325EA03031362136A1C4314629E
:10CAC000C6F300137209CDE900323846C6F381037C
:10CAD00006F003026EF02CFC03B0F0BD704700BFFF
:10CAE0005C3D080810B50409013C032C19D80F4A15
:10CAF00000F00F0332F8140040FA03F212F00102C2
:10CB000011D0012202FA03F3013B184076F02EFF08
:10CB1000074B084A1B5D184400EB400002EB800005
:10CB200010BD002010BD104610BD00BF503D0808CC
:10CB30004C3D08082C2B00202DE9F04F54220446D0
:10CB40000021C34891B075F055FFC24A611EE01C38
:10CB5000144611F8013F5D1E052D88BF0023814258
:10CB600044F8043BF5D102F11003114651F8040BCF
:10CB7000012800F058819942F8D1114651F8040B70
:10CB8000022800F046819942F8D1114651F8040B71
:10CB9000032800F052819942F8D152F8041B04296D
:10CBA00000F02D819A42F8D10520FAF7FBF8062013
:10CBB000DFF89C92DFF8BC82FAF7F4F84C464FF0AD
:10CBC0001A0A002608F2345B277B57B3384694F9DB
:10CBD0000D50FFF787FF28B105238371002380F8EC
:10CBE00007A003721321FFF71DFF00231BF833106A
:10CBF000B9422FD00133102BF8D10021964B21617F
:10CC000005EB450503EBC5050122D5F8D43923759D
:10CC10001344C5F8D4390723A375627585F8D02964
:10CC200016440AF1010A5FFA8AFABAF1200F04F1F8
:10CC30000C04C9D15EB1894D894F00262B7C73B994
:10CC40000136032E05F1180507F58C77F6D111B0E2
:10CC5000BDE8F08F08EBC303D3F83815CEE7687949
:10CC60006BF0E2F828796BF0DFF8D5F808A05046B1
:10CC7000F6F7B0FDD5F814802C680397142303FB56
:10CC800008F305930023CDE90C33CDE90E3304936B
:10CC90000693EB68019304F14C034FF48062029316
:10CCA0004FF40063CDE907234FF400514FF4807334
:10CCB000CDE9091350464FF4003301A90B936BF0F3
:10CCC00087F8DAF800206749674B42F00102CAF89A
:10CCD00000204A68134043F440334B606368B8F166
:10CCE000010F23F04073D4BF0022012223F480738C
:10CCF00043EA02236360A2685C4B134043F00203E3
:10CD0000A360E36A08F1FF385FFA88F823F4700340
:10CD100043EA0853E36209F148014B4601204FFA08
:10CD200086FC02E00C338B4231D05A7D002AF9D0C8
:10CD300093F90D206245F5D11A7C93F816A0092AC3
:10CD400036D802EB420BD4F810800AFA0BFE4FF0F3
:10CD5000070A0AFA0BFA28EA0A084EEA080EC4F88B
:10CD600010E0062837D800F1FF3ED4F834800EEBEF
:10CD70008E0E4FF01F0A02FA0EF20AFA0EFE28EA91
:10CD80000E0E42EA0E0262630130C0B2CAE7A36827
:10CD900043F40073A360A36843F48073A360A368A3
:10CDA00043F00103A360A36843F08043A36047E717
:10CDB000A2F10A0ED4F80C800EEB4E0E4FF0070BCA
:10CDC0000AFA0EFA0BFA0EFE28EA0E0E4AEA0E0EC8
:10CDD000C4F80CE0C5E70C284ED8A0F1070ED4F833
:10CDE00030800EEB8E0E4FF01F0A02FA0EF20AFA96
:10CDF0000EFE28EA0E0E42EA0E022263C4E71C4B26
:10CE000093F8602C3021013283F83C1C83F8602CAD
:10CE1000CAE6174991F8600C3524013081F8244C9A
:10CE200081F8600CB1E6124991F8600C34240130AD
:10CE300081F8184C81F8600C9FE60D4991F8600C60
:10CE40002024013081F8304C81F8600CA5E600BF49
:10CE50000C6B0020045F0020400D00200017002014
:10CE6000646B002000230140E030FCFFFDF7FFC0B1
:10CE7000005F00205C3D0808A0F10D0ED4F82C8066
:10CE80000EEB8E0E4FF01F0A02FA0EF20AFA0EFE99
:10CE900028EA0E0E42EA0E02E26275E710B5036858
:10CEA0001A79022A044603D000232371236010BD9F
:10CEB000987AFFF717FE0028F6D040F61A61002294
:10CEC000C18002722021FFF7ADFD00232371236092
:10CED00010BD00BF2DE9F04FB04EB14CA64285B059
:10CEE00056D21D4602E00C36A64251D273798B42CF
:10CEF000F9D13379834201D00028F4D1F3799342F8
:10CF0000F1D13468002C43D000236360A360E36058
:10CF100023616361A361E36126603379237196F82D
:10CF200006B0C4F808B0317AE160012B32D0022B90
:10CF30002ED1F07AFFF7D6FD96F90970A061B07A8C
:10CF40002774FFF7CFFD06466061F0B1DFF870820D
:10CF500007EB8701BB0058F82190019308EB810192
:10CF6000B9F1000F11D0887CE8B10E220023F271D4
:10CF70003372B57109213046FFF754FD3368B2882A
:10CF80001A83204605B0BDE8F08F2046FFF786FFE4
:10CF90000024F6E7F07AFFF7A5FD727AB37A63749E
:10CFA000A0612274EDE791F808A050466AF03CFFBA
:10CFB0004FEA5A1001210AF01F0A023801FA0AF159
:10CFC000032808D8DFE800F0AA9EA402754B586930
:10CFD00020EA01015961BB00D91908EB810107F171
:10CFE000010A4879FFF77EFD5FFA8AFA014620B10F
:10CFF00080F808A040F60A30C880BB00D81908EBBA
:10D0000080000291C079FFF76DFD029901900346FF
:10D0100020B180F808A040F60A50D880BB00D8198B
:10D0200008EB800002918079FFF75CFD02990346CE
:10D0300020B180F808A040F60A40D880BA00D01984
:10D0400008EB80001BF0040290F809A0CDE9022350
:10D050000846524668D04A21FFF708FD019852461B
:10D060002A21FFF703FD039B524618460A21FFF7CA
:10D07000FDFCBB00DA1908EB820292F804B0BBF1A8
:10D08000000F61D1484A914571D0484A914563D01B
:10D09000474A914500F0A180464A914500F09280B0
:10D0A000454A91456ED0454A914500F0A180029BCA
:10D0B000B9F80010002B01F441510CBF03220022EB
:10D0C0000A4342F44572A9F80020B9F81C2022F462
:10D0D00000621204120CA9F81C200722A9F81020E3
:10D0E000B9F8002092B242F04002A9F80020BBF14A
:10D0F000000F20D1BB003B4408EB8308012388F8D4
:10D10000123032E7274B186A20EA0101196262E700
:10D11000244B186920EA010119615CE7214B586A28
:10D1200020EA0101596256E70A21FFF79FFC0198A6
:10D1300052460A2195E75846FFF7D4FC0028D9D07B
:10D14000026883881383D5E75846FFF7CBFC524625
:10D150000921FFF78BFC95E702F50032116A41F4D3
:10D1600080411162116A21F4804111629FE702F54A
:10D170008432516A41F480515162516A21F48051E4
:10D18000516294E702F56842516A41F4801151629C
:10D19000516A21F48011516289E700BF586C090877
:10D1A000146E090800380240003001400038004089
:10D1B000003C004000340140005001400054014058
:10D1C000400D002002F58232516A41F40051516253
:10D1D000516A21F40051516269E702F5FE32116A89
:10D1E00041F400411162116A21F4004111625EE7CD
:10D1F00002F56442516A41F400115162516A21F40E
:10D200000011516253E700BF074B53F8203021B1A2
:10D210004BB11A689B8853837047002BFCD01A6867
:10D220009B88138370477047403D08081E4AF8B535
:10D23000D2F82C3173B15D6892F830216C790646D2
:10D240004AB1032C2CD8DFE804F0222528022B68F1
:10D2500040331E60F8BDDF681449D7F808C031F8C4
:10D2600014E0DCF80010286821F00101CCF800106F
:10D27000818989B221EA0E0181811A7403889BB2E7
:10D2800043F0010303803A77FAF7B8FCD9E72B683B
:10D290003433DEE72B683833DBE72B683C33D8E7E1
:10D2A00000231B60FFDE00BF005F0020503C080829
:10D2B00010B5224CD4F82C3183B194F830216AB1E6
:10D2C00094F8F42F032A0AD0022A10D0002384F8FD
:10D2D0003031FAF7BDFB08B984F8F50F10BD5A6874
:10D2E0005379032B27D8DFE803F023201D185A6851
:10D2F0005379032B1FD8DFE803F00D0A07021368E8
:10D30000403300221A6010BD13683C33F9E71368FC
:10D310003833F6E713683433F3E713684033642295
:10D320001A6010BD13683C33F9E713683833F6E729
:10D3300013683433F3E700231B60FFDE005F002037
:10D340002DE9F04FC44BC54993F8F87F93F8F98F56
:10D3500093F8FAEF83B003F6FC704FF0000C00F581
:10D36000007ACDF804C001228378C578C3F1FF03A9
:10D370009BB22C46002B00F03B81B0F80090B84ED9
:10D38000C3F1FF03A6FB09B605FB03F376091B12E5
:10D39000052E00F26E81DFE816F01701FB00E300B6
:10D3A000C600AB000600AE4EA6FB09E46409C4EB60
:10D3B0000414A9EB8404A4B2EF1AC4F13C0407FBE3
:10D3C00004F4A6FB04645FFA83F808EB54145FFAD4
:10D3D00084FE2F461C462B460125764601951D02EC
:10D3E00045EA04451724354383460CEB0406331BFA
:10D3F00002FA04F99BB219EA050F03F12A030CBFE4
:10D4000001200220013C41F82300631CEFD1584663
:10D4100004300CF1180C50451FFA8CFCA4D1914B30
:10D420004FF44062A3F804218022A3F80621019B57
:10D4300033B1894B83F8FAEF83F8F98F83F8F87FDB
:10D44000854A92F8F53F002B4FD0D2F82C31002BB3
:10D450004BD0EFF31181102282F31288D8685D68F7
:10D460008468226822F0010222602C687E4A6D796D
:10D4700032F81550A28992B222EA0502A28102690D
:10D4800044681F2A40F2BC80203A202000FA02F2B1
:10D49000E260CAB282F31188DA686F489268D0F805
:10D4A0002C0140F62B415160116801242143116089
:10D4B0001C7403681A7DA24204BF02221A7593F8F5
:10D4C0002C100CBF4FF400720022012900F0B18033
:10D4D00093F84410012900F0988093F85C1001291A
:10D4E00000F0B480002A40F0C18003B0BDE8F08FA6
:10D4F000DFF86CE1EF1A2E46AEFB09546409C4EB69
:10D500000414A9EB8404A4B204FB07F7AEFB07E7FD
:10D510005FFA83F808EB5717FFB201251C46B646A1
:10D520003B4601955BE74E4FA5EB030E2E46A7FB4E
:10D5300009546409C4EB0414A9EB84081FFA88F8A1
:10D54000C8F13C080EFB08F8A7FB0878DFB207EB30
:10D5500058185FFA88F801254446B64601953EE71B
:10D560003F4FEE1AA846A7FB09E56D09C5EB051567
:10D57000A9EB8505ADB205FB06FEA7FB0E7EDFB26B
:10D5800007EB5E1E5FFA8EFE01257646019526E7C3
:10D59000334EA5EB030EA846A6FB09756D09C5EB36
:10D5A0000515A9EB8507BFB2C7F13C070EFB07F7CE
:10D5B000A6FB07675FFA83FE0EEB5717FFB21E4606
:10D5C000012301933B460AE7A5EB0308244C09FB22
:10D5D00008F8A4FB08485FFA83FE0EEB58185FFAC0
:10D5E00088F81E462F462B46012544460195F6E64F
:10D5F000AE462E462B46A8462F4601250195EEE65F
:10D60000202000FA02F2A26043E7022183F84410CE
:10D6100093F85C10012942F4006217D043681B683C
:10D6200000215962998989B20A439A8103B0BDE801
:10D63000F08F022183F82C1093F84410012942F452
:10D640008062E2D093F85C100129E7D1022183F8CF
:10D650005C1042F48052E1E7005F00204475002036
:10D6600089888888F86F0020503C08084FF40072C1
:10D67000D4E744463B467646B1E600BF70B500218C
:10D680002120F5F79DFBC36813F080730ED12E4C5B
:10D69000224602E001330C2B2ED0D168C90102F1E1
:10D6A0001402F7D5142202FB034400E0044620468E
:10D6B000F5F736FB254E0546C6F82C01E0B120797A
:10D6C000FFF710FA224BC3F8080120B140F21523EE
:10D6D000C38000230372227A4A21FFF7C7F996F824
:10D6E000F44F022C28D0032C07D1FAF787FA2846EA
:10D6F000F5F7F4FC6423036070BDFAF7A9F910B9DB
:10D7000086F8F50F70BD134843F2AC02002175F0A6
:10D7100071F9012C03D1104BFF22C3F8A82096F811
:10D720003031012286F8F52F002BE5D12B7C002B20
:10D73000E2D1BDE8704003E6FAF760FA2846F5F753
:10D74000CDFC0023036070BD040A0020005F0020B0
:10D75000F86F00204475002044A500202DE9F04F0B
:10D76000A04FA7B000210A260C4607F586754FF09A
:10D77000050B01968BE0BAF1000F19D143F040037D
:10D78000BEF18C0F87F8103500F2E48004F1010C33
:10D7900098340DEB040A0CF198040DEB040C74465C
:10D7A0004FF0040E0AF88CEC0CF88C3C04F1020EDD
:10D7B000BEF18C0F42F0020C00F2CC8004F1980311
:10D7C0006B4403F88BCC04F1040CBCF18C0F03F810
:10D7D0008CBC00F2BF800EF198060DEB060E4FF0E8
:10D7E000060A0EF88CAC04EB0A0E4FEA8909BEF16A
:10D7F0008C0F5FFA89F603F8890C00F2AB8004F114
:10D800009C0CEC444FF007090CF88C9C04F1080CBC
:10D81000BCF18C0F03F8876C00F29C800EF1980627
:10D820000DEB060E0EF88CBC03F8852C04F10A02F1
:10D830008C2A00F28F8004F1A0060DEB060C0CF888
:10D840008CAC03F8830C04F10C008C2800F282806D
:10D8500004F1A20204F1A3036A446B4402F88C9C15
:10D86000044603F88C8C480901F01F0C55F8203051
:10D87000012202FA0CF223EA020345F82030019B50
:10D88000013B01936ED00131B1F5F07F6AD23C22A9
:10D890002846FAF7D9F9011E5FDB07EB410297F83A
:10D8A0001035B2F848C11CF0040FC1F30722C8B20A
:10D8B0005FFA8CF94FEA1C2803F0400A04F1020ECB
:10D8C0007FF459AFBAF1000F03D103F0380CCC4507
:10D8D00019D003F0870343EA0903BEF18C0F87F8E0
:10D8E000103537D804F1010C0CF1980698346C44CB
:10D8F0000DEB060C4FF0040904F88C9C74460CF8F0
:10D900008C3C0EF1020EBEF18C0F23D804F198036B
:10D910000DEB030C231D8C2B0CF88B2C0CF88CBC02
:10D9200018D80EF198020DEB020E06220EF88C2C80
:10D930000CF8890CA0188C280CD804F19C0304F175
:10D940009D026B446A44072403F88C4C044602F899
:10D950008C8C88E76FF0004485E7204614B927B027
:10D96000BDE8F08FD7F808551F4995F91030AA681F
:10D9700003EB8303920751F8230020D5234603AA23
:10D9800000216DF015FFAB689B0701D50120E6E78C
:10D99000164B17491A68174B4FF4FA7000FB02F246
:10D9A000A3FB0232486892094B681B1A9A42FBD2C9
:10D9B0006B69002BEAD01A689B881383E6E76B69D2
:10D9C00013B11A689B885383084B09491A68094B9D
:10D9D0004E68D200A3FB023292094B689B1B9A420D
:10D9E000FBD2CBE7F86F0020400D0020AC360020C2
:10D9F000001000E0D34D6210F0B5284CD4F80805B3
:10DA000083B010B194F80E350BB103B0F0BD012313
:10DA10000DF10702842184F80E35FDF713FD94F80B
:10DA20001025D4F8080504210A43FBF747FED4F873
:10DA300008050DF107028421FDF704FD9DF807306C
:10DA400013F00406F3D1164D84F810353C2231460C
:10DA5000284674F0CFFF3246124E05F13A0005F227
:10DA6000FA374FF0010E30F8023F334002F01F0149
:10DA70009BB24FEA521C0EFA01F1013223B155F864
:10DA80002C300B4345F82C30B842ECD1FFF766FE42
:10DA90000028FBD184F80E0503B0F0BDF86F00201C
:10DAA0000471002004DFFFFF70B5404DD5F8084534
:10DAB00082B08CB395F80C35012B41D0022B2DD1BF
:10DAC000082294F910303A4985F80F2503EB8303B7
:10DAD00000208DF8040051F82300A3688DF805207C
:10DAE00040F20442ADF806209A0742D504230DEB1C
:10DAF000030200216DF05CFEA3689B0722D52D4830
:10DB00003C22FF2174F076FF95F80D3523B9FFF71D
:10DB100073FF012385F80D3502B070BD0DF10302CE
:10DB2000A0212046FDF78EFC9DF8033003F005038D
:10DB3000012B37D0002B2FD1D5F808450822C0E79C
:10DB40004822BEE71C4B1D491A681D4B48684FF41C
:10DB5000FA7606FB02F2A3FB023292094B681B1A0B
:10DB60009A42FBD26369002BC9D01A689B88138341
:10DB7000C5E7636913B11A689B8853830E4B0F493D
:10DB80001A680F4B4E68D200A3FB023292094B6811
:10DB90009B1B9A42FBD2A9E70A4A126840F2DC5367
:10DBA0009A42B9D9D5F8084548228AE7F86F00208B
:10DBB000400D002004710020AC360020001000E071
:10DBC000D34D6210242A00202DE9F041334D95F801
:10DBD0000E3582B003B1FEE7012285F80E2595F8D7
:10DBE0000F25044602F0F702D5F8080585F80F2541
:10DBF0000E461946FBF762FDE2B207460921D5F849
:10DC00000805FBF75BFDB4F5807F3FD0D5F808052C
:10DC1000DFF88C8050220821FBF750FDD5F808056D
:10DC20000DF10702A021FDF70DFC48B9D8F8D83056
:10DC3000B8F8DC2059690A4214BF5A831A83EDE709
:10DC40009DF8074014F02004F0D1E2B20A21D5F883
:10DC50000805FBF733FD3219D5F80805C02101345A
:10DC6000FDF7F0FB362CF0D157B995F80F25D5F814
:10DC7000080502F0F702394685F80F25FBF71EFD6F
:10DC8000002385F80E3502B0BDE8F081D5F808050F
:10DC900040220A21FBF712FDB8E700BFF86F002011
:10DCA0002C2B00202DE9F04F5F4D95F80E75C3B079
:10DCB00007B1FEE795F80F25044602F0F7020123AD
:10DCC000D5F8080585F80F250E46394685F80E3536
:10DCD000FBF7F4FCFF2C4FF009038DF8054088BFDB
:10DCE000A40801AA8CBF04F0C008B84602204FF077
:10DCF000000C4FF00A0B0DF1050A4FF00B091370E1
:10DD000014E0B1F5827F02F800B00AF8003016F88E
:10DD10000C3017D80CF1010CBCF1360F02F807904B
:10DD200004F1060402F80E30084614D0871C48EAB5
:10DD30000C03B7F5827F00F104010446DBB200F169
:10DD4000030EDED90CF1010C6FF00041BCF1360F6F
:10DD5000364C0846EAD1B4F5827F61D80823535483
:10DD60000DF10503A0211954831CD5F8084530484E
:10DD700094F9101001EB810150F82100A168890786
:10DD800022D500216DF014FDA3689B0731D5294CE5
:10DD9000D5F808050DF10302A021FDF753FB48B9A2
:10DDA000D4F8D830B4F8DC2059690A4214BF5A8339
:10DDB0001A83EDE79DF8033013F02003F0D185F8C6
:10DDC0000E3543B0BDE8F08F616911B10E688988E6
:10DDD00071831949194F0E681949D7F804C0F60024
:10DDE000A1FB0616B6097968A1EB0C018E42FAD2A6
:10DDF000C7E7114B11491A68114B48684FF4FA767E
:10DE000006FB02F2A3FB023292094B681B1A9A42EC
:10DE1000FBD26369002BBAD01A689B881383B6E7DC
:10DE20006FF00043A1E700BFF86F00200100008001
:10DE3000400D00202C2B0020AC360020001000E00C
:10DE4000D34D6210002ABCBF80185242002B30B55F
:10DE500003EB010503DA0C465B4229462546002800
:10DE6000B7BF121A841814460020A4F11D0C002913
:10DE7000BCBF2B460021BCF1000FC4BFA2EB0C02BB
:10DE80001418A5F10F02002AC4BF9B1A5D18844222
:10DE90001EDBC1F1010C0F4AAC44C1EB0113CCEB0A
:10DEA0000C1C00EB430301344FEA4C0C02EB430221
:10DEB0004FF0200E8D42A8BF002304DB22F813E0B0
:10DEC0001E339C45FAD10130A04202F10202F1D189
:10DED00030BD00BF407100201B4B1C48196C1C4A10
:10DEE00010B441F080510124196404625321FF24CD
:10DEF000CA205462506251625B6FDB0085B013D45C
:10DF00000023144902930291029A134804320292A8
:10DF1000029A136003930391039B0393039B18607E
:10DF200005B05DF8044B70470A4B00220192019343
:10DF3000019B0193019A084B12689A42E0D105B007
:10DF40005DF8044B704700BF0038024000000E42ED
:10DF5000002800405028004076614E69012070473B
:10DF6000012070470120704731B10C4BD3ED007A8E
:10DF7000F8EEE77AC1ED007A72B1084BDFED086A7E
:10DF80005B68A3F5D543333B07EE903AF8EEE77AAA
:10DF900087EEA67A82ED007A704700BFF0A50020D8
:10DFA0000000C842012070470120704710B4414C66
:10DFB0000023224692F90410012902F10C022DD00F
:10DFC0000133052BF6D12246002392F904100329D0
:10DFD00002F10C0234D00133052BF6D1002394F961
:10DFE0000420052A04F10C043FD00133052BF6D19F
:10DFF000314B1B68D9034ED5304B016803F1F00457
:10E0000002E01433A34246D01A689142F9D1DA688B
:10E01000D201F6D501205DF8044B7047284A03EB86
:10E02000430302EB83039B68EBB1264A037992F822
:10E030003DC09C45EED092F83C209A42C3D1E9E71E
:10E040001F4A03EB430302EB83039B68002BC6D0FC
:10E050001D4A037992F83D109942DBD092F83C209A
:10E060009A42BBD1D6E72246AFE7154A03EB4303FA
:10E0700002EB83039B68002BBAD0144A037992F811
:10E080003D109942C6D092F83C209A42C2D00A4B29
:10E090001B68D903B0D40379203BDBB2152B06D81B
:10E0A0000B495DF8044BD94001F001007047002096
:10E0B000B1E700BFF8A50020B4000010040A00205A
:10E0C000F0A50020200300206C050020B8070020E8
:10E0D000010031000C4B10B5844603F1F00E002016
:10E0E00002E014339E450ED01A686245F9D1DA6811
:10E0F0008A4218BFD96000F1010403F1140318BF6C
:10E10000E0B29E45F0D110BD040A0020704700BF68
:10E11000044B40F2FF7203EBC0039142A8BF1146CB
:10E12000998070477C600020112806D8044B03EBCF
:10E1300080039B6C0BB19B6819602DF061BB00BF25
:10E14000F0A50020112806D8034B03EB80039B6C3D
:10E150000BB19B6819607047F0A500200C4A13783A
:10E160007BB10C4B93F8901059B193F8911059B1C1
:10E1700050680022FA2883F89120A8BF4FF0FF30A2
:10E1800070476FF0010070476FF00200704700BFEA
:10E1900048170020F0A500200B4B93F8922082B185
:10E1A00093F8932052B1094988680022B0F5967F10
:10E1B00083F89320A8BF4FF0FF3070476FF0020044
:10E1C00070476FF001007047F0A50020481700204D
:10E1D000024BD3F894305B68184700BFF0A50020CD
:10E1E000024BD3F894309B68184700BFF0A500207D
:10E1F000024BD3F89430DB68184700BFF0A500202D
:10E200002DE9F041104C04F1980884F89910174654
:10E21000002502234246FF21064684F89850FCF769
:10E2200077F968B1424630460223FF21FCF7E8F94E
:10E2300030B1B4F898305BBA28463B80BDE8F08135
:10E240006FF00C00FAE700BFF0A50020014BD86882
:10E25000704700BF48170020044B93F8983113B162
:10E26000034B186970476FF001007047F0A500205C
:10E270004817002070B5324C05460323006804F5AA
:10E28000CE720021FCF7BCF958B96FF00103C4F855
:10E29000A0312C4AD4F8A431116832338B4245D3D3
:10E2A00070BDB4F89C3194F89E015BBA9BB207EE46
:10E2B000903AF8EEE77AF2EE046A87EEA67A94F8DE
:10E2C0009C310821BDEEC77A84ED687A4FFA83FC51
:10E2D000BCF1000F4FEA4C02A8BF5B0082F00702BE
:10E2E000B4BFD3B2DBB20139F0D194F89D2108213B
:10E2F00053405AB2002AB8BF52004FEA4303B6BF98
:10E3000082F00702DBB2D3B20139F2D19842C0D118
:10E31000D4F8A0312BB1D4F8A0214FF6FF739A4264
:10E32000B7D14FF0FF33C4F8A031B2E7C4F8A4115D
:10E330002868054ABDE8704001233121FCF7E8B8A0
:10E34000F0A50020242A002098A70020014BD3F834
:10E35000A0017047F0A50020437A5A1C0344D2B2B2
:10E3600042729972037A934200D97047002AFCD016
:10E3700010B5044604F10A01D0E9003098470023A3
:10E38000637210BD324ED6F8A851D6F8B40180B5EC
:10E3900031F06EF8284631F06BF8D6F8B47179791F
:10E3A0008B074BD500210846FEF72EFF00210120E8
:10E3B000FEF72AFF274C3B6838465B68984760B9F0
:10E3C0002B6828465B68984708BBD6F8B4713B6851
:10E3D00038465B6898470028F2D0D6F8B401D4F8E4
:10E3E000D8200368B4F8DC10DB68518398472B68A9
:10E3F00001461B6828469847D4F8D830B4F8DC208A
:10E400001A832B6828465B6898470028DDD0D4F82B
:10E410009C202B68B4F8A010DB68518328469847ED
:10E420000146D6F8B40103681B689847D4F89C30BD
:10E43000B4F8A020D6F8B4711A83BCE73B6838461C
:10E440009B6941F002019847D6F8B471AAE700BF72
:10E45000F0A500202C2B002070B50668F56982B06D
:10E460000446002D59D000232B7004230DEB03022A
:10E470003046FF21FCF7C4F810B9002002B070BD8F
:10E48000206804236A46FF21FCF7BAF80028F4D07C
:10E490009DF804309B09023B012BEED9BDF80430F6
:10E4A000BDF80620BDF80010BDF802605BBA43F667
:10E4B000FF74C3F30D03A342DFD0002BDDD052BAAB
:10E4C000C2F34A1240F2FF7C6245D6D0002AD4D073
:10E4D00049BAC1F30D01A142CFD00029CDD076BAFF
:10E4E000C6F34A166645C8D0002EC6D05C1A002C6A
:10E4F000B8BF6442FF2CC0DC941B002CB8BF644240
:10E50000FF2CBADC0B445B1032445210C5F80530C6
:10E510000123C5F801202B70B0E709211420FAF778
:10E520003BF9F061054626689DE700BF70B50668B7
:10E53000F0690D461446A0B3D0F80130CDB1D0F843
:10E5400005209FED1B7ADFED1B5ADFED1B6A07EEFE
:10E55000902AF8EE677AB7EE006A77EEC77A77EE20
:10E56000A77A87EEA57A77EE467A67EEE67AC5ED6A
:10E57000007AACB107EE903A9FED107ADFED106AA9
:10E580009FED106AF8EEE77A67EE877A87EEA67A53
:10E59000DFED0D6A77EE467A77EEA67AC4ED007A63
:10E5A00070BD09211420FAF7F7F8F061C4E700BF45
:10E5B0009AC9CC449AC94C460E76D74500004843C8
:10E5C00000E0FF44000048423393884370B506687A
:10E5D000F46982B0F4B10023237004230DEB03022D
:10E5E000FF213046FCF70CF810B39DF804309B096E
:10E5F00019D1BDF80420BDF8063052BA5BBA92B208
:10E60000C3F34A1301212170C4F80520C4F8013076
:10E6100002B070BD054609211420FAF7BDF8F0617B
:10E6200004462E68D7E7044A04210320FAF72EF89F
:10E63000002002B070BD00BFC4E5080870B50668D0
:10E64000F06982B00D461446002848D0D0F8053055
:10E65000DFED266A9FED267A07EE903AF8EE677AAC
:10E66000D0F8013077EEE67AF3EE096A67EE877A42
:10E67000B2EE047A67EEA67AF4EEC77AF1EE10FAFB
:10E6800020DCBAEE047AF4EEC77AF1EE10FA19D46F
:10E690002DB19FED187A67EE877AC5ED007A7CB1CF
:10E6A00007EE903A9FED146ADFED146AB8EE677AD0
:10E6B000DFED137AE7EE067A77EEA67AC4ED007AFC
:10E6C00002B070BD17EE900A6DF0BEFC0D4ACDE9A8
:10E6D000000104210320F9F7D9FF02B070BD092120
:10E6E0001420FAF759F8F061B0E700BF00000046C7
:10E6F000000080380AD778430319C83D3393884314
:10E70000000048C2E8E50808F0B52DED028B4E4E3A
:10E7100016F81C3C022B83B00D46144619D0DFEDD1
:10E720004B7A7DB19FED4A7A9FED4A6ADFED4A6AE6
:10E7300067EEA77A67EE877A87EE867A77EE267A93
:10E74000C5ED007A0CB1454B236003B0BDEC028BE4
:10E75000F0BD434B96F840105B6803F0020239BBF2
:10E760005B0525D42AB3B6F9663007EE903AB6F9C0
:10E770006430F8EEE77A06EE903A27EEA77AF8EEE4
:10E78000E66AB6F96830A6EEA67A07EE903AF8EE99
:10E79000E77AA7EEA77AB5EEC07AF1EE10FABEDB03
:10E7A000F1EEC77AF4EE677AF1EE10FAB9D7B6E770
:10E7B00022B9D6F88030D3ED337AB2E7294F0DF184
:10E7C00006002BF003FEBDF80630D7F8CC259FEDF0
:10E7D000266ADFED266A9FED267A9B1A07EE903AAD
:10E7E000F8EEE77AB0EE408A67EE867AA7EEA67A70
:10E7F000FDEEC77AB0EE470A17EE903A2033402B71
:10E800001FD8F9F78BFD1B4B97F8F211D6ED137A51
:10E81000A3F12C021846443B002918BF134693ED80
:10E82000057AD0ED006A77EE877AE8EE406A27EE47
:10E83000A77AA6EEA67AB5EEC07AF1EE10FAAFDAB4
:10E840006DE79FED020ADEE7E8B600200000000059
:10E85000CDCC9C3F00409C4682E6C5473313904395
:10E86000B4000010F0A500200AD7233C35FA8E3CF6
:10E87000DB0FC93FD0AB002010B50B4B82B053F873
:10E88000304001916CB107EE901A94ED047A94ED4A
:10E89000030AF8EEE77AA7EE870A6FF00DF8A3688F
:10E8A000186002B010BD00BF7C6000202DE9F0416F
:10E8B0004C4F97F8903082B043B14B4E96F884504D
:10E8C000012D04463AD0022D59D015B102B0BDE851
:10E8D000F081012280210068FAF7F0FE2068012211
:10E8E000FF21FAF7EBFE2A4629462068FAF7E6FEF2
:10E8F00096F8852020689121FAF7E0FE29462068E5
:10E900000122FAF7DBFE2A462068FF21FAF7D6FE3D
:10E910002A4620688021FAF7D1FE29462068012284
:10E92000FAF7CCFE314B32491A6808700123C6F859
:10E93000882086F8843002B0BDE8F08101AA006822
:10E94000DFF8AC800021FCF77DFD9DF8043088F8ED
:10E950000000DA073ED5D6F88C30002BB6D0234A1B
:10E96000D6F88810126892B2521A9342AED24FF083
:10E97000FF320023C8F8042086F88430A6E7006838
:10E98000DFF86C8001AA1321FCF75CFD9DF80430D0
:10E9900088F800005B07DED020682B4601AA1E2104
:10E9A000FBF72EFEBDF80430206801220B215CBA73
:10E9B000FAF784FE0F4B88F80000A4B2A3FB0434DE
:10E9C000E40801220023C8F8044087F8912086F863
:10E9D00084307BE7054A02231268C6F8882086F84F
:10E9E000843073E7F0A50020E8B60020242A002038
:10E9F00048170020CDCCCCCC2DE9F041DFF8B48015
:10EA00002A4E2B4D41F0010284B000210446FAF752
:10EA100055FED8F80070C6F8887018E0022B3CD17B
:10EA2000A368DB070DF10F024FF0130120465EBF14
:10EA30000DF10F0293212046FCF7B4FC9DF80F3036
:10EA4000287013F0070318D1D6F88C203ABB23792D
:10EA5000012BE3D1A268617C94F9100002F001025D
:10EA600001920DF10F0200921322F5F721FD9DF89E
:10EA70000F30287013F00703E6D001220B21204647
:10EA8000FAF71CFE002211462046FAF717FE012372
:10EA90002870184604B0BDE8F0810020CEE7D8F811
:10EAA000001089B2C91B8A42D1D2F2E7E8B6002031
:10EAB00048170020242A002010B5164C84F899101D
:10EAC000017984F89A2001294FF0000282B084F87D
:10EAD000982010D0022903D06FF00C0002B010BDB6
:10EAE000032304F19802FF21FBF7BCFC0028F3D0BC
:10EAF000002002B010BD8268417C90F9100098346B
:10EB000002F00102CDE900420323FF22F5F704FDE4
:10EB1000ECE700BFF0A5002000680379012B0BD0C3
:10EB2000022B00D0704783680E4A13F0010315D002
:10EB300000235121FBF796BC00B58368094A417C4C
:10EB400090F9100083B003F00103CDE90023002306
:10EB50005122F5F7E1FC03B05DF804FBD121FBF78E
:10EB600081BC00BF78B7002000680379012B0CD06E
:10EB7000022B00D0704783680E4A13F0010F4FF04C
:10EB8000010313D00021FBF76DBC00B58268417C06
:10EB900090F9100083B002F001020192054A009240
:10EBA0000022F5F7B9FC03B05DF804FB8021FBF708
:10EBB00059BC00BF98A7002030B5194D95F8923088
:10EBC00083B00BB903B030BD04460DF105010068F8
:10EBD0006AF07CFD9DF805307BB92068114A01215F
:10EBE0004FF4064485F89A100323FF21A5F89840B6
:10EBF00003B0BDE83040FBF78BBC0DF10602962157
:10EC00002068FFF7FDFA084ABDF806300749A2FB65
:10EC10000323DB0801228B6085F89320DDE700BF2A
:10EC2000F0A5002088A60020CDCCCCCC4817002031
:10EC300010B5044600680379012B84B029D0022B5B
:10EC40000DD01F4B6FF00102DA601E4A1E49D2F848
:10EC50009030096832338B4229D304B010BD8268EA
:10EC600012F0010F18BF512103AA08BFD121FBF7F1
:10EC700071FC0028E5D0BDF80C30114A5BBA9BB29C
:10EC8000D360D368B3F5C87FDFDD4FF0FF33D360C7
:10EC9000DBE78368417C90F9100003F001030193E6
:10ECA00003AB009351220223F5F702FCE1E742F89F
:10ECB000901F206800235121FBF72AFC04B010BDEF
:10ECC00048170020E8B60020242A002000B500687C
:10ECD0000379012B85B02DD0022B24D1826812F04C
:10ECE000010F18BF002103AA08BF8021FBF732FCE7
:10ECF0001B4B83F8980198B1BDF80C305BBA9BB2FE
:10ED0000B3F5FA6F24D2174A1749A2FB0323DB0895
:10ED100007EE903AF8EEE77AFDEEE77AC1ED047A75
:10ED200005B05DF804FB0E4B002283F8982105B076
:10ED30005DF804FB8368417C90F9100003AA03F09E
:10ED40000103CDE9002302230022F5F7B1FBCFE751
:10ED5000054B4FF0FF321A6105B05DF804FB00BFB0
:10ED6000F0A50020CDCCCCCC4817002010B5006811
:10ED70000379012B84B00C461FD0022B02D0002057
:10ED800004B010BD826812F0010F18BF002103AA61
:10ED900008BF8021FBF7DEFB0028F0D05CB19DF8B6
:10EDA0000D309DF90C20DB0903EB830302EB82029B
:10EDB00003EB4203238004B010BD8368417C90F9CB
:10EDC000100003F00103019303AB00930022022320
:10EDD000F5F76EFBE0E700BFF8B504460F461646B0
:10EDE00000252046202174F0CCFC0446C8B10378ED
:10EDF000202B03D114F8013F202BFBD02046FAF73B
:10EE0000BDF9B0F5617F10DB40F63403984211DDA7
:10EE100030231A46C5B17B703378013333702046F6
:10EE2000F8BD002DFBD10125DBE700231A46002D9C
:10EE3000F1D109E0074AA0F56173A2FB0323DA08C8
:10EE4000C3F3C703002DE6D13A7033780133337032
:10EE5000E9E700BF1F85EB5170B50546BDF81060AE
:10EE600001600C4619B119462046F3F7C5FF31463B
:10EE70002046F4F739F861680B68B3F844206FEA6C
:10EE800042426FEA524292B2A3F844201A8892B2E8
:10EE900042F001021A804A79032A17D8DFE802F00B
:10EEA000110C070240330022AB601A6070BD3C3386
:10EEB0000022AB601A6070BD38330022AB601A606C
:10EEC00070BD34330022AB601A6070BD0023AB60AC
:10EED0001B60FFDE2DE9F04F85B00646BDF838B067
:10EEE0009DF83CA0894617469846F3F719FF00287D
:10EEF00056D02C4C94F894300A2B4CD803EB430298
:10EF000004EB421202900020C2F8980082F89C00A4
:10EF10005A1CD2B284F8942003EB43033079039255
:10EF2000983404EB4314FDF7DDFD0299054618B350
:10EF3000039A027280F806900220E87143463A462E
:10EF4000CDF800B02046FFF787FFBAF1000F0AD1D5
:10EF500011212846FDF766FD2B68AA885A832046B2
:10EF600005B0BDE8F08F2846327A0221FDF77EFD1C
:10EF7000204605B0BDE8F08FCDF800B043463A46D4
:10EF80002046FFF769FFBAF1000FECD1112150467E
:10EF9000FDF748FDE3E7044A00210420F9F776FB7A
:10EFA0000024DCE7E8B600200CE6080830B503686A
:10EFB000284D294C2DED028BAB42246883B0F0EE36
:10EFC000408AB0EE608A10D005F58065AB420CD067
:10EFD00005F57055AB4208D005F58065AB4204D00D
:10EFE00005F58065AB4218BF6408B4FBF1F303F587
:10EFF0007F43FF331B0CB4FBF3F40023B4FBF1F5A8
:10F00000019200932246ABB20221FFF763FFE0B109
:10F01000B5EE408A07EE904AF1EE10FAF8EE677A04
:10F020000ABF07EE105A28EE278AB8EE478A9FEDEE
:10F030000B7AC8EE076A0123037127EE667AC0EDEA
:10F04000046AA8EEA77A80ED037A03B0BDEC028BC8
:10F0500030BD00BF00000140F40A002000007A44E7
:10F060002DE9F04F2DED028BAA4BAB4E1B78AB4D2B
:10F07000DFF8CC92B5B000270293B046B246BB464B
:10F08000DAF80040002355F83320944203D00133CE
:10F090000E2BF8D1FF234B4493F8B834022B00F029
:10F0A000BB80032B00F0AF80012B09D1DAF80C30C4
:10F0B00023F0807323F0080343F00403CAF80C30F4
:10F0C0005046FEF773FF48B90BEB8B0308EB830345
:10F0D000D96801F00C03042B00F0A9800BF1010B9F
:10F0E000BBF10C0F0AF1140ACAD18D4DDDF808806E
:10F0F000A5F1F00408E02068E260FEF7EBFF504461
:10F10000C7B21434A5421FD02046FEF74FFF002897
:10F11000F7D1E368590703F00C02F2D5042AF0D0C6
:10F1200023F0080242F00402781C474511465FFABA
:10F1300080FA23F00403DED32068E3601946143418
:10F14000FEF7C8FFA542DFD10025764FDFF8F4A116
:10F150002C46A846AB463046FEF728FF002840F074
:10F16000A880F06842076AD5029B57F80C2C4345EB
:10F1700000F2A680030764D4002D57F80C3C40F33E
:10F18000BD8028A900229C4602E0AA4200F0B5807A
:10F1900051F8043F1B689C4502F10102F5D1C20100
:10F1A00064D40BF1010BBBF10C0F06F1140607F14F
:10F1B0001407D0D1574B93F800E0BEF10C0F00F3C9
:10F1C0000E82594B594A1B791370032B40F2BC80B5
:10F1D0001A1F022A00F27582052B00F06382062BAB
:10F1E0000CBF4FF47A564FF47A66514951480022C9
:10F1F0004A600027504AB2FBF6F200260A60C0E9D6
:10F2000000674E4AA1E0DAF80C3023F00C0343F01B
:10F210008073CAF80C3053E7DAF80C3023F08073AF
:10F2200023F0040343F00803CAF80C3048E72046F3
:10F23000FEF750FF0137FFB20744FFB24EE7020767
:10F24000ADD5002C57F80C3C4BDD1DA900229C4687
:10F2500001E0A24244D051F8043F1B689C4502F1F2
:10F260000102F6D1410787D4C2019AD5002C57F884
:10F270000C3C0ADD1DA9002251F8040F00688342EE
:10F2800002F101028DD0A242F6D1002D0ADD28A99B
:10F29000002251F8040F0068834202F1010280D07D
:10F2A000AA42F6D14FF080711846F160FEF712FFC6
:10F2B00077E75B46524601210420F9F7E7F970E74A
:10F2C00020F00801F1601046FEF704FFF06808F135
:10F2D000010803075FFA88F8B3D44107C4D54BE7A8
:10F2E0006346184634AB03EB85020821F16042F80F
:10F2F0002C6C0135FEF7EEFE53E76346184634AB3F
:10F3000003EB84020421F16042F8586C0134FEF7EB
:10F31000E1FE46E7AC000010040A0020AC3C0808FF
:10F32000F40A0020100A0020406200203160002012
:10F33000386000204060002040420F0011E10008CA
:10F34000E8B6002048E60808B74AC9F8C824B74A12
:10F3500012F81330002B00F0AE81A64500F3B38104
:10F36000BEF1000F00F0A6809FEDB18ADFF818B360
:10F37000DFF80C8304951DAC4FF0000A7746AD4BC7
:10F38000DBF800201B7854F8046FC2F30072062BE0
:10F3900000F23A81DFE803F0B4AAA0790404040083
:10F3A000052B00F07381A449A448062B18BF014621
:10F3B0000025019200950A46142302213046FFF7EA
:10F3C00089FD0290002800F01F819D4B31681A785A
:10F3D000002A00F01081CDF80C8003E00135954241
:10F3E00000F00B812B0158F803309942F6D1EAB2B4
:10F3F000082A00F009810298924B016805910D6876
:10F400004E6807954FF4907101FB0231039BC16573
:10F4100003EB02130691996013016A6E0893356835
:10F42000002A00F05481B5F844306FEA43436FEA94
:10F4300053439BB2A5F844302B889BB243F0800322
:10F440002B8073790A9319467F4B585CB379298CCA
:10F450005B074CBF0423012383409BB289B221EA9E
:10F4600003012984298C89B20B432B842B889BB2FE
:10F4700043F001032B80002A00F05781029A0123F8
:10F480001371724B43F83A200EE0DFED710A714BB5
:10F49000B0EE600A59883046FFF788FD6B4B43F8A1
:10F4A0003A00002800F09D810AF1010A57457FF4D7
:10F4B00066AF049D99F8CC3D63BB674A02210420E6
:10F4C000F9F7E4F899F8C604B0FA80F0400935B0CD
:10F4D000BDEC028BBDE8F08FDFED600A9FED600AA6
:10F4E00030464FF4FA61FFF761FDD7E7DFED5D0AC3
:10F4F0003046B0EE600A4FF47A71FFF757FDCDE762
:10F500009FED4B0AF0EE480A30464FF4C871FFF702
:10F510004DFDC3E799F8CD8D99F8CE3D08F101086E
:10F52000A8EB0308B8F1120F0BDD122302210093A0
:10F530004D4A89F8C614434600210420F9F7A6F87D
:10F54000C0E799F8D83D012B00F0B180022B40F0C4
:10F550009F8069F0C5FD454A99F8D83DC9F8DC2D72
:10F56000002B00F0A280022B40F09680122D2B463B
:10F57000B8BF12239BB24345C0F2CD80A845A8BFB7
:10F58000A846B8F1000F9DDD394EDFF8FCB0394FC9
:10F5900028AD002404E00134444546F8040B91D022
:10F5A000DBF80030B9F8D01DC3F30072B9F8D23DD2
:10F5B00001920091B7FBF3F32E4A55F8040F9BB26A
:10F5C0000321FFF787FC0028E5D1052501462A4ADB
:10F5D00089F8C65423460420F9F758F872E7274AF9
:10F5E000CDF800B0012189F8C6147346002104202B
:10F5F000F9F74CF85EE7224B039313010398C150CF
:10F600000F49531C0B70F3E6104A049D002342F887
:10F610003A30052189F8C6141A4A534600210420BD
:10F62000F9F734F846E700BF79E80008803D08089C
:10F630006F12833A31600020001BB700C0C62D0056
:10F6400078600020B4BB00205C3D08087C6000208E
:10F65000000000004062002010E70808ACC5A73792
:10F66000ACC5A7366F1203392CE7080829E100085A
:10F6700038A6002040420F00CCE7080860E60808E2
:10F68000DC600020E8E60808B400001056498FE668
:10F69000564AC9F8DC2D43B1554A02210420F8F737
:10F6A000F5FF0FE74FF4FA569FE52B4662E769F046
:10F6B00017FD504A50E7504A02210420F8F7E6FFB0
:10F6C000F8E64E4A41E64E4A009403218BE7D6F80D
:10F6D00010C04C49099213464FEA431E01EB4310F8
:10F6E00051F80E208CEA020E1EF47C5F03F1010338
:10F6F00009D0102BF0D1059A0023D360424B029A17
:10F7000043F83A20D0E6059B099AD860037F002B86
:10F710003FF489AEF2E7042000953C4A89F8C6041C
:10F7200043460021F8F7B2FFCCE6059B3849DB6879
:10F7300009931A46374B526809989A42364A136B16
:10F740000CBF43F4001343F4800313630723838344
:10F750000322059BF3F72CFE099880680B90F4F7C1
:10F7600039F80B98069A03680F9223F00103327C54
:10F7700003602A4B069053F822300D930023CDE905
:10F780001833CDE91A3312931693122311934FF4C1
:10F79000806313934FF480464FF48053CDE91436C1
:10F7A00040234C3510930DA94FF400330E95179359
:10F7B00068F00EFB0698089D039A036809992A448D
:10F7C000079D43F0100303606966154B0A9933F8EF
:10F7D0001130A5F8683093815060059A01231374A5
:10F7E0004CE6049D15E700BF808D5B0045E10008F5
:10F7F00058E7080801B803088CE608080DE100087E
:10F80000ACE60808F80A00207C60002094E70808AD
:10F81000A10200080060024000380240603D080874
:10F82000503C080810B5104CD4E90423A16882B0FC
:10F8300002FB03F38B428DF8070012D06368E06887
:10F840000DF10701184471F0B3FF63682269A168E4
:10F8500013446269B3FBF1F0013201FB10336360C2
:10F86000626102B010BD00BF5060002010B5037986
:10F87000012B84B00C4626D0022B22D18368DB07F3
:10F880000DF10F024CBF01218121FBF78BFD9DF88B
:10F890000F300022C3F3001161F30702C3F38001AC
:10F8A00061F30F220F49C3F3C00C6CF317420870C9
:10F8B000C3F3801161F31F62DB092260237104B07E
:10F8C00010BD0020E3E782680DF10F0102F0010294
:10F8D000CDE900121A46417C90F91000F4F7E8FDDA
:10F8E000D5E700BF481700202DE9F04182B014464B
:10F8F0000E4601AA50210546FBF7A4FD9DF80430F1
:10F90000DFF8F080394F01335B00DBB24621238002
:10F9100001AA2846FBF796FD23789DF8042008FBF2
:10F9200003F303F5FA73A7FB031301329909DB090B
:10F9300002FB0133A280A7FB03239B0901AAE3601A
:10F94000512102232846FAF75BFE2378BDF8040014
:10F9500008FB03F340BA03F5FA73A7FB0323C2B213
:10F96000C0F307208240013292B29809DB0902FB02
:10F970000033A7FB03739B097021E280238201AA55
:10F980002846FBF75FFD9DF8043001335B00DBB2D6
:10F9900001AA6380712102232846FAF731FEBDF8DF
:10F9A0000430134AF17810705BBADAB2C3F307235C
:10F9B0009A40013292B2228119B1E388D21A92B2EE
:10F9C00022810C48A378094900FB03F303F5FA737D
:10F9D000A1FB03039809DB0902FB0033A1FB03131E
:10F9E0009B09638202B0BDE8F08100BFD34D621075
:10F9F00048170020002F3A002DE9F04FDFF89882D9
:10FA0000DFF89892DFF898A2A24F8DB00546002645
:10FA10004FF4FA7307AA89210068C8F88C3089F876
:10FA20009060FBF70FFD9DF81C202868892142F0AB
:10FA30000102F9F743FE324688212868F9F73EFEB5
:10FA4000012280212868F9F739FE0122FF21286868
:10FA5000F9F734FE324631462868F9F72FFE07AA37
:10FA600091212868FBF7EEFC9DF81C30286888F887
:10FA7000853031460122F9F721FE3246FF21286800
:10FA8000F9F71CFE324680212868F9F717FE07AA0D
:10FA900060212868FBF7D6FC9DF81C2028686021AF
:10FAA00042F01202F9F70AFE4FF40053ADF81C3091
:10FAB00007AA022344212868FAF72AFDFF22012120
:10FAC0002868F9F7FBFD2C68012280212046F9F710
:10FAD000F5FD0122FF212046F9F7F0FD32463146BF
:10FAE0002046F9F7EBFD0622FF212046F9F7E6FD57
:10FAF00007AA83212046FBF7A5FC9DF81C20832143
:10FB000042F004022046F9F7D9FD0722FF212046E2
:10FB1000F9F7D4FD012281212046F9F7CFFD01221A
:10FB200080212046F9F7CAFD6B2294212046F9F77F
:10FB3000C5FD324683212046F9F7C0FDDAF80060A2
:10FB4000C8F888602379012B00F09680022B0ED034
:10FB500000209DF81C303870D3B9DAF800309BB221
:10FB60009B1BB3F5FA7FEDD90DB0BDE8F08FA3680C
:10FB7000DB0707AA4FF0830120465EBF07AA832157
:10FB80002046FBF70FFC9DF81C303870002BE4D0AA
:10FB9000012283212046F9F791FD07AA92212046F0
:10FBA000FBF750FC0022812120469DF81CB0F9F79C
:10FBB00085FD0622FF212046F9F780FD07AA832153
:10FBC0002046FBF73FFC9DF81C20832102F0FB023E
:10FBD0002046F9F773FD0122FF212046F9F76EFD5B
:10FBE000012200212046F9F769FD0022FF2120466D
:10FBF000F9F764FD204600228021F9F75FFD062316
:10FC0000B02105AA2868FAF7FBFC0122FF21286829
:10FC1000F9F754FD00224F212868F9F74FFD2C22F7
:10FC20004E212868F9F74AFD0022FF212868F9F7DC
:10FC300045FD4FEADB162868B422B621F9F73EFDF0
:10FC40000024002E18BF0C260BF07F0BA2464FF0AD
:10FC5000010EC4F3C40330336B44E2B213F81C0C3E
:10FC600004F0070C0EFA0CF1964220EA010119D9B2
:10FC700003F81C1C0134ECE7A268617C94F91000C5
:10FC800002F00102019207AA00928322F4F710FC0D
:10FC90005FE700BF48170020E8B60020F0A500206D
:10FCA000242A0020DA4540FA0CF200F00E83D30734
:10FCB00044BF0AF1010A5FFA8AFA0134302CC8D134
:10FCC000062305AAB0212868FAF722FC0122FF21A9
:10FCD0002868F9F7F3FC002211462868F9F7EEFCD2
:10FCE0000022FF212868F9F7E9FC00220921286891
:10FCF000F9F7E4FC002210212868F9F7DFFC002264
:10FD000011212868F9F7DAFC012224212868F9F783
:10FD1000D5FCFF2225212868F9F7D0FC00227521A7
:10FD20002868F9F7CBFC0122FF212868F9F7C6FC07
:10FD30002C224E212868F9F7C1FC002248212868AE
:10FD4000F9F7BCFC214620222868F9F7B7FC00220D
:10FD5000FF212868F9F7B2FC214609222868F9F743
:10FD6000ADFC002254212868F9F7A8FC04223121B7
:10FD70002868F9F7A3FC032232212868F9F79EFCD2
:10FD8000832240212868F9F799FC2522462128681A
:10FD9000F9F794FC002260212868F9F78FFC002213
:10FDA00027212868F9F78AFC062250212868F9F7EC
:10FDB00085FC002251212868F9F780FC9622522107
:10FDC0002868F9F77BFC082256212868F9F776FCA9
:10FDD000224657212868F9F771FC00226121286822
:10FDE000F9F76CFC002262212868F9F767FC002211
:10FDF00064212868F9F762FC002265212868F9F778
:10FE00005DFCA02266212868F9F758FC0122FF2139
:10FE10002868F9F753FC322222212868F9F74EFCB2
:10FE2000142247212868F9F749FCFF224921286854
:10FE3000F9F744FC00224A212868F9F73FFC002228
:10FE4000FF212868F9F73AFC0A227A212868F9F795
:10FE500035FC00227B212868F9F730FC212278212B
:10FE60002868F9F72BFC0122FF212868F9F726FC06
:10FE7000342223212868F9F721FC00224221286836
:10FE8000F9F71CFCFF2244212868F9F717FC262209
:10FE900045212868F9F712FC052246212868F9F760
:10FEA0000DFC402211462868F9F708FC06220E21B5
:10FEB0002868F9F703FC1A2220212868F9F7FEFBCD
:10FEC000402243212868F9F7F9FB0022FF21286826
:10FED000F9F7F4FB032234212868F9F7EFFB4422F9
:10FEE00035212868F9F7EAFB0122FF212868F9F794
:10FEF000E5FB042231212868F9F7E0FB09224B21B8
:10FF00002868F9F7DBFB05224C212868F9F7D6FBB6
:10FF100004224D212868F9F7D1FB0022FF2128682F
:10FF2000F9F7CCFB002244212868F9F7C7FB20220F
:10FF300045212868F9F7C2FB082247212868F9F70C
:10FF4000BDFB282248212868F9F7B8FB0022672169
:10FF50002868F9F7B3FB042270212868F9F7AEFB93
:10FF6000012271212868F9F7A9FBFE227221286875
:10FF7000F9F7A4FB002276212868F9F79FFB0022FD
:10FF800077212868F9F79AFB0122FF212868F9F701
:10FF900095FB01220D212868F9F790FB0022FF2133
:10FFA0002868F9F78BFB012280212868F9F786FB86
:10FFB000F82201212868F9F781FB0122FF21286836
:10FFC000F9F77CFB01228E212868F9F777FB0122E3
:10FFD00000212868F9F772FB0022FF212868F9F751
:10FFE0006DFB002280212868F9F768FB04220A21B2
:10FFF0002868F9F763FB2C68842107AA2046FBF7E1
:020000040801F1
:1000000021FA9DF81C20204602F0EF028421F9F726
:1000100055FB01220B212868F9F750FB2C6803A936
:100020002046FFF723FC07AA03A92046FFF75CFC44
:100030009DF80C30002B00F059810A9C04F6845482
:100040009DF80E30002B00F047810A9B03F2B2238B
:1000500004EB43049DF80F3023B1BDF82C3003F5B9
:1000600025731C449DF8103023B1BDF82E3003F2E7
:1000700026231C44E82201212868C8F8E04DF9F73E
:100080001DFB2868214669F057FB012211462868AC
:10009000F9F714FB402138702868FEF7ADFC002802
:1000A0003FF462AD012128680222F9F707FB002125
:1000B00038702868FEF7A0FC00283FF455ADE82210
:1000C00001212868F9F7FAFA4FF4005307AAADF8AE
:1000D0001C30442102232868FAF71AFA2C6803A975
:1000E0002046FFF7C3FB07AA03A92046FFF7FCFB46
:1000F000502257212046F9F7E1FA082256212046DE
:10010000F9F7DCFA082250212046F9F7D7FABDF8B2
:100110002C204FF47A7148F20E6301FB0233784AC7
:10012000934240F2EA80774AA2FB0332120C013A72
:10013000FF2A4FF0000306DD52080133FF2A9BB26D
:10014000FAD81B029BB21343C3F30722DBB28DF82C
:1001500008208DF8093002AA022351212046FAF71F
:10016000D7F90A9A4FF47A7148F20E6301FB023311
:10017000654A934200F2BF80624AA2FB0332120C2E
:10018000013AD2B246212046F9F798FA2046D8F82B
:10019000E01D69F0D1FA02AA01212046FBF752F9CD
:1001A00002229DF8086001212046F9F787FA002114
:1001B0002046FEF721FC324620460121F9F77EFA5F
:1001C0002C6803A92046FFF751FB07AA03A9204684
:1001D000FFF78AFB482211462046F9F76FFA0822FA
:1001E00047212046F9F76AFA032232212046F9F71F
:1001F00065FA072230212046F9F760FA0122FF2133
:100200002046F9F75BFA202230212046F9F756FA0A
:100210000022FF212046F9F751FA062270212046DC
:10022000F9F74CFABDF82E10384A4FF47A7046F6BA
:10023000440300FB0133A2FB03239DF80F201B0B9B
:100240001AB1BDF8222013449BB2002B51D05A1E84
:10025000FF2A4FF0000306DD52080133FF2A9BB24C
:10026000FAD81B029BB21343C3F30722DBB28DF80B
:1002700008208DF8093002AA022371212046FAF7DE
:1002800047F9D8F8E01D204669F056FA02AA012184
:100290002046FBF7D7F89DF808500222012120469E
:1002A000F9F70CFA00212046FEF7A6FB2A46204665
:1002B0000121F9F703FA642201233870C8F88C2071
:1002C00089F890300DB0BDE8F08F0EFA0CFC20EAF2
:1002D0000C0003F81C0CF0E49DF80D30002B3FF4EB
:1002E000B9AE0A9B03F525731C44B3E640F63634D9
:1002F000A6E61A46BBE7FF2244E700231A4626E794
:100300001B0C0100950370F41B280D014963A41315
:1003100010B5164C84F89910017952BAA4F89A20B5
:1003200001294FF0000282B084F8982010D00229F1
:1003300003D06FF00C0002B010BD042304F198024A
:10034000FF21FAF78FF80028F3D0002002B010BD8B
:100350008268417C90F91000983402F00102CDE9E6
:1003600000420423FF22F4F7D7F8ECE7F0A50020C1
:100370002DE9F04F9D4F9E4D06683C464FF000081A
:1003800085B0834685F892805B37C4F12D0905F16D
:10039000980A13E0022B0FD1B26812F0010F4FF050
:1003A000030352464FF0FF01304601BF032352467C
:1003B000FF213046FAF756F8A7421AD0337985F86C
:1003C000988009EB0401012B14F8012F85F899108E
:1003D00085F89A20DED1B368717C96F9100003F09D
:1003E0000103CDE900A3FF220323F4F795F8A74208
:1003F000E4D14FF40743A5F89830402385F89A30AC
:1004000052460323FF213046FAF782F800238DF885
:100410000E300DF10E01304669F058F99DF80E309E
:10042000002BF6D04FF40643A5F898300123714A0B
:1004300085F89A30FF2103233046FAF769F84FF424
:1004400007436C4AA5F8983000240323FF21304667
:1004500085F89A40FAF75CF84FF40063A5F89830F5
:100460000923644A85F89A30FF2103233046FAF7BE
:100470004FF84FF43063A5F898305E4A85F89A40FB
:1004800030460323FF21FAF743F8002800F0AC8040
:10049000DBF800400DF10E025E212046FDF7B0FEB4
:1004A000BDF80E30B3F5D77F00F08C806AD8512BA1
:1004B00000F0848078D81D2B7ED10F2608BB0A223D
:1004C0004B212046FEF7F8FA0F2260212046FEF766
:1004D000F3FA0D2263212046FEF7EEFAB8226921D5
:1004E0002046FEF7E9FA40F60D7278212046FFF724
:1004F0000FFF40F60E627A212046FFF709FF002821
:100500006DD0DBF80000212169F036F8DBF80040FF
:100510000DF10E02DE212046FDF772FEBDF80E3011
:100520009FED357AC3F3090303EB8303DB0007EE8A
:10053000903AF8EEE77A4FF4D84267EE877AA5F85A
:100540009820FCEEE77A524617EE903A1BBAC5F8AF
:100550009A30FF2106232046F9F7DAFF4FF40741CE
:100560004023DBF80000A5F8981085F89A30524631
:100570000323FF21F9F7CCFFB0B385F8920005B053
:10058000BDE8F08F40F2E132934219D01CD840F21E
:10059000D922934214D040F2E122934202D0B3F523
:1005A000E67FAED1642689E7AD2B0BD0D62B01D0E8
:1005B000602BA6D1212681E71E2BA2D114267DE730
:1005C000C8267BE7322679E740F28F42934203D078
:1005D00040F29152934294D14FF4FA766EE731464D
:1005E000204668F0C9FF8CE70020C6E727430808CB
:1005F000F0A5002088A600209A99893F03682DE97C
:10060000F0411F6A1FB13B46BDE8F0411847002A80
:10061000164611DD04460D460E4400E023689B6833
:10062000204698470028F9D0236815F8011B1B685D
:1006300020469847B542F1D1BDE8F081DEE700BF22
:10064000204A214B116893F8EE2DC90603D5B3F863
:10065000F01D490715D4F2B993F80C2ED3F8083ED3
:1006600052B143B120B11A689B88138370473BB3E2
:100670001A689B885383704780F00100002BF1D1EA
:10068000F9E7B2B993F80C2ED3F8083E002AEED160
:10069000002BE8D17047D3F8002E002AEBD058B1D8
:1006A0009268B3F8041E094BB3FBF1F35B101360BF
:1006B0007047D3F8002E22B1936800221A60704769
:1006C00070477047B0000010E8B6002040420F00AD
:1006D000BFF34F8F0549064BCA6802F4E06213432B
:1006E000CB60BFF34F8F00BFFDE700BF00ED00E020
:1006F0000400FA0508B572B600224FF0FF319300EE
:1007000003F1604303F561430132082AC3F8801006
:10071000C3F88011F3D1FFF7DBFF00BF012108B55B
:100720000846F4F787F8FFF7E5FF00BF00B583B090
:100730000D49002200920091009B04330093009B1E
:100740001B68012B02D003B05DF804FB01920191FC
:10075000019B064904330193019B1A600B6883F3E4
:1007600008884B689847FEE7502800400000FF1FAC
:1007700010B4EFF31183102282F31288094C0A4857
:1007800022684FF0E021013222608A69C0F8102E01
:100790000022C0F8142E0A69DBB283F311885DF8D9
:1007A000044B7047242A0020E8B6002030B4EFF351
:1007B0001182102383F312884FF0E023D2B299699B
:1007C000186910F4803F0D481EBF0121C0F8141EA7
:1007D00099690B4B1D68D0F8143E82F311880948C3
:1007E00004684FF47A7202FB04F02B44401A002193
:1007F000B0FBF4F030BCE3FB02017047E8B6002028
:10080000242A0020AC360020124B5B68C3F3080397
:10081000FBB9EFF31183E3B930B40F4A0F4C4FF03B
:10082000E02C1368DCF8180011688B42F9D1D4F879
:10083000101E8842F5D80A4A15684FF47A7404FBF2
:1008400005F20021101AB0FBF5F0E3FB040130BC07
:100850007047ABE700ED00E0242A0020E8B6002056
:10086000AC36002090B170B5461EFFF7CDFF0446B0
:100870000D46FFF7C9FF001B61EB0501B0F57A7F5C
:1008800071F10001F5D3013EEFD270BD704700BF9A
:1008900070B5006801220921F8F710FF6426FFF700
:1008A000B3FF04460D46FFF7AFFF001B61EB0501E8
:1008B000B0F57A7F71F10001F5D3013EEFD170BD43
:1008C0002DE9804883B0431C0193DFF83C810A2363
:1008D0000093D8F89C10D8F8D830B8F8A000B8F831
:1008E000DC20DDF804B048834FF0320A1A834FF061
:1008F0000509D8F89C30B8F8A02059690A4214BFFD
:100900005A831A83D8F8D830B8F8DC2059690A42DB
:1009100014BF5A831A830120FFF792FE56465746AA
:10092000FFF772FF04460D46FFF76EFF001B61EBF9
:100930000501B0F57A7F71F10001F5D3013FEFD1E8
:10094000D8F89C30B8F8A02059690A4214BF5A83DD
:100950001A83D8F8D830B8F8DC2059690A4214BF95
:100960005A831A830020FFF76BFEFFF74DFF044602
:100970000D46FFF749FF001B61EB0501B0F57A7FDB
:1009800071F10001F5D3013EEFD1B9F1000F1CD098
:10099000B9F10109ADD14FF4FA76FFF735FF0446FE
:1009A0000D46FFF731FF001B61EB0501B0F57A7FC3
:1009B00071F10001F5D3013EEFD14FF0FA0ABBF11E
:1009C000000F07D04FF0000993E70BF1FF3BBBF19D
:1009D000000FF7D14FF47A76FFF716FF04460D4665
:1009E000FFF712FF001B61EB0501B0F57A7F71F193
:1009F0000001F5D3013EEFD1009B013B00937FF452
:100A000068AFFFF78BFE00BF2C2B002018B10368E6
:100A10005B6903B11847704718B103681B6A03B1DB
:100A200018470020704700BF38B50B4D0C4620B169
:100A30000368DB6A0BB1984760B90020C4E9000085
:100A4000C4E90200C4E906552D2230232061227535
:100A500084F8203038BD00BFF44409080178F9B1AA
:100A6000F8B5104F0546002602E015F8011FB1B198
:100A7000D7F8184E637A5A1C2344D2B26272997224
:100A8000237A9342F1D804F10A01002AEDD0D4E987
:100A900000309847667215F8011F0029E8D1F8BDAB
:100AA000704700BFE8B6002070B5124C05460E46F0
:100AB0001148FFF7D3FF2A461049D4F8180E3346E1
:100AC0006AF008FFD4F8185E6A7A32B12B68686859
:100AD00005F10A01984700236B7294F81C3E3BB164
:100AE00094F81E3E0122134484F81D2E84F81E3E05
:100AF00070BD00BFE8B60020F4E7080859E300081D
:100B00000FB470B582B006A951F8040B0191FFF73C
:100B1000CBFF0E48FFF7A2FF0D4BB3F8206E36B99E
:100B200002B0BDE8704004B07047013EF8D0FFF756
:100B30006BFE04460D46FFF767FE001B61EB0501E7
:100B4000B0F57A7F71F10001F5D3EEE7D8E8080837
:100B5000E8B60020D8B10378CBB12DE9F04F87B0CB
:100B6000714905AA70F0F9FD8246002800F0D08096
:100B70000024DFF8F4B16C4EA1462546A0464FF0A4
:100B8000FF37032C32D8DFE804F0686D2104674892
:100B9000B6E750466BF0ECF8032868D19AF80020CD
:100BA000382A64D19AF80120452A00F083804E2A21
:100BB0005DD100229AF80230312B00F08B80322B6D
:100BC00055D149EA020242F002090FE05946504667
:100BD00072F027FE002876D045F0010554495046B2
:100BE00072F01FFE002867D045F0020505AA3146C5
:100BF000002070F0B2FD013482460028C1D178B2E5
:100C00004C4A002392F90010814233D00133052B66
:100C100002F10C02F6D1B8F1000F5ED0002D08BF32
:100C200003250023EDB2CDE90085CDF808901A46E2
:100C300019462EF08DFB0446002870D03E484246EF
:100C40003946F7F7EFFC39463C48F7F7EBFC3C4BED
:100C50002146D3F8A80166F097F85046F8F78EFAC7
:100C60000746C3E75046F8F789FA8046BEE74FF0DB
:100C7000FF09BBE7334A03EB430302EB8303D3F8DB
:100C8000284E002CC7D030483946F7F7CBFC15B1B9
:100C90006179A94228D1B9F1000F02D0A179494563
:100CA0002CD1E36A002BCED02848F7F7BBFC0023F9
:100CB000E362C8E704227DE72549504672F0B1FDA2
:100CC000002891D192E72349504672F0AAFD0028EE
:100CD00082D183E749EA020988E71F483946F7F7D6
:100CE000A1FC07B0BDE8F08F2A461C48F7F79AFC34
:100CF0002368E9B29B6920469847CCE74A461848E2
:100D0000F7F790FC23684946DB6920469847C8E717
:100D100081464FF0FF305546D046074670E73946CA
:100D20001048F7F77FFCDCE75448090800E808089A
:100D300010E808080CC5002060E80808F4E8080876
:100D4000F0A50020E8B6002080E80808DCE80808E4
:100D500014E808084018090818E8080898E808087E
:100D6000B8E8080840E808080CE8080890B32DE93E
:100D7000F04F037887B005462BB300F100404F4C8D
:100D80000138294603E09F4228D1814212D011F850
:100D9000013BA3F14102192A14F8012BA2F14106EB
:100DA00098BF2033192E02F12007ECD99A4215D1B1
:100DB000002BEAD1424B00225A605A73A3F80B2051
:100DC00007B0BDE8F08F0021012007B0BDE8F04F6B
:100DD00066F084B80021012066F080B8394C2946BD
:100DE00003E09F421AD1814212D011F8013BA3F1D6
:100DF0004102192A14F8012BA2F1410698BF2033B1
:100E0000192E02F12007ECD99A4207D1002BEAD122
:100E1000012007B0BDE8F04F56F0B2BF2A4C29467A
:100E200003E09F4256D1814212D011F8013BA3F159
:100E30004102192A14F8012BA2F1410698BF203370
:100E4000192E02F12007ECD99A4243D1002BEAD1A6
:100E50001B4C00231D4694F90B0023712A46A4F570
:100E6000626393F8D6140129A1F1030608D0052E78
:100E700006D905B1E072154807B0BDE8F04F3FE66E
:100E800093F8D714A52903F1140303D00132782A6B
:100E9000E7D1EEE7012803D0013840B20125F5E79C
:100EA0000B49207100230132627181F8603EE372C8
:100EB00007B0BDE8F04F56F0C5BF00BF24E90808F1
:100EC000F0B500202CE908085C0C090800E80808C7
:100ED000E8B60020DFF8F4B22846F8F74FF99BF99E
:100EE00060AE0AFA80F6772E074600F2DC802846CC
:100EF000202172F046FC0446002800F0528103785D
:100F0000202B03D114F8013F202BFBD02046F8F70B
:100F100035F901255FFA80F82046202172F031FC76
:100F20000446002800F01C810378202B03D114F81C
:100F3000013F202BFBD02046F8F720F90135019026
:100F4000EDB22046202172F01CFC0446002800F07F
:100F500005810378202B03D114F8013F202BFBD00F
:100F60002046F8F70BF901350290EDB2204620211A
:100F700072F007FC0446002800F020810378202B43
:100F800003D114F8013F202BFBD02046F8F7F6F8E8
:100F900001350390EDB22046202172F0F2FB0446A9
:100FA000002800F009810378202B03D114F8013FB9
:100FB000202BFBD02046F8F7E1F8013503B204936B
:100FC000EDB22046202172F0DCFB0446002800F040
:100FD000EB800378202B03D114F8013F202BFBD0AA
:100FE0002046F8F7CBF820210346204605931CB293
:100FF00072F0C7FB0135059BEDB2024600285AD0BE
:101000001378202B03D112F8013F202BFBD0104680
:101010000592F8F7B3F8059A0FFA80F920211046E7
:1010200072F0AFFB00284DD00378202B03D110F8CD
:10103000013F202BFBD0F8F7A1F805F0FD05042DAA
:1010400008BFC0B27FF417AFB8F1010F0AD9B8F1E9
:10105000040F07D0A8F10503032B03D9B8F1030F40
:101060007FF409AF20B1A52858D048287FF403AFFA
:10107000002E39D1524B019AC3F8A426029AC3F824
:10108000A826039AC3F8AC26049A83F8B686A3F878
:10109000B026A3F8B246A3F8B49683F8B70603F5D2
:1010A0008053DE728CE6474947487723002207B019
:1010B000BDE8F04F24E5062D7FF4DDAE81461446F1
:1010C000D8B2C1E7052D7FF4D6AEB8F1010FCFD964
:1010D000B8F1040FCCD0A8F10503032BC8D9B8F19F
:1010E000030F7FF4C8AEC3E7354B019A06EB8606C3
:1010F00003EB8603C3F8A426029AC3F8A826039A32
:10110000C3F8AC26049A83F8B686A3F8B026A3F8F1
:10111000B246A3F8B49683F8B70651E616BB284B3F
:10112000019AC3F8A426029AC3F8A826039AC3F822
:10113000AC26049AA3F8B026A3F8B24683F8B68684
:10114000A3F8B49683F8B706012203F580540AF198
:1011500001033B448BF8603EE27231E6029005E702
:101160000190EEE6164A019906EB860602EB86032D
:10117000A3F8B24602F58054C3F8A416E27A0299A5
:10118000C3F8A8160399C3F8AC160132049983F882
:10119000B686A3F8B016A3F8B49683F8B70652B291
:1011A000D5E705468046B7E6202172F0EAFA024606
:1011B00000287FF425AF5EE6049002E70390EAE69C
:1011C000F0A5002034E9080840E90808E8B6002046
:1011D0002DE9F04782B03C4901AA70F0BEFA002820
:1011E00063D04FF0000A4FF0FF34374DD1465646DA
:1011F000D0462746BAF1040F37D8DFE80AF0423C60
:10120000310B03000378482B41D0562B2DD14FF0E2
:10121000010904E0F7F7B2FF3F28064625D8002071
:1012200001AA29460AF1010A70F097FA0028E1D1D3
:10123000BAF1040F2ED0BAF1050F40D1234AB30101
:10124000A62103F47C6308F03F0801FB074443EA4E
:10125000080302EB440243EA4933A2F8643E07E084
:10126000F7F78CFF3F288046D9D91948FFF748FC8B
:1012700002B0BDE8F087F7F781FFA5280446CED974
:10128000F3E7F7F77BFF03280746C8D9EDE74FF0F0
:101290000009C4E70D4AA62303FB074302EB4303FF
:1012A000B3F8649EC9F34039C9E74FF0FF373C46B5
:1012B000084923463A46012065F09CFED8E7BAF17A
:1012C000030FD2D0F4E700BF54480908E8B6002065
:1012D00000E808084CC5002080B51A48FFF7BEFB9F
:1012E0001948FFF7BBFB194BD3F8184E627A32B19D
:1012F0002146606851F80A3B984700236372144BFB
:10130000D3F8A8713B6838465B699847B0B90A269C
:10131000FFF77AFA04460D46FFF776FA001B61EBF9
:101320000503B0F57A7F73F10003F5D3013EEFD1E9
:101330003B6838465B6998470028E8D001200AF0EE
:10134000C5FA00BF60E908087CE90808E8B6002093
:10135000F0A50020174B93F89C22012A00D070477B
:1013600010B593F8A122062A84B00FD00A2A07D11B
:1013700034F0B8FB104804B0BDE81040FFF76EBB76
:101380000E4804B0BDE81040FFF768BBD3F8BC427C
:101390004CB10B4A07CA01AB03C301A91A7020461E
:1013A0000922FFF72BF9074804B0BDE81040FFF70A
:1013B00055BB00BFE0C7002098E9080888E9080885
:1013C000D0E90808B4E9080880B53048304FFFF785
:1013D00045FB3048FFF742FBB7F8206E002E45D1A1
:1013E000D7F8184E627A32B12146606851F80A3B4C
:1013F000984700236372284B284A0025157083F80C
:10140000C052C3F8005324F013FC2548FFF726FB15
:10141000D7F8184E627A2AB12146606851F80A3B23
:10142000984765721F4BD3F8A8713B6838465B69D3
:101430009847B0B90A26FFF7E7F904460D46FFF7CB
:10144000E3F9001B61EB0503B0F57A7F73F100034C
:10145000F5D3013EEFD13B6838465B6998470028D9
:10146000E8D000200AF032FA013EB9D0FFF7CCF9FB
:1014700004460D46FFF7C8F9001B61EB0501B0F506
:101480007A7F71F10001F5D3EEE700BFDCE90808CF
:10149000E8B60020D8E80808E0C70020BC5F0020BC
:1014A0007CE90808F0A50020F0B5394C94F81C3E02
:1014B00091B01BB194F81D3E002B53D1354D3648E9
:1014C000FFF7CCFA012385F8073385F84033F7F7A7
:1014D000F1FE40B9F7F7EEFE28B9F7F7EBFE10B9C9
:1014E0000520FFF7EDF9F7F771FE0028F8D02B4B38
:1014F0002B481A68C5F814230026012385F8406399
:1015000085F8076385F83633FFF7A8FAD4F8184E44
:10151000627A2AB12368606804F10A01984766720A
:10152000204BD3F8A8713B6838465B699847B0B93F
:101530000A26FFF769F904460D46FFF765F9001B17
:1015400061EB0501B0F57A7F71F10001F5D3013E41
:10155000EFD13B6838465B6998470028E8D0002007
:101560000AF0B4F994F81E2E0F4901A8F7F776F89F
:1015700001A8FFF7C5FA0D48FFF7C2FA002384F867
:101580001C3E84F81D3E84F81E3E11B0F0BD00BF25
:10159000E8B60020E0C700206CEA0808242A0020F2
:1015A0007CE90808F0A5002008EA08084CEA0808C9
:1015B00070B50C48FFF752FA0B4BB3F8206E16B912
:1015C00070BD013EFCD0FFF71FF904460D46FFF742
:1015D0001BF9001B61EB0501B0F57A7F71F1000189
:1015E000F5D3EEE7D8E80808E8B6002070B52D4935
:1015F00090B00522044672F0D1F838BB2A4C94F81A
:101600001C3EDBB12948FFF729FA2948FFF726FAE3
:10161000B4F8206E1EB910B070BD013EFBD0FFF7CC
:10162000F3F804460D46FFF7EFF8001B61EB0501E8
:10163000B0F57A7F71F10001F5D3EEE7012284F86D
:101640001C2E84F81D3E84F81E3EDBE71949032258
:10165000204672F0A3F8F0B9134C94F81C3E13B175
:1016600094F81D3E6BB91448FFF7F8F9FFF7A0FF97
:10167000002384F81C3E84F81D3E84F81E3E10B002
:1016800070BD94F81E2E0D4901A8F6F7E7FF01A8DA
:10169000FFF736FAECE70A4810B0BDE87040FFF7F4
:1016A0002FBA00BF74EA0808E8B600207CEA0808F0
:1016B000D8E80808140D090894EA080808EA080898
:1016C000A8EA080870B504460F48FFF7C7F9204696
:1016D000FFF7C4F90D48FFF7C1F90D4BB3F8206EC1
:1016E00016B970BD013EFCD0FFF78EF804460D46DA
:1016F000FFF78AF8001B61EB0501B0F57A7F71F105
:101700000001F5D3EEE700BFB8EA0808D8E80808FA
:10171000E8B60020800601D5002933D10CB470B59D
:10172000194C1A49D4F8180E82B007AB069A0193E7
:101730006AF0D0F8D4F8185E6A7A32B12B6868681B
:1017400005F10A01984700236B721148FFF786F9EB
:10175000B4F8206E3EB9012002B0BDE8704002B07E
:101760007047013EF7D0FFF74FF804460D46FFF7EC
:101770004BF8001B61EB0501B0F57A7F71F10001B8
:10178000F5D3EEE700207047E8B6002059E30008E3
:10179000D8E80808F0B5054683B040B304783CB3F8
:1017A00000F1004E424C0EF1FF3E014603E098422C
:1017B00032D1714513D011F8013BA3F14102192A2E
:1017C00014F8012BA2F1410C98BF2033BCF1190F82
:1017D00002F12000EBD99A421ED1002BE9D1354B02
:1017E000354AC3E9D122C3E9D32203B0F0BD044690
:1017F000324D334E35F8243005EB840200215288F7
:101800000120CDE90032234632460134FFF782FF42
:10181000042CEFD103B0F0BD2846F7F7AFFC032846
:10182000064639D82021284671F0ABFF044600282F
:101830003BD00378202B03D114F8013F202BFBD0A1
:101840002046F7F79BFC012705462021204671F032
:1018500098FFD8B10378202B03D110F8013F202B3B
:10186000FBD0F7F78BFC8FB1A5F2EE2240F2DC53F0
:101870009A420BD8A0F2EE229A4207D80D4B03EB06
:101880008603A3F84453A3F84603AEE70D4803B01C
:10189000BDE8F040FFF734B90B490C4803230022A0
:1018A00003B0BDE8F040FFF72BB905460746CCE78B
:1018B00024E90808E0C70020E803D00724CB002073
:1018C000C0EA080800E80808D4EA080840E908085F
:1018D0002DE9F04385B040B3037806462BB300F101
:1018E000004C564C0CF1FF3C014603E0984232D1CB
:1018F000614512D011F8013BA3F14102192A14F8F5
:10190000012BA2F1410598BF2033192D02F12000CF
:10191000ECD99A421FD1002BEAD14948602200211C
:1019200005B0BDE8F04371F065B8454D454E002463
:10193000D5E9012115F80C3B0093CDE9012123469F
:101940003246002101200134FFF7E4FE082CEFD1DC
:1019500005B0BDE8F0833046F7F710FCC3B2072BA3
:10196000054655D82021304671F00BFF044600286B
:1019700057D00378202B03D114F8013F202BFBD044
:101980002046F7F7FBFB071E18BF0127012620465C
:10199000202171F0F6FE044600284CD00378202B5D
:1019A00003D114F8013F202BFBD02046F7F7E6FBCC
:1019B00001368046F6B22046202171F0E2FE044650
:1019C00090B30378202B03D114F8013F202BFBD0D8
:1019D0002046F7F7D3FB0136814620212046F6B298
:1019E00071F0CFFE08B10136F6B2032E05D01648CD
:1019F00005B0BDE8F043FFF783B8144B6DB205EBBB
:101A0000450503EB8503C3E9D68983F854739FE743
:101A10000F4910480723002205B0BDE8F043FFF747
:101A20006FB806460746B2E7202171F0AAFEA1462C
:101A30000028D8D1DBE78046BDE700BF24E90808CD
:101A400034CB0020DCEA080800E80808E0C70020E2
:101A5000F4EA080840E90808F0B585B010B1037849
:101A60000446C3B9384C394E002594F8831294F8D3
:101A70008222B4F880320093CDE901212B46324610
:101A8000002101200135FFF745FE102D04F104046B
:101A9000EBD105B0F0BDF7F771FB0F2805463BDC35
:101AA0002046202171F06DFE044630B10378202BD2
:101AB00003D114F8013F202BFBD0254F2046F7F728
:101AC0005DFB3A8890424FF0000605F1A005034601
:101AD00018DC204A012E204602EB85022CD0022E73
:101AE00023D02C21A2F8B43371F04BFE50B1441C2A
:101AF00002372046F7F742FB3A88904206F101068A
:101B00000346E6DD104B1448002243F8252005B0BB
:101B1000BDE8F040FEF7F4BF104911480F23002242
:101B200005B0BDE8F040FEF7EBBF0A4A02EB8502C4
:101B300082F8B73305B0F0BD2C2182F8B63371F0CE
:101B400020FE0028D3D1DDE794CB002004EB080869
:101B500084430808E0C7002000E8080868F5080882
:101B600040E9080870B588B0002841D003780446E1
:101B7000002B3DD000252D2B54D0A3F13002092A93
:101B800050D9202B62D163780134002BF3D1052D7D
:101B9000BDF914305AD19AB2112A57D8BDF916108E
:101BA000A1F5FA7292B2B2F5FA6F4FD8BDF91800EA
:101BB000A0F5FA7292B2B2F5FA6F47D8BDF91A40A1
:101BC000A14243DCA04241DBBDF91C5005F17D027E
:101BD00092B2FA2A3AD8204A02EBC303A3F8A41619
:101BE000A3F8A606A3F8A84683F8AA5608B070BDC5
:101BF0001A4C1B4E002594F90600B4F90410B4F9F0
:101C0000022034F9083BCDE90210CDE90032002171
